:020000040800F2
:1000000000000220A9030008153D0008213D00085A
:10001000293D0008313D0008393D0008000000007E
:100020000000000000000000000000004D3D00083E
:10003000413D000800000000593D00088D450008C2
:10004000F9030008F9030008F9030008F9030008A0
:10005000F9030008F9030008F9030008F903000890
:10006000F9030008F9030008F9030008F903000880
:10007000F9030008F9030008F9030008F903000870
:10008000F9030008F9030008F9030008F903000860
:10009000F9030008F9030008F9030008F903000850
:1000A000F9030008F9030008F9030008F903000840
:1000B000F9030008653D0008793D0008F9030008D0
:1000C000F9030008F9030008F9030008F903000820
:1000D000F9030008F9030008F9030008F903000810
:1000E000F9030008F9030008F9030008F903000800
:1000F000F9030008F9030008F9030008F9030008F0
:10010000F9030008F9030008F9030008F9030008DF
:10011000F9030008F9030008F9030008F9030008CF
:10012000F9030008F9030008F9030008F9030008BF
:10013000F9030008F9030008F9030008F9030008AF
:10014000F9030008F9030008F9030008F90300089F
:10015000F9030008F9030008F9030008F90300088F
:10016000F9030008F9030008F9030008F90300087F
:10017000F9030008F9030008F90300080000000073
:10018000F9030008F9030008F9030008F90300085F
:10019000F9030008F9030008F9030008F90300084F
:1001A000F9030008F9030008F903000880B58EB0D0
:1001B00000AF40F6C803C2F200034BF6BA22CCF6F9
:1001C000DE221A6044F64C13C2F200034BF6BA2248
:1001D000CCF6DE221A6040F6C803C2F200033B638D
:1001E00044F65013C2F20003FB623B6BBB6207E0B4
:1001F000BB6A4FF000021A60BB6A03F10403BB62E2
:10020000FA6ABB6A9A42F3D840F6C803C2F2000306
:100210001B68002B06D144F64C13C2F200031B6886
:10022000002B00D0FEE740F20003C2F200034BF6C1
:10023000BA22CCF6DE221A6040F6C403C2F20003F2
:100240004BF6BA22CCF6DE221A604FF2D403C0F687
:1002500001037B6240F20003C2F200033B6240F6FE
:10026000C803C2F20003FB613B6ABB610BE07B6A1F
:100270001A68BB691A60BB6903F10403BB617B6A3E
:1002800003F104037B62FA69BB699A42EFD840F23A
:100290000003C2F200031A6845F27863C1F2342306
:1002A0009A420BD140F6C403C2F200031A6840F62A
:1002B000C403C2F200031B689A4200D0FEE707F0B5
:1002C000FBFF07F104023B461046194603F05CFCB5
:1002D00040F20042C0F6000240F20043C0F60003C4
:1002E000D31A4FEAA3037B614FF000033B610BE09D
:1002F00040F20043C0F600033A6953F822309847B1
:100300003B6903F101033B617A693B699A42EFDC87
:1003100040F20042C0F6000240F20043C0F6000383
:10032000D31A4FEAA3037B614FF000033B610BE05C
:1003300040F20043C0F600033A6953F82230984770
:100340003B6903F101033B617A693B699A42EFDC47
:100350007A683B681046194605F092F803467B63BD
:1003600040F20042C0F6000240F20043C0F6000333
:10037000D31A4FEAA303FB60FB68BB600DE0BB68C8
:1003800003F1FF3240F20043C0F6000353F822307D
:100390009847BB6803F1FF33BB60BB68002BEEDC02
:1003A000786B03F04DFC00BF80B500AFFFF7FEFE99
:1003B00080B400AFFEE700BF80B400AFFEE700BF2F
:1003C00080B400AFFEE700BF80B400AFFEE700BF1F
:1003D00080B400AFFEE700BF80B400AFFEE700BF0F
:1003E00080B400AFFEE700BF80B400AFFEE700BFFF
:1003F00080B400AFFEE700BF80B400AFFEE700BFEF
:1004000080B483B000AF786007F10C07BD4680BCB4
:10041000704700BF80B483B000AF786007F10C076D
:10042000BD4680BC704700BF80B582B000AF786029
:100430007B68002B02D14FF00103C4E07B681A688F
:100440004FF00003C4F201039A426CD07B681B6832
:10045000B3F1804F67D07B681A684FF48063C4F2B1
:1004600000039A425FD07B681A684FF40063C4F2BD
:1004700000039A4257D07B681A684FF44063C4F275
:1004800000039A424FD07B681A684FF48053C4F23D
:1004900000039A4247D07B681A684FF4A053C4F215
:1004A00000039A423FD07B681A684FF48063C4F21D
:1004B00001039A4237D07B681A684FF48043C4F234
:1004C00001039A422FD07B681A684FF48843C4F224
:1004D00001039A4227D07B681A684FF49043C4F214
:1004E00001039A421FD07B681A684FF4C053C4F2CC
:1004F00000039A4217D07B681A684FF4E053C4F2A5
:1005000000039A420FD07B681A684FF40053C4F27C
:1005100000039A4207D040F6F810C0F601004FF0F1
:10052000D10103F025FB7B689B68002B17D07B680B
:100530009B68102B13D07B689B68202B0FD07B68A7
:100540009B68402B0BD07B689B68602B07D040F6E4
:10055000F810C0F601004FF0D20103F009FB7B68F0
:100560001B69002B11D07B681B69B3F5807F0CD011
:100570007B681B69B3F5007F07D040F6F810C0F622
:1005800001004FF0D30103F0F3FA7B6893F83930A0
:10059000DBB2002B02D1786800F01AF87B684FF0CC
:1005A000020283F839207B681A687B6803F1040330
:1005B0001046194600F00AFA7B684FF0010283F8F2
:1005C00039204FF00003184607F10807BD4680BDEB
:1005D00080B483B000AF786007F10C07BD4680BCE3
:1005E000704700BF80B582B000AF78607B681A6842
:1005F0004FF00003C4F201039A426CD07B681B6881
:10060000B3F1804F67D07B681A684FF48063C4F2FF
:1006100000039A425FD07B681A684FF40063C4F20B
:1006200000039A4257D07B681A684FF44063C4F2C3
:1006300000039A424FD07B681A684FF48053C4F28B
:1006400000039A4247D07B681A684FF4A053C4F263
:1006500000039A423FD07B681A684FF48063C4F26B
:1006600001039A4237D07B681A684FF48043C4F282
:1006700001039A422FD07B681A684FF48843C4F272
:1006800001039A4227D07B681A684FF49043C4F262
:1006900001039A421FD07B681A684FF4C053C4F21A
:1006A00000039A4217D07B681A684FF4E053C4F2F3
:1006B00000039A420FD07B681A684FF40053C4F2CB
:1006C00000039A4207D040F6F810C0F6010040F24D
:1006D0005B1103F04DFA7B681B687A681268D26878
:1006E00042F00102DA607B681B687A68126812685F
:1006F00042F001021A604FF00003184607F10807A4
:10070000BD4680BD80B582B000AF78607B681B6855
:100710001B6903F00203002B27D07B681B68DB6892
:1007200003F00203002B20D07B681B687A681268F4
:10073000126922F002021A617B684FF001021A76F8
:100740007B681B689B6903F00303002B03D0786868
:1007500000F01EF905E0786800F010F9786800F004
:1007600021F97B684FF000021A767B681B681B69D1
:1007700003F00403002B27D07B681B68DB6803F0C1
:100780000403002B20D07B681B687A68126812690A
:1007900022F004021A617B684FF002021A767B682D
:1007A0001B689B6903F44073002B03D0786800F04A
:1007B000EFF805E0786800F0E1F8786800F0F2F80A
:1007C0007B684FF000021A767B681B681B6903F098
:1007D0000803002B27D07B681B68DB6803F0080345
:1007E000002B20D07B681B687A681268126922F09F
:1007F00008021A617B684FF004021A767B681B6856
:100800009B6903F00303002B03D0786800F0C0F865
:1008100005E0786800F0B2F8786800F0C3F87B680B
:100820004FF000021A767B681B681B6903F0100307
:10083000002B27D07B681B68DB6803F01003002BBC
:1008400020D07B681B687A681268126922F0100257
:100850001A617B684FF008021A767B681B689B69F7
:1008600003F44073002B03D0786800F091F805E0A2
:10087000786800F083F8786800F094F87B684FF0AF
:1008800000021A767B681B681B6903F00103DBB268
:10089000002B12D07B681B68DB6803F00103DBB21E
:1008A000002B0AD07B681B687A681268126922F0F4
:1008B00001021A61786806F085FD7B681B681B6978
:1008C00003F08003002B11D07B681B68DB6803F00A
:1008D0008003002B0AD07B681B687A681268126953
:1008E00022F080021A617868FFF794FD7B681B682C
:1008F0001B6903F04003002B11D07B681B68DB6889
:1009000003F04003002B0AD07B681B687A681268EA
:10091000126922F040021A61786800F04DF87B6895
:100920001B681B6903F02003002B11D07B681B6838
:10093000DB6803F02003002B0AD07B681B687A6811
:100940001268126922F020021A617868FFF758FDD8
:1009500007F10807BD4680BD80B483B000AF786062
:100960007B681B687A681268126922F001021A61BA
:1009700007F10C07BD4680BC704700BF80B483B050
:1009800000AF786007F10C07BD4680BC704700BF20
:1009900080B483B000AF786007F10C07BD4680BC1F
:1009A000704700BF80B483B000AF786007F10C07D8
:1009B000BD4680BC704700BF80B483B000AF786094
:1009C00007F10C07BD4680BC704700BF80B485B0FE
:1009D00000AF786039604FF00003FB607B681B68F4
:1009E000FB607A684FF00003C4F201039A421FD003
:1009F0007B68B3F1804F1BD07A684FF48063C4F2F8
:100A000000039A4214D07A684FF40063C4F20003E2
:100A10009A420DD07A684FF44063C4F200039A42C0
:100A200006D07A684FF48063C4F201039A4202D17F
:100A30004FF0010301E04FF00003002B08D0FB68EA
:100A400023F07003FB603B685B68FA681343FB604C
:100A50007A684FF00003C4F201039A4249D07B68E0
:100A6000B3F1804F45D07A684FF48063C4F200033D
:100A70009A423ED07A684FF40063C4F200039A426F
:100A800037D07A684FF44063C4F200039A4230D002
:100A90007A684FF48063C4F201039A4229D07A68DD
:100AA0004FF48043C4F201039A4222D07A684FF493
:100AB0008843C4F201039A421BD07A684FF49043F2
:100AC000C4F201039A4214D07A684FF4C053C4F2BE
:100AD00000039A420DD07A684FF4E053C4F2000349
:100AE0009A4206D07A684FF40053C4F200039A4247
:100AF00002D14FF0010301E04FF00003002B08D0BA
:100B0000FB6823F44073FB603B68DB68FA681343BF
:100B1000FB607B68FA681A603B689A687B68DA62F7
:100B20003B681A687B689A627A684FF00003C4F2E7
:100B300001039A4206D07A684FF48063C4F201033D
:100B40009A4202D14FF0010301E04FF00003002B65
:100B500003D03B681A697B681A637B684FF0010217
:100B60005A6107F11407BD4680BC704780B582B05A
:100B700000AF78607B68002B02D14FF0010332E1B7
:100B80007B685B68002B0CD07B685B68B3F5827F69
:100B900007D040F62820C0F601004FF0A50102F072
:100BA000E7FF7B689B68002B11D07B689B68B3F5DF
:100BB000806F0CD07B689B68B3F5004F07D040F680
:100BC0002820C0F601004FF0A60102F0D1FF7B689B
:100BD000DB68B3F5006F0BD07B68DB68002B07D0B8
:100BE00040F62820C0F601004FF0A70102F0C0FF38
:100BF0007B681B69002B0BD07B681B69022B07D01D
:100C000040F62820C0F601004FF0A80102F0B0FF26
:100C10007B685B69002B0BD07B685B69012B07D07D
:100C200040F62820C0F601004FF0A90102F0A0FF15
:100C30007B689B69B3F5007F10D07B689B69002BB4
:100C40000CD07B689B69B3F5802F07D040F6282035
:100C5000C0F601004FF0AA0102F08AFF7B68DB6951
:100C6000002B23D07B68DB69082B1FD07B68DB69F6
:100C7000102B1BD07B68DB69182B17D07B68DB69D6
:100C8000202B13D07B68DB69282B0FD07B68DB69B6
:100C9000302B0BD07B68DB69382B07D040F628203F
:100CA000C0F601004FF0AB0102F062FF7B681B6AE7
:100CB000002B0BD07B681B6A802B07D040F62820C6
:100CC000C0F601004FF0AC0102F052FF7B685B6A96
:100CD000002B0BD07B685B6A102B07D040F62820D6
:100CE000C0F601004FF0AD0102F042FF7B689B6A45
:100CF000002B0CD07B689B6AB3F5005F07D040F6F1
:100D00002820C0F601004FF0AE0102F031FF7B68F1
:100D1000DB6A002B05D07B68DA6A4FF6FF739A42D4
:100D200007D940F62820C0F601004FF0AF0102F0CD
:100D30001FFF7B6893F84930DBB2002B02D1786843
:100D400000F056F87B684FF0020283F849207B6878
:100D50001B687A681268126822F040021A607B6889
:100D60001B687A6851687A68926811437A68D26819
:100D700011437A68126911437A68526911437A689B
:100D8000926902F4007211437A68D26911437A6859
:100D9000126A11437A68926A0A431A607B681B6878
:100DA0007A6892694FEA124202F004017A68526A44
:100DB0000A435A607B681B687A68D26A1A617B684A
:100DC0001B687A681268D26922F40062DA617B6873
:100DD0004FF0000283F84A207B684FF0010283F84D
:100DE00049204FF00003184607F10807BD4680BDB3
:100DF00080B483B000AF786007F10C07BD4680BCBB
:100E0000704700BF80B584B000AFF860B9603B6048
:100E10001346FB80FB6893F84930DBB2012B40F0AE
:100E20004F81BB68002B02D0FB88002B02D14FF012
:100E3000010347E1FB689B68002B0CD0FB689B68B3
:100E4000B3F5004F07D040F62820C0F601004FF45C
:100E5000AE7102F08DFEFB6893F84830012B02D191
:100E60004FF002032EE1FB684FF0010283F84820A7
:100E7000FB684FF0120283F84920FB684FF0000234
:100E800083F84A20FB68BA681A63FB68FA889A8676
:100E9000FB68FA88DA86FB684FF000025A64FB6848
:100EA0004FF000021A64FB684FF000029A87FB685B
:100EB0004FF00002DA87FB689B6AB3F5005F0FD141
:100EC000FB681B68FA681268126822F400521A6004
:100ED000FB681B68FA681268126842F400521A60D4
:100EE000FB689B68B3F5004F07D1FB681B68FA6885
:100EF0001268126842F480421A60FB681B681B6823
:100F000003F04003002B07D1FB681B68FA681268E6
:100F1000126842F040021A60FB68DB68002B42D185
:100F2000FB681A68FB681B6B1978D16003F101023A
:100F3000FB681A63FB68DB8E03F1FF339AB2FB6830
:100F4000DA861EE0F8684FF002014FF000023B68BD
:100F500000F0BEF80346002B02D04FF00303B1E0CF
:100F6000FB681A68FB681B6B1978D16003F10102FA
:100F7000FB681A63FB68DB8E03F1FF339AB2FB68F0
:100F8000DA86FB68DB8E002BDCD1FB689B6AB3F54D
:100F9000005F4ED1FB681B68FA681268126842F461
:100FA00080521A6045E0FB681B68FA68126B128871
:100FB000DA60FB681B6B03F10202FB681A63FB68D3
:100FC000DB8E03F1FF339AB2FB68DA8620E0F86823
:100FD0004FF002014FF000023B6800F079F8034641
:100FE000002B02D04FF003036CE0FB681B68FA682B
:100FF000126B1288DA60FB681B6B03F10202FB685C
:101000001A63FB68DB8E03F1FF339AB2FB68DA8662
:10101000FB68DB8E002BDAD1FB689B6AB3F5005FBF
:1010200007D1FB681B68FA681268126842F48052A4
:101030001A60F8684FF002014FF000023B6800F0C0
:1010400047F80346002B0CD0FB6893F84A30DBB21C
:1010500043F02003DAB2FB6883F84A204FF0030321
:1010600030E0F8684FF080014FF001023B6800F07B
:101070002FF80346002B0CD0FB6893F84A30DBB204
:1010800043F02003DAB2FB6883F84A204FF00303F1
:1010900018E0FB689B68002B05D1FB681B68DB68C8
:1010A000FB681B689B68FB684FF0010283F84920CE
:1010B000FB684FF0000283F848204FF0000301E086
:1010C0004FF00203184607F11007BD4680BD00BF70
:1010D00080B586B000AFF860B9603B601346FB7125
:1010E0004FF000037B6102F037FD02463B68D318E6
:1010F0007B61FB79002B40F083803BE03B68B3F1E0
:10110000FF3F37D002F028FD02467B699A4231D377
:10111000FB681B68FA681268526822F0E0025A60A5
:10112000FB681B68FA681268126822F040021A60B5
:10113000FB689B6AB3F5005F0FD1FB681B68FA6818
:101140001268126822F400521A60FB681B68FA6881
:101150001268126842F400521A60FB684FF00102F4
:1011600083F84920FB684FF0000283F848204FF0D5
:10117000030351E0FB681B689B681A46BB681A4072
:10118000BB689A42BAD145E03B68B3F1FF3F38D023
:1011900002F0E2FC02467B699A4232D3FB681B688C
:1011A000FA681268526822F0E0025A60FB681B6815
:1011B000FA681268126822F040021A60FB689B6AA3
:1011C000B3F5005F0FD1FB681B68FA6812681268FC
:1011D00022F400521A60FB681B68FA6812681268F1
:1011E00042F400521A60FB684FF0010283F8492074
:1011F000FB684FF0000283F848204FF003030BE038
:1012000000BFFB681B689B681A46BB681A40BB6836
:101210009A42B9D04FF00003184607F11807BD46AF
:1012200080BD00BF80B483B000AF03463960FB715E
:1012300097F90730002B10DA4FF46D43CEF200031C
:10124000FA7902F00F02A2F104013A68D2B24FEA31
:101250000212D2B25B181A760DE04FF46143CEF25F
:10126000000397F907103A68D2B24FEA0212D2B2DD
:101270005B1883F8002307F10C07BD4680BC70475C
:1012800080B582B000AF78607B6803F1FF326FF009
:101290007F439A4202D94FF001031DE04EF2100342
:1012A000CEF200037A6802F1FF325A604FF0FF304D
:1012B0004FF00F01FFF7B6FF4EF21003CEF200031E
:1012C0004FF000029A604EF21003CEF200034FF08E
:1012D00007021A604FF00003184607F10807BD46E1
:1012E00080BD00BF90B595B000AF78604FF00003AF
:1012F000FB647B681B680F2B07D940F66820C0F69B
:1013000001004FF49D7102F033FC7B681B6803F011
:101310000103DBB2002B00F0A6807B685B68002B2A
:101320000FD07B685B68012B0BD07B685B68052B5B
:1013300007D040F66820C0F6010040F23F1102F0ED
:1013400017FC4FF46053C4F202039B6803F00C03D4
:10135000042B11D04FF46053C4F202039B6803F0D6
:101360000C03082B18D14FF46053C4F202035B68DE
:1013700003F48003002B0FD04FF46053C4F2020338
:101380001B6803F40033002B6CD07B685B68012B77
:1013900068D04FF0010358E343F60203C4F202039E
:1013A0004FF000021A7002F0D7FB034603F59C537E
:1013B00003F10803FB6408E002F0CEFB0246FB6C7D
:1013C0009A4202D34FF003033FE34FF46053C4F259
:1013D00002031B6803F40033002BEDD143F6020334
:1013E000C4F202037A685268D2B21A707B685B68F2
:1013F000012B1BD102F0B0FB034603F59C5303F114
:101400000803FB6408E002F0A7FB0246FB6C9A426B
:1014100002D34FF0030318E34FF46053C4F2020306
:101420001B6803F40033002BEDD01CE002F094FBAA
:10143000034603F59C5303F10803FB6408E002F044
:101440008BFB0246FB6C9A4202D34FF00303FCE293
:101450004FF46053C4F202031B6803F40033002B03
:10146000EDD100E000BF7B681B6803F00203002B96
:1014700000F0AE807B68DB68002B0BD07B68DB68FC
:10148000012B07D040F66820C0F6010040F27F1122
:1014900002F06EFB7B681B691F2B07D940F66820A2
:1014A000C0F601004FF4C07102F062FB4FF46053CC
:1014B000C4F202039B6803F00C03002B11D04FF41D
:1014C0006053C4F202039B6803F00C03082B18D18D
:1014D0004FF46053C4F202035B6803F48003002BF3
:1014E0000FD14FF46053C4F202031B6803F00203F0
:1014F000002B6CD07B68DB68012B68D04FF00103B8
:10150000A3E27B68DB68002B40D04FF00003C4F2FD
:1015100047234FF001021A6002F01EFB034603F15D
:101520006403FB6408E002F017FB0246FB6C9A427E
:1015300002D34FF0030388E24FF46053C4F2020376
:101540001B6803F00203002BEDD04FF46053C4F28C
:1015500002034FF46052C4F20202126822F0F80152
:101560007A6810694FF0F802BA64BA6C92FAA2F481
:101570007C647A6C3A643A6CB2FA82F4FC63FA6B7B
:10158000D2B200FA02F20A431A6021E04FF00003DF
:10159000C4F247234FF000021A6002F0DDFA03465E
:1015A00003F16403FB6408E002F0D6FA0246FB6C28
:1015B0009A4202D34FF0030347E24FF46053C4F260
:1015C00002031B6803F00203002BEDD100E000BF13
:1015D0007B681B6803F00803002B54D07B685B69B1
:1015E000002B0BD07B685B69012B07D040F668208D
:1015F000C0F601004FF4DC7102F0BAFA7B685B6957
:10160000002B20D04FF46863C4F247234FF001024F
:101610001A6002F0A1FA034603F16403FB6408E0D8
:1016200002F09AFA0246FB6C9A4202D34FF003038F
:101630000BE24FF46053C4F202035B6F03F002034A
:10164000002BEDD01FE04FF46863C4F247234FF046
:1016500000021A6002F080FA034603F16403FB649F
:1016600008E002F079FA0246FB6C9A4202D34FF08E
:101670000303EAE14FF46053C4F202035B6F03F02B
:101680000203002BEDD17B681B6803F00403002BE1
:1016900000F0AA807B689B68002B0FD07B689B685A
:1016A000012B0BD07B689B68052B07D040F6682088
:1016B000C0F601004FF4F17102F05AFA4FF4605392
:1016C000C4F202034FF46052C4F20202126C42F000
:1016D00080521A644FF4E043C4F200034FF4E04236
:1016E000C4F20002126842F480721A6002F034FA06
:1016F000034603F16403FB6408E002F02DFA02469E
:10170000FB6C9A4202D34FF003039EE14FF4E04397
:10171000C4F200031B6803F48073002BEDD043F682
:101720007003C4F202034FF000021A7002F014FAC0
:10173000034603F59C5303F10803FB6408E002F041
:101740000BFA0246FB6C9A4202D34FF003037CE192
:101750004FF46053C4F202031B6F03F00203002B2B
:10176000EDD143F67003C4F202037A689268D2B2F4
:101770001A707B689B68012B1BD102F0EDF90346C0
:1017800003F59C5303F10803FB6408E002F0E4F95D
:101790000246FB6C9A4202D34FF0030355E14FF42B
:1017A0006053C4F202031B6F03F00203002BEDD061
:1017B0001AE002F0D1F9034603F59C5303F1080344
:1017C000FB6408E002F0C8F90246FB6C9A4202D3BF
:1017D0004FF0030339E14FF46053C4F202031B6F6F
:1017E00003F00203002BEDD17B689B69002B0FD027
:1017F0007B689B69012B0BD07B689B69022B07D010
:1018000040F66820C0F6010040F2262102F0B0F94F
:101810007B689B69002B00F016814FF46053C4F283
:1018200002039B6803F00C03082B00F009817B681E
:101830009B69022B40F0E3807B68DB69002B0CD0B6
:101840007B68DB69B3F5800F07D040F66820C0F6EF
:10185000010040F22F2102F08BF97B681B6A3F2BBD
:1018600007D940F66820C0F601004FF40C7102F071
:101870007FF97B685B6ABF2B04D97B685B6AB3F531
:10188000D87F07D940F66820C0F6010040F2312128
:1018900002F06EF97B689B6A022B13D07B689B6A0F
:1018A000042B0FD07B689B6A062B0BD07B689B6A4E
:1018B000082B07D040F66820C0F6010040F2322124
:1018C00002F056F97B68DB6A032B03D97B68DB6A7D
:1018D0000F2B07D940F66820C0F6010040F23321F3
:1018E00002F046F94FF06003C4F247234FF00002C4
:1018F0001A6002F031F9034603F16403FB6408E067
:1019000002F02AF90246FB6C9A4202D34FF003031D
:101910009BE04FF46053C4F202031B6803F00073B2
:10192000002BEDD14FF46053C4F202037A68116AC0
:101930007A68506A47F6C072BA63BA6B92FAA2F438
:101940007C637A6B3A633A6BB2FA82F4FC62FA6AAD
:10195000D2B200FA02F211437A68926A4FEA520256
:1019600002F1FF304FF44032BA62BA6A92FAA2F43E
:101970007C627A6A3A623A6AB2FA82F4FC61FA6983
:10198000D2B200FA02F211437A68D26911437A683E
:10199000D06A4FF07062BA61BA6992FAA2F47C61BF
:1019A0007A693A613A69B2FA82F4FC60FA68D2B2B2
:1019B00000FA02F20A4342F000525A604FF060030C
:1019C000C4F247234FF001021A6002F0C5F8034643
:1019D00003F16403FB6408E002F0BEF80246FB6C0E
:1019E0009A4202D34FF003032FE04FF46053C4F246
:1019F00002031B6803F00073002BEDD023E04FF0CF
:101A00006003C4F247234FF000021A6002F0A4F80A
:101A1000034603F16403FB6408E002F09DF802460C
:101A2000FB6C9A4202D34FF003030EE04FF4605375
:101A3000C4F202031B6803F00073002BEDD102E037
:101A40004FF0010301E04FF00003184607F154077F
:101A5000BD4690BD80B584B000AF786039604FF06E
:101A60000003FB607B681B68002B03D07B681B684E
:101A70000F2B07D940F66820C0F6010040F29621EE
:101A800002F076F83B68002B34D03B68012B31D054
:101A90003B68022B2ED03B68032B2BD03B68042BDA
:101AA00028D03B68052B25D03B68062B22D03B680D
:101AB000072B1FD03B68082B1CD03B68092B19D083
:101AC0003B680A2B16D03B680B2B13D03B680C2BC2
:101AD00010D03B680D2B0DD03B680E2B0AD03B6815
:101AE0000F2B07D040F66820C0F6010040F2972186
:101AF00002F03EF84FF47053C4F202031B6803F087
:101B00000F023B689A4280F0B7804FF47053C4F2E2
:101B100002033A68D2B21A704FF47053C4F202034F
:101B20001B6803F00F023B689A4202D04FF001039A
:101B300015E27B681B6803F00103DBB2002B00F0A9
:101B400051817B685B68002B0FD07B685B68012B41
:101B50000BD07B685B68022B07D040F66820C0F68C
:101B6000010040F2AD2102F003F87B685B68012BB5
:101B70000BD14FF46053C4F202031B6803F400332B
:101B8000002B1ED14FF00103E9E17B685B68022B5B
:101B90000BD14FF46053C4F202031B6803F00073CF
:101BA000002B0ED14FF00103D9E14FF46053C4F282
:101BB00002031B6803F00203002B02D14FF0010364
:101BC000CDE14FF46053C4F202034FF46052C4F20B
:101BD0000202926822F003017A6852680A439A600E
:101BE00001F0BAFF034603F59C5303F10803FB60C1
:101BF0007B685B68012B13D108E001F0ADFF024662
:101C0000FB689A4202D34FF00303A8E14FF46053FC
:101C1000C4F202039B6803F00C03042BEDD1E1E056
:101C20007B685B68022B1CD108E001F095FF02463F
:101C3000FB689A4202D34FF0030390E14FF46053E4
:101C4000C4F202039B6803F00C03082BEDD1C9E03A
:101C500001F082FF0246FB689A4203D34FF0030370
:101C60007DE100BF4FF46053C4F202039B6803F0B0
:101C70000C03002BECD1B5E07B681B6803F001037B
:101C8000DBB2002B00F09A807B685B68002B0FD0E2
:101C90007B685B68012B0BD07B685B68022B07D0ED
:101CA00040F66820C0F6010040F2F52101F060FF27
:101CB0007B685B68012B0BD14FF46053C4F20203C5
:101CC0001B6803F40033002B1ED14FF0010346E1E3
:101CD0007B685B68022B0BD14FF46053C4F20203A4
:101CE0001B6803F00073002B0ED14FF0010336E1A7
:101CF0004FF46053C4F202031B6803F00203002B8D
:101D000002D14FF001032AE14FF46053C4F2020301
:101D10004FF46052C4F20202926822F003017A6822
:101D200052680A439A6001F017FF034603F59C537B
:101D300003F10803FB607B685B68012B13D108E0AB
:101D400001F00AFF0246FB689A4202D34FF00303F8
:101D500005E14FF46053C4F202039B6803F00C03E7
:101D6000042BEDD12AE07B685B68022B1CD108E0D4
:101D700001F0F2FE0246FB689A4202D34FF00303E1
:101D8000EDE04FF46053C4F202039B6803F00C03D0
:101D9000082BEDD112E001F0DFFE0246FB689A420B
:101DA00003D34FF00303DAE000BF4FF46053C4F2F3
:101DB00002039B6803F00C03002BECD14FF470532B
:101DC000C4F202033A68D2B21A704FF47053C4F2EC
:101DD00002031B6803F00F023B689A4202D04FF0E7
:101DE0000103BCE07B681B6803F00203002B3AD0C0
:101DF0007B689B68002B27D07B689B68802B23D057
:101E00007B689B68902B1FD07B689B68A02B1BD0A6
:101E10007B689B68B02B17D07B689B68C02B13D066
:101E20007B689B68D02B0FD07B689B68E02B0BD026
:101E30007B689B68F02B07D040F66820C0F6010055
:101E400040F2453101F094FE4FF46053C4F20203B6
:101E50004FF46052C4F20202926822F0F0017A68F4
:101E600092680A439A607B681B6803F00403002BA6
:101E70002ED07B68DB68002B1BD07B68DB68B3F55A
:101E8000805F16D07B68DB68B3F5A05F11D07B68FC
:101E9000DB68B3F5C05F0CD07B68DB68B3F5E05F4F
:101EA00007D040F66820C0F601004FF4537101F0EE
:101EB0005FFE4FF46053C4F202034FF46052C4F269
:101EC0000202926822F4E0517A68D2680A439A606A
:101ED0007B681B6803F00803002B30D07B681B690C
:101EE000002B1BD07B681B69B3F5805F16D07B6825
:101EF0001B69B3F5A05F11D07B681B69B3F5C05FA8
:101F00000CD07B681B69B3F5E05F07D040F6682012
:101F1000C0F6010040F2533101F02AFE4FF4605345
:101F2000C4F202034FF46052C4F20202926822F437
:101F300060417A6812694FEAC2020A439A6000F06F
:101F4000D7F8024644F6D353C1F26203A3FB02134F
:101F50004FEA93131846FFF793F94FF00003184622
:101F600007F11007BD4680BD90B494B000AF4FF0AC
:101F700000037B644FF00003FB644FF000033B64FD
:101F80004FF00003BB644FF46053C4F202039B683C
:101F900003F00C03042B0AD0082B0ED0002B40F0CA
:101FA0009A804FF41053C0F2F403BB6499E04FF4ED
:101FB0005853C0F26E13BB6493E04FF46053C4F205
:101FC00002035B6803F03F037B644FF46053C4F289
:101FD00002035B6803F480024FF48003FB63FB6B36
:101FE00093FAA3F4BC63BB6B7B637B6BB3FA83F4A0
:101FF0003C633B6BDBB222FA03F3002B24D04FF49B
:102000005853C0F26E137A6CB3FBF2F24FF4605384
:10201000C4F202035B68194647F6C0730B4047F6EB
:10202000C071F962F96A91FAA1F4BC62B96A796285
:10203000796AB1FA81F43C62396AC9B223FA01F3D0
:1020400003FB02F3FB6423E04FF41053C0F2F403EC
:102050007A6CB3FBF2F24FF46053C4F202035B6894
:10206000194647F6C0730B4047F6C071F961F9692C
:1020700091FAA1F4BC61B96979617969B1FA81F425
:102080003C613969C9B223FA01F303FB02F3FB6433
:102090004FF46053C4F202035B6803F440324FF420
:1020A0004033FB60FB6893FAA3F4BC60BB687B60C1
:1020B0007B68B3FA83F43C603B68DBB222FA03F33B
:1020C00003F101034FEA43033B64FA6C3B6CB2FB40
:1020D000F3F3BB6405E04FF41053C0F2F403BB64A8
:1020E00000BFBB6C184607F15007BD4690BC704757
:1020F00090B585B000AFFFF737FF02464FF460534D
:10210000C4F202039B6803F0F0014FF0F003FB60A0
:10211000FB6893FAA3F4BC60BB687B607B68B3FA8E
:1021200083F43C603B68DBB221FA03F140F65823AC
:10213000C0F601035B5C22FA03F240F20C03C2F228
:1021400000031A6040F20C03C2F200031B68184639
:1021500007F11407BD4690BD90B587B000AF786019
:1021600039604FF000033B614FF00003FB604FF01C
:102170000003BB603B681B68002B07D140F698202A
:10218000C0F601004FF0C30101F0F2FC3B685B6850
:10219000002B4BD03B685B68012B47D03B685B68EA
:1021A000112B43D03B685B68022B3FD03B685B68D8
:1021B000122B3BD03B685A684FF00003C1F2110369
:1021C0009A4233D03B685A684FF00003C1F22103B2
:1021D0009A422BD03B685A684FF00003C1F231039A
:1021E0009A4223D03B685A684FF00003C1F21203B1
:1021F0009A421BD03B685A684FF00003C1F2220399
:102200009A4213D03B685A684FF00003C1F2320380
:102210009A420BD03B685B68032B07D040F69820AE
:10222000C0F601004FF0C40101F0A2FC3B689B68BE
:10223000002B0FD03B689B68012B0BD03B689B6841
:10224000022B07D040F69820C0F601004FF0C501E0
:1022500001F08EFC4FF000037B61F5E27B694FF0EB
:10226000010202FA03F33B613B681A683B691340C1
:10227000FB60FA683B699A4240F0E2823B685B6827
:10228000022B04D03B685B68122B40F0FA803B685D
:102290001B69002B00F0BB803B681B69092B00F019
:1022A000B6803B681B69002B00F0B1803B681B695E
:1022B000002B00F0AC803B681B69002B00F0A7806E
:1022C0003B681B69002B00F0A2803B681B69012B57
:1022D00000F09D803B681B69012B00F098803B68F3
:1022E0001B69022B00F093803B681B69022B00F0F6
:1022F0008E803B681B69022B00F089803B681B695C
:10230000032B00F084803B681B69042B7FD03B6863
:102310001B69042B7BD03B681B69042B77D03B687F
:102320001B69052B73D03B681B69052B6FD03B687D
:102330001B69092B6BD03B681B69062B67D03B6878
:102340001B69092B63D03B681B69072B5FD03B6877
:102350001B69072B5BD03B681B69072B57D03B6879
:102360001B69082B53D03B681B69082B4FD03B6877
:102370001B69082B4BD03B681B69092B47D03B6876
:102380001B69092B43D03B681B690A2B3FD03B6874
:102390001B690A2B3BD03B681B690B2B37D03B6872
:1023A0001B690C2B33D03B681B690C2B2FD03B686F
:1023B0001B690D2B2BD03B681B690F2B27D03B686B
:1023C0001B69052B23D03B681B69052B1FD03B687D
:1023D0001B69052B1BD03B681B69082B17D03B687A
:1023E0001B69082B13D03B681B690C2B0FD03B6873
:1023F0001B69062B0BD03B681B690E2B07D040F6E0
:102400009820C0F601004FF0D60101F0B1FB3B6807
:102410001A697B6903F007034FEA830302FA03F3A7
:10242000BB607B694FEAD3027B694FEAD3017B68CB
:1024300001F1080153F8213019467B6903F00703C5
:102440004FEA83034FF00F0000FA03F36FEA030330
:1024500019407B6802F1080243F822107B694FEAB9
:10246000D3027B694FEAD3017B6801F1080153F87D
:1024700021301946BB6819437B6802F1080243F812
:1024800022107B681B681A467B694FEA43034FF0B2
:10249000030101FA03F36FEA03031A407B681A6031
:1024A0007B681B681A463B685B6803F003017B6925
:1024B0004FEA430301FA03F31A437B681A603B684F
:1024C0005B68012B0BD03B685B68022B07D03B6835
:1024D0005B68112B03D03B685B68122B4FD13B68C4
:1024E000DB68002B13D03B68DB68012B0FD03B6807
:1024F000DB68022B0BD03B68DB68032B07D040F670
:102500009820C0F601004FF0E60101F031FB7B6836
:102510009B681A467B694FEA43034FF0030101FAB7
:1025200003F36FEA03031A407B689A607B689B6839
:102530001A463B68D9687B694FEA430301FA03F303
:102540001A437B689A607B685B681A467B694FF028
:10255000010101FA03F36FEA03031A407B685A6032
:102560007B685B681A463B685B6803F010034FEAC0
:1025700013117B6901FA03F31A437B685A607B6885
:10258000DB681A467B694FEA43034FF0030101FA07
:1025900003F36FEA03031A407B68DA607B68DB6849
:1025A0001A463B6899687B694FEA430301FA03F3D3
:1025B0001A437B68DA603B685B6803F08053002B4A
:1025C00000F03E814FF46053C4F202034FF46052B6
:1025D000C4F20202526C42F480425A647B6903F0F6
:1025E00003034FEA83034FF00F0202FA03F3BB60C9
:1025F0004FF46053C4F201037A694FEA92004FF43A
:102600006052C4F2010279694FEA910101F10201BD
:1026100052F821201146BA686FEA0202114000F117
:10262000020243F822104FF46053C4F201037A69A6
:102630004FEA92004FF46052C4F2010279694FEA06
:10264000910101F1020152F8212011467C684FF0FE
:102650000002C4F2020294425CD07C684FF48062B3
:10266000C4F20202944252D07C684FF40062C4F279
:102670000202944248D07C684FF44062C4F20202E5
:1026800094423ED07C684FF48052C4F202029442DD
:1026900034D07C684FF4A052C4F2020294422AD093
:1026A0007C684FF4C052C4F20202944220D07C688D
:1026B0004FF4E052C4F20202944216D07C684FF408
:1026C0000052C4F2020294420CD07C684FF41052C3
:1026D000C4F20202944202D14FF0090201E04FF02D
:1026E0000A0201E04FF0080201E04FF0070201E0AA
:1026F0004FF0060201E04FF0050201E04FF0040246
:1027000001E04FF0030201E04FF0020201E04FF060
:10271000010201E04FF000027C6904F003044FEA7B
:10272000840402FA04F2114300F1020243F8221079
:102730004FF47053C4F201034FF47052C4F201021B
:1027400012681146FA686FEA02020A401A604FF4F2
:102750007053C4F201034FF47052C4F20102526884
:102760001146FA686FEA02020A405A603B685B68E9
:1027700003F48033002B0CD04FF47053C4F20103E8
:102780004FF47052C4F2010212681146FA680A430B
:102790001A603B685B6803F40033002B0CD04FF4E5
:1027A0007053C4F201034FF47052C4F20102526834
:1027B0001146FA680A435A604FF47053C4F2010399
:1027C0004FF47052C4F2010292681146FA686FEA3F
:1027D00002020A409A604FF47053C4F201034FF4AE
:1027E0007052C4F20102D2681146FA686FEA02021E
:1027F0000A40DA603B685B6803F48013002B0CD05E
:102800004FF47053C4F201034FF47052C4F201024A
:1028100092681146FA680A439A603B685B6803F461
:102820000013002B0CD04FF47053C4F201034FF48B
:102830007052C4F20102D2681146FA680A43DA60A3
:102840007B6903F101037B617B690F2B7FF606AD8A
:1028500007F11C07BD4690BD80B584B000AF78601D
:102860000B467B807B88012B3CD07B88022B39D0A8
:102870007B88042B36D07B88082B33D07B88102BA9
:1028800030D07B88202B2DD07B88402B2AD07B8892
:10289000802B27D07B88B3F5807F23D07B88B3F54E
:1028A000007F1FD07B88B3F5806F1BD07B88B3F58A
:1028B000006F17D07B88B3F5805F13D07B88B3F5AA
:1028C000005F0FD07B88B3F5804F0BD07B88B3F5CA
:1028D000004F07D040F69820C0F6010040F2751175
:1028E00001F046F97B681B691A467B881340002B70
:1028F00003D04FF00103FB7302E04FF00003FB73C2
:10290000FB7B184607F11007BD4680BD80B582B03D
:1029100000AF786013460A467A807B707B88012B73
:102920003CD07B88022B39D07B88042B36D07B8827
:10293000082B33D07B88102B30D07B88202B2DD0D8
:102940007B88402B2AD07B88802B27D07B88B3F5CF
:10295000807F23D07B88B3F5007F1FD07B88B3F5C1
:10296000806F1BD07B88B3F5006F17D07B88B3F5E1
:10297000805F13D07B88B3F5005F0FD07B88B3F501
:10298000804F0BD07B88B3F5004F07D040F69820DE
:10299000C0F601004FF4CB7101F0EAF87B78002B10
:1029A0000AD07B78012B07D040F69820C0F60100B2
:1029B00040F2971101F0DCF87B78002B03D07B68A4
:1029C0007A881A8302E07B687A885A8307F10807BD
:1029D000BD4680BD80B582B000AF78607B68002BBB
:1029E00002D14FF0010325E07B681A684FF4E843F9
:1029F000C4F200039A4207D040F6C820C0F6010096
:102A00004FF0E80101F0B4F87B681B79DBB2002BD2
:102A100002D1786800F014F87B684FF002021A7156
:102A20007B684FF000021A617B684FF001021A7157
:102A30004FF00003184607F10807BD4680BD00BFF0
:102A400080B483B000AF786007F10C07BD4680BC4E
:102A5000704700BF80B584B000AF786039604FF038
:102A60000003FB604FF00003BB603B68002B0AD003
:102A70003B68102B07D040F6C820C0F6010040F29A
:102A80006B1101F075F87B685B79012B02D14FF077
:102A9000020358E07B684FF001025A717B684FF0E7
:102AA00002021A717B681B687A6812681268114604
:102AB0003A684FF0010000FA02F20A431A603B68DC
:102AC000002B1AD17B681B681B6803F00403FB60B2
:102AD0007B681B681B6803F03803BB60FB68042B32
:102AE00027D1BB68382B24D17B681B687A681268B1
:102AF000526842F001025A601BE07B681B681B6849
:102B000003F48023FB607B681B681B6803F460137D
:102B1000BB60FB68B3F5802F0BD1BB68B3F5601FBA
:102B200007D17B681B687A681268526842F002021B
:102B30005A607B684FF001021A717B684FF0000207
:102B40005A714FF00003184607F11007BD4680BDCB
:102B500080B586B000AFF860B9607A604FF00003CE
:102B60007B614FF000033B61BB681B68002B27D0E3
:102B7000BB681B68242B23D0BB681B680C2B1FD0A1
:102B8000BB681B68142B1BD0BB681B681C2B17D0A1
:102B9000BB681B68042B13D0BB681B682C2B0FD0A1
:102BA000BB681B68342B0BD0BB681B683C2B07D061
:102BB00040F6C820C0F6010040F2F32100F0D8FF33
:102BC000BB685B68002B0BD0BB685B68022B07D02F
:102BD00040F6C820C0F601004FF43D7100F0C8FF78
:102BE000BB681B68002B27D0BB681B68242B23D035
:102BF000BB681B680C2B1FD0BB681B68142B1BD039
:102C0000BB681B681C2B17D0BB681B68042B13D038
:102C1000BB681B682C2B0FD0BB681B68342B0BD0F8
:102C2000BB681B683C2B07D040F6C820C0F60100EB
:102C300040F2F52100F09CFF7B68002B0AD07B68F6
:102C4000102B07D040F6C820C0F6010040F2F62154
:102C500000F08EFFFB685B79012B02D14FF002037D
:102C600047E0FB684FF001025A71FB684FF0020227
:102C70001A714FF4E843C4F200031B687B617B6860
:102C800040F6FE7202FA03F36FEA03037A69134017
:102C90007B61BB681A68BB685B6813433B617B68F8
:102CA0003A6902FA03F37A6913437B614FF4E8430C
:102CB000C4F200037A691A604FF4E843C4F20003D7
:102CC0004FF4E842C4F20002126811467A684FF0ED
:102CD000C00000FA02F26FEA02020A401A60FB68C2
:102CE0004FF001021A71FB684FF000025A714FF069
:102CF0000003184607F11807BD4680BD80B586B0B1
:102D000000AFF860B9607A603B604FF000037B6110
:102D1000BB68002B0AD0BB68102B07D040F6C82038
:102D2000C0F601004FF44B7100F022FF7B68002BCE
:102D30000DD07B68042B0AD07B68082B07D040F6A7
:102D4000C820C0F6010040F22D3100F011FF3A68B2
:102D50004FF6F0739A4207D940F6C820C0F601003A
:102D600040F22E3100F004FFFB681B687B61BB68FA
:102D7000002B06D17A697B68D31803F108037B61C5
:102D800005E07A697B68D31803F114037B617B69E2
:102D90003A681A604FF00003184607F11807BD465D
:102DA00080BD00BF80B485B000AF78607B6803F061
:102DB0000703FB604FF46D43CEF20003DB68BB609A
:102DC000BA684FF6FF031340BB60FB684FEA03226B
:102DD000BB68134343F0BE6343F42023BB604FF44E
:102DE0006D43CEF20003BA68DA6007F11407BD46FE
:102DF00080BC704780B400AF4FF46D43CEF2000347
:102E0000DB6803F4E0634FEA13231846BD4680BC39
:102E1000704700BF80B483B000AF0346FB714FF42E
:102E20006143CEF2000397F907204FEA5212F97975
:102E300001F01F014FF0010000FA01F143F82210E8
:102E400007F10C07BD4680BC704700BF80B483B05B
:102E500000AF03463960FB7197F90730002B10DA99
:102E60004FF46D43CEF20003FA7902F00F02A2F1A3
:102E700004013A68D2B24FEA0212D2B25B181A7653
:102E80000DE04FF46143CEF2000397F907103A6862
:102E9000D2B24FEA0212D2B25B1883F8002307F1D4
:102EA0000C07BD4680BC704780B489B000AFF860A5
:102EB000B9607A60FB6803F00703FB61FB69C3F14B
:102EC0000703042B28BF0423BB61FB6903F1040340
:102ED000062B03D9FB69A3F1030301E04FF00003C4
:102EE0007B61BB694FF0010202FA03F303F1FF3388
:102EF0001A46BB681A407B6902FA03F27B694FF0FD
:102F0000010101FA03F303F1FF3319467B680B401B
:102F10001343184607F12407BD4680BC704700BF25
:102F200080B582B000AF78607B6803F1FF326FF04C
:102F30007F439A4202D94FF001031DE04EF2100385
:102F4000CEF200037A6802F1FF325A604FF0FF3090
:102F50004FF00F01FFF77AFF4EF21003CEF200039D
:102F60004FF000029A604EF21003CEF200034FF0D1
:102F700007021A604FF00003184607F10807BD4624
:102F800080BD00BF80B582B000AF78607B68072B42
:102F900013D07B68062B10D07B68052B0DD07B6887
:102FA000042B0AD07B68032B07D040F6F820C0F62C
:102FB00001004FF0BA0100F0DBFD7868FFF7F2FE88
:102FC00007F10807BD4680BD80B586B000AF034657
:102FD000B9607A60FB734FF000037B617B680F2B55
:102FE00007D940F6F820C0F601004FF0D20100F0FA
:102FF000BFFDBB680F2B07D940F6F820C0F60100D3
:103000004FF0D30100F0B4FDFFF7F4FE03467B61FF
:103010007869B9687A68FFF747FF034697F90F2088
:1030200010461946FFF712FF07F11807BD4680BD8D
:1030300080B582B000AF0346FB7197F907301846A0
:10304000FFF7E8FE07F10807BD4680BD80B582B0F6
:1030500000AF78607868FFF763FF0346184607F112
:103060000807BD4680BD00BF80B582B000AF786064
:103070007B68002B02D14FF001035DE17B681A6889
:103080004FF40053C4F201039A4217D07B681A68C8
:103090004FF40453C4F201039A420FD07B681A68BC
:1030A0004FF40853C4F201039A4207D040F62C3083
:1030B000C0F601004FF0D70100F05AFD7B685B6855
:1030C000002B16D07B685B68B3F5803F11D07B681E
:1030D0005B68B3F5003F0CD07B685B68B3F5403F9D
:1030E00007D040F62C30C0F601004FF0D80100F0B8
:1030F0003FFD7B689B68002B16D07B689B68B3F113
:10310000807F11D07B689B68B3F1007F0CD07B6817
:103110009B68B3F1407F07D040F62C30C0F6010029
:103120004FF0D90100F024FD7B681B69002B0BD008
:103130007B681B69012B07D040F62C30C0F60100DC
:103140004FF0DA0100F014FD7B689B69002B0BD077
:103150007B689B69012B07D040F62C30C0F601003C
:103160004FF0DB0100F004FD7B68DB6A002B16D01A
:103170007B68DB6AB3F1805F11D07B68DB6AB3F1F7
:10318000005F0CD07B68DB6AB3F1405F07D040F68C
:103190002C30C0F601004FF0DC0100F0E9FC7B6848
:1031A0001B6B002B52D07B681B6BB3F1807F4DD023
:1031B0007B681B6BB3F1007F48D07B681B6BB3F15E
:1031C000407F43D07B681B6BB3F1806F3ED07B6840
:1031D0001B6BB3F1A06F39D07B681B6BB3F1C06F71
:1031E00034D07B681B6BB3F1E06F2FD07B681B6B17
:1031F000B3F1006F2AD07B681B6BB3F1106F25D041
:103200007B681B6BB3F1206F20D07B681B6BB3F125
:10321000306F1BD07B681B6BB3F1406F16D07B689F
:103220001B6BB3F1506F11D07B681B6BB3F1606FF8
:103230000CD07B681B6BB3F1706F07D040F62C305D
:10324000C0F601004FF0DD0100F092FC7B68DB6806
:10325000002B0CD07B68DB68B3F5006F07D040F61D
:103260002C30C0F601004FF0DE0100F081FC7B68DD
:103270001B6A002B03D07B681B6A102B07D940F612
:103280002C30C0F601004FF0DF0100F071FC7B68CC
:10329000DB69002B0BD07B68DB69012B07D040F684
:1032A0002C30C0F601004FF0E00100F061FC7B68BB
:1032B0005B69012B0FD07B685B69002B0BD07B68AF
:1032C0005B69022B07D040F62C30C0F601004FF0AE
:1032D000E10100F04DFC7B685B6A002B0BD07B6842
:1032E0005B6A012B07D040F62C30C0F601004FF08E
:1032F000E20100F03DFC7B6893F83D30DBB2002B2F
:1033000002D1786800F01EF87B684FF0020283F863
:103310003D20786800F0DAFA7B684FF000021A640A
:103320007B684FF0010283F83D207B684FF000027C
:1033300083F83C204FF00003184607F10807BD460C
:1033400080BD00BF80B483B000AF786007F10C0788
:10335000BD4680BC704700BF80B584B000AF7860C8
:103360004FF00003FB817B689B69002B0BD07B68CF
:103370009B69012B07D040F62C30C0F601004FF4BA
:10338000B37100F0F5FB7B68DB6A002B16D07B681D
:10339000DB6AB3F1805F11D07B68DB6AB3F1005F59
:1033A0000CD07B68DB6AB3F1405F07D040F62C306D
:1033B000C0F6010040F2671100F0DAFB7B6893F879
:1033C0003C30012B02D14FF002035FE07B684FF0ED
:1033D000010283F83C207B6893F83D30DBB2222B5E
:1033E00005D17B684FF0320283F83D2004E07B6812
:1033F0004FF0120283F83D207B681B689B6803F046
:103400000103002B11D17B681B687A6812689268EF
:1034100042F001029A6004E000BFFB8903F101035E
:10342000FB81FB89B3F5077FF6D94FF40C53C4F247
:1034300001035B6803F01F03002B0CD17B68DB6A80
:10344000002B1CD17B681B687A681268926842F076
:1034500080429A6013E07B681A684FF40053C4F20C
:1034600001039A420BD17B68DB6A002B07D17B6892
:103470001B687A681268926842F080429A607B68A2
:103480004FF0000283F83C204FF00003184607F18C
:103490001007BD4680BD00BF80B584B000AF786026
:1034A000396000F059FB02463B68D318FB6016E018
:1034B0003B68B3F1FF3F12D000F04EFB0246FB68C1
:1034C0009A420CD37B684FF0030283F83D207B685F
:1034D0004FF0000283F83C204FF0030319E07B68B3
:1034E0001B681B6803F00203002BE1D07B6893F894
:1034F0003D30DBB2252B05D17B684FF0350283F8D8
:103500003D2004E07B684FF0150283F83D204FF02A
:103510000003184607F11007BD4680BD80B483B094
:1035200000AF78607B681B68DB6C184607F10C07FE
:10353000BD4680BC704700BF90B583B000AF7860D7
:1035400039603B681B68002B4FD03B681B68012B20
:103550004BD03B681B68022B47D03B681B68032B92
:1035600043D03B681B68042B3FD03B681B68052B8E
:103570003BD03B681B68062B37D03B681B68072B8A
:1035800033D03B681B68082B2FD03B681B68092B86
:103590002BD03B681B680A2B27D03B681B680B2B82
:1035A00023D03B681B680C2B1FD03B681B680D2B7E
:1035B0001BD03B681B680E2B17D03B681B680F2B7A
:1035C00013D03B681B68102B0FD03B681B68112B76
:1035D0000BD03B681B68122B07D040F62C30C0F68E
:1035E000010040F2DE3100F0C3FA3B685B68002B5B
:1035F00003D03B685B68102B07D940F62C30C0F62F
:10360000010040F2DF3100F0B3FA3B689B68002B09
:1036100023D03B689B68012B1FD03B689B68022B23
:103620001BD03B689B68032B17D03B689B68042B1F
:1036300013D03B689B68052B0FD03B689B68062B1B
:103640000BD03B689B68072B07D040F62C30C0F6A8
:1036500001004FF4787100F08BFA7B6893F83C30EE
:10366000012B02D14FF002031CE17B684FF00102F5
:1036700083F83C203B681B68092B2AD97B681968B2
:103680007B681B68DB6818463B681A6813464FEA7C
:1036900043039B18A3F11E034FF0070202FA03F342
:1036A0006FEA03030340CB607B6819687B681B6883
:1036B000DB6818463B689C683B681A6813464FEA0B
:1036C00043039B18A3F11E0304FA03F30343CB60E7
:1036D00025E07B6819687B681B681B6918463B6896
:1036E0001A6813464FEA43039B184FF0070202FA89
:1036F00003F36FEA030303400B617B6819687B687F
:103700001B681B6918463B689C683B681A6813462F
:103710004FEA43039B1804FA03F303430B613B682E
:103720005B68062B2AD87B6819687B681B685B6B13
:1037300018463B685A6813464FEA83039B18A3F167
:1037400005034FF01F0202FA03F36FEA030303407D
:103750004B637B6819687B681B685B6B18463B682A
:103760001C683B685A6813464FEA83039B18A3F111
:10377000050304FA03F303434B6358E03B685B68BB
:103780000C2B2AD87B6819687B681B681B6B184652
:103790003B685A6813464FEA83039B18A3F123033F
:1037A0004FF01F0202FA03F36FEA030303400B63B7
:1037B0007B6819687B681B681B6B18463B681C6834
:1037C0003B685A6813464FEA83039B18A3F123030F
:1037D00004FA03F303430B6329E07B6819687B68F1
:1037E0001B68DB6A18463B685A6813464FEA830336
:1037F0009B18A3F141034FF01F0202FA03F36FEA93
:1038000003030340CB627B6819687B681B68DB6A33
:1038100018463B681C683B685A6813464FEA8303A6
:103820009B18A3F1410304FA03F30343CB627B68C3
:103830001A684FF40053C4F201039A420FD13B6857
:103840001B68122B0BD14FF40C53C4F201034FF43D
:103850000C52C4F20102526842F480025A607B6842
:103860001A684FF40053C4F201039A4213D13B6823
:103870001B68102B03D03B681B68112B0BD14FF436
:103880000C53C4F201034FF40C52C4F2010252680B
:1038900042F400025A607B684FF0000283F83C203B
:1038A0004FF00003184607F10C07BD4690BD00BF5E
:1038B00080B483B000AF78607B6893F83D30DBB2B2
:1038C000184607F10C07BD4680BC704780B582B032
:1038D00000AF78604FF40C53C4F201034FF40C5264
:1038E000C4F20102526822F440325A604FF40C5381
:1038F000C4F201034FF40C52C4F2010252681146A3
:103900007A6852680A435A607B681B687A68126852
:10391000526822F480725A607B681B687A68126869
:10392000526811467A6812694FEA02220A435A60C5
:103930007B681B687A681268526822F040725A608D
:103940007B681B687A681268526811467A689268C8
:103950000A435A607B681B687A681268926822F48E
:1039600000629A607B681B687A68126892681146E8
:103970007A68D2680A439A607B681B687A68126822
:10398000926822F070629A607B681B687A6812689D
:10399000926811467A68126B0A439A607B681B68CA
:1039A0007A681268926822F040529A607B681B68BD
:1039B0007A681268926811467A68D26A0A439A60F5
:1039C0007B681B687A681268926822F002029A602B
:1039D0007B681B687A681268926811467A689269F7
:1039E0004FEA42020A439A607B685B6A002B2ED042
:1039F0007B689B6A002B03D07B689B6A082B07D9E6
:103A000040F62C30C0F601004FF4986100F0B0F899
:103A10007B681B687A681268526842F400625A60D8
:103A20007B681B687A681268526822F460425A60A8
:103A30007B681B687A681268526811467A68926AD5
:103A400002F1FF324FEA42320A435A6007E07B68D4
:103A50001B687A681268526822F400625A607B68B8
:103A60001B687A681268D26A22F47002DA627B6894
:103A70001B687A681268D26A11467A68126A02F183
:103A8000FF324FEA02520A43DA627B681B687A68A7
:103A90001268926822F400729A607B681B687A68E8
:103AA0001268926811467A68D2694FEA42220A4344
:103AB0009A607B681B687A681268926822F4806258
:103AC0009A607B681B687A681268926811467A6807
:103AD00052694FEA82220A439A6007F10807BD46FD
:103AE00080BD00BF80B500AF4FF47053C4F2020335
:103AF0004FF47052C4F20202126842F400721A606B
:103B00004FF47053C4F202034FF47052C4F2020235
:103B1000126842F480621A604FF47053C4F20203D8
:103B20004FF47052C4F20202126842F480721A60BA
:103B30004FF47A50FFF78AFA4FF00300FFF722FAAA
:103B400000F004F84FF00003184680BD80B400AFC9
:103B5000BD4680BC704700BF80B400AF40F6CC03C8
:103B6000C2F200031B681846BD4680BC704700BF08
:103B700080B584B000AF7860396040F6A033C0F6FD
:103B80000103FB6000F062F880B483B000AF78609E
:103B900039607B684FF001021A603A6840F2040312
:103BA000C2F20003136007F10C07BD4680BC7047EA
:103BB00080B584B000AF786040F6D403C2F2000351
:103BC0001B68002B08D140F6D403C2F2000344F670
:103BD0005012C2F200021A6040F6D403C2F200038F
:103BE0001B68FB607B6803F1030323F003037B6026
:103BF00040F6D403C2F200031A687B68D2184FF66D
:103C00000043C2F201039A4208D909F099F9034628
:103C10004FF00C021A604FF0FF330CE040F6D40373
:103C2000C2F200031A687B68D21840F6D403C2F2CD
:103C300000031A60FB68184607F11007BD4680BDF7
:103C400080B483B000AF7860FEE700BF80B582B07B
:103C500000AF40F6CC33C0F601037B604FF00100AB
:103C6000FFF7EEFF80B400AF4FF46D43CEF20003D8
:103C70004FF46D42CEF20002D2F8882042F4700276
:103C8000C3F888204FF46053C4F202034FF460522B
:103C9000C4F20202126842F001021A604FF460534B
:103CA000C4F202034FF000029A604FF46053C4F272
:103CB00002034FF46052C4F20202126822F08472CE
:103CC00022F480321A604FF46053C4F2020343F2CC
:103CD0001002C2F200425A604FF46053C4F2020371
:103CE0004FF46052C4F20202126822F480221A6079
:103CF0004FF46053C4F202034FF00002DA604FF455
:103D00006D43CEF200034FF000629A60BD4680BC66
:103D1000704700BF80B400AFBD4680BC704700BF95
:103D200080B400AFFEE700BF80B400AFFEE700BF85
:103D300080B400AFFEE700BF80B400AFFEE700BF75
:103D400080B400AFBD4680BC704700BF80B400AFF8
:103D5000BD4680BC704700BF80B400AFBD4680BC8C
:103D6000704700BF80B500AF40F67460C2F200003B
:103D7000FCF7C8FC80BD00BF80B500AF02F0A8FE14
:103D800080BD00BF80B590B000AF40F6C460C2F205
:103D90000000FDF72DF84FF46053C4F202034FF416
:103DA0006052C4F20202526C42F480525A6445F6E8
:103DB000F453C0F601039B883B604FF00203FB60A5
:103DC0004FF002037B604FF005033B614FF00003AF
:103DD000BB6045F6F453C0F601031A683B46104633
:103DE0001946FEF7B9F945F6E453C0F601039B887E
:103DF0003B604FF00203FB604FF002037B604FF02B
:103E00000003BB604FF005033B6145F6E453C0F689
:103E100001031A683B4610461946FEF79DF945F620
:103E2000EC53C0F601039B883B604FF00203FB603C
:103E30004FF000037B604FF00103BB604FF00503C0
:103E40003B6145F6EC53C0F601031A683B46104649
:103E50001946FEF781F945F69C53C0F601039B888D
:103E60003B604FF00203FB604FF001037B604FF0BB
:103E70000003BB604FF000033B6145F69C53C0F666
:103E800001031A683B4610461946FEF765F945F6E8
:103E90009C53C0F601031A6845F69C53C0F6010313
:103EA0009B88104619464FF00102FEF72FFD40F6A1
:103EB000C463C2F200034FF44052C4F201021A601C
:103EC00040F6C463C2F200034FF000029A6040F66D
:103ED000C463C2F200034FF482725A6040F6C463B6
:103EE000C2F200034FF00002DA6040F6C463C2F28F
:103EF00000034FF002021A6140F6C463C2F20003ED
:103F00004FF001025A6140F6C463C2F200034FF45D
:103F100000729A6140F6C463C2F200034FF00002DF
:103F2000DA6140F6C463C2F200034FF000021A6285
:103F300040F6C463C2F200034FF000029A6240F6FA
:103F4000C463C2F200034FF000025A6240F6C46339
:103F5000C2F200034FF00702DA6240F6C460C2F218
:103F60000000FCF703FE07F14007BD4680BD00BF1F
:103F700084B080B500AF07F1080C8CE80F00FB6D32
:103F80009BB240F6C460C2F20000B96D1A464FF011
:103F90000103FCF737FFBD46BDE8804004B0704721
:103FA00080B582B000AF87ED010A3860D7ED017AA5
:103FB000F5EEC07AF1EE10FAD4BF00230123DBB294
:103FC000002B0BD097ED010A07F0CCFCF0EE407A05
:103FD0003B68C3ED007A4FF0000304E03B68054AFC
:103FE0001A604FF0FF035BB2184607F10807BD46A1
:103FF00080BD00BF000000002DE9B0438CB000AFD1
:10400000F860B9607A604FF06403FB84BB68022BF0
:1040100000F38E814FF00003FB627CE0BB68012B54
:1040200027D0022B45D0002B71D17A68FB68D318BA
:10403000C3F50072FB6A9A4210DA7B68C3F500721E
:10404000FB6A9A420ADD40F61873C2F20003FA6A6C
:104050004FEA82029B18C04A1A6058E040F6187373
:10406000C2F20003FA6A4FEA82029B18BB4A1A6046
:104070004DE0FA6A7B689A4210DD7A68FB68D218D4
:10408000FB6A9A420ADD40F61873C2F20003FA6A2C
:104090004FEA82029B18B04A1A6038E040F6187363
:1040A000C2F20003FA6A4FEA82029B18AB4A1A6016
:1040B0002DE07A68FB68D318C3F50072FB6A9A4258
:1040C00005DA7B68C3F50072FB6A9A4209DCFA6A7A
:1040D0007B689A4210DD7A68FB68D218FB6A9A42C4
:1040E0000ADD40F61873C2F20003FA6A4FEA820250
:1040F0009B18994A1A6009E040F61873C2F200034F
:10410000FA6A4FEA82029B18944A1A6000BFFB6A5F
:1041100003F10103FB62FA6A40F2FF139A427FF750
:104120007DAF40F61873C2F2000303F580638B4A3B
:104130001A6040F61873C2F2000303F5FE6303F140
:104140000C03864A1A6007F1100318464FF4807179
:104150004FF001024FF0010305F012FC07F11003CC
:10416000184640F61871C2F2000107F005F84FF04A
:104170000003FB6226E0FB8C4FEA53039BB21A4616
:10418000FB6AD318BB62BA6A40F2FF139A4203DD9E
:10419000BB6AA3F50073BB6240F61873C2F200035A
:1041A000FA6A4FEA82029B181A6843F69C73C2F2BD
:1041B0000003B96A4FEA81015B181A60FB6A03F1D8
:1041C0000103FB62FA6A40F2FF139A42D3DD4FF01B
:1041D0000003FB6215E043F69C73C2F20003FA6A27
:1041E0004FEA82029B181A6840F61873C2F2000365
:1041F000F96A4FEA81015B181A60FB6A03F1010357
:10420000FB62FA6A40F2FF139A42E4DD4FF00003CA
:10421000FB6273E0FA8CFB6A9A425DDB40F618732E
:10422000C2F20003FA6A4FEA82029B181B68184622
:1042300008F028F804460D46F86A08F011F802461E
:104240000B46104619463EA3D3E9002308F06EF84A
:1042500002460B4690469946FB8C184608F000F83B
:1042600002460B464046494608F08AF902460B468C
:104270001046194608F01CFB034600EE103A07F002
:10428000BBF810EE103A184607F0FCFF02460B464A
:10429000104619462CA3D3E9002308F047F802463C
:1042A0000B462BA1D1E9000107F08CFE02460B461C
:1042B0002046294608F03AF802460B4610461946B1
:1042C00008F0F6FA024640F61873C2F20003F96AE3
:1042D0004FEA81015B181A60FA8CFB6A9A4209DA8C
:1042E00040F61873C2F20003FA6A4FEA82029B1882
:1042F0001A4A1A60FB6A03F10103FB62FA6A40F290
:10430000FF139A4286DD07F1100318464FF48071BF
:104310004FF000024FF0010305F032FB07F11003EC
:10432000184640F61871C2F2000106F025FF00E0C1
:1043300000BF07F13007BD46BDE8B083AFF3008092
:10434000F1D4C853FB211940713D0AD7A370DD3F5A
:1043500048E17A14AE47E13F0000803F00000000D2
:1043600080B485B000AF786039604FF00003FB6027
:104370007DE0FB684FEA4302FB684FEAC3037968BC
:10438000CB1893ED007AFB684FEA430140F61873AF
:10439000C2F200034FEA81015B18D3ED007A27EEE9
:1043A000277AFB684FEAC30303F104037968CB184B
:1043B000D3ED006AFB684FEA430303F1010140F6C5
:1043C0001873C2F200034FEA81015B18D3ED007A43
:1043D00066EEA77A77EE677A43F69C73C2F2000323
:1043E0004FEA82029B18C3ED007AFB684FEA430351
:1043F00003F10102FB684FEAC30303F10403796888
:10440000CB1893ED007AFB684FEA430303F10101F7
:1044100040F61873C2F200034FEA81015B18D3ED36
:10442000007A27EE277AFB684FEAC3037968CB1836
:10443000D3ED006AFB684FEA430140F61873C2F2FD
:1044400000034FEA81015B18D3ED007A66EEA77A8C
:1044500077EE277A43F69C73C2F200034FEA82029A
:104460009B18C3ED007AFB6803F10103FB60FB6856
:10447000FF2B7FF77EAF4FF00003FB6032E03B681D
:104480004FEA4302FB68D318BB60FB68002B06DAD7
:10449000FB684FEA83037A68D318174A1A60FA68F0
:1044A00040F2FF139A4206DDFB684FEA83037A6805
:1044B000D318114A1A60FB684FEA83037A68D2184E
:1044C0003B684FEA4301FB68C91843F69C73C2F28C
:1044D00000034FEA81015B181B681360FB6803F15E
:1044E0000103FB60FA6840F2FF139A42C7DD07F14F
:1044F0001407BD4680BC70470000000080B400AFC8
:104500004FF46053C4F202034FF46052C4F202024B
:10451000126B42F001021A634FF46053C4F20203BB
:104520004FF46052C4F20202126B42F002021A63AC
:104530004FF46053C4F202034FF46052C4F202021B
:10454000126B42F004021A634FF46053C4F2020388
:104550004FF46052C4F20202126B42F008021A6376
:10456000BD4680BC704700BF80B400AF40F64053EA
:10457000C2F200031B6803F1010240F64053C2F28D
:1045800000031A60BD4680BC704700BF80B500AF15
:1045900040F6D803C2F20003D3E900014FF0010254
:1045A0004FF00003801841EB030140F6D803C2F23C
:1045B0000003C3E9000103F05DFF44F24163C0F66C
:1045C0000003984740F6D853C2F200031B68002B43
:1045D0000BD040F6D853C2F200031B6803F1FF3240
:1045E00040F6D853C2F200031A6080BD80B400AF19
:1045F00041F21873C2F200034FF000021A6040F655
:104600001473C2F200034FF000021A6042F22073EA
:10461000C2F200034FF07F021A6041F21C73C2F233
:1046200000034FF000021A6044F63013C2F2000398
:104630004FF064021A601846BD4680BC704700BF48
:1046400098B500AF45F60463C0F601031A6845F655
:104650000463C0F601039B8810461946FEF7FCF878
:1046600003464FEA430445F6FC53C0F601031A68BB
:1046700045F6FC53C0F601039B8810461946FEF729
:10468000EBF80346E21840F61473C2F200031A6016
:1046900040F61473C2F200031A6841F21873C2F2B2
:1046A00000031B689A4200F0B88041F21873C2F20E
:1046B00000031B68002B06D140F61473C2F20003FE
:1046C0001B68012B29D041F21873C2F200031B684A
:1046D000012B06D140F61473C2F200031B68032BB2
:1046E0001BD041F21873C2F200031B68032B06D1E2
:1046F00040F61473C2F200031B68022B0DD041F286
:104700001873C2F200031B68022B09D140F6147320
:10471000C2F200031B68002B02D14FF0010201E03E
:104720004FF0000243F62C73C2F200031A6045F604
:104730000C63C0F601031A6845F60C63C0F601036A
:104740009B8810461946FEF787F80346002B44D194
:1047500043F62C73C2F200031B68002B0DD040F609
:10476000E403C2F200031B8803F101039AB240F68E
:10477000E403C2F200031A800CE040F6E403C2F244
:1047800000031B8803F1FF339AB240F6E403C2F240
:1047900000031A8040F6E403C2F200031B884FEACC
:1047A00053039AB240F6E203C2F200031A8040F6C5
:1047B000E203C2F200031A8840F22003C2F20003AF
:1047C0001B88B2FBF3F103FB01F3D31A9AB240F654
:1047D000E203C2F200031A801FE043F62C73C2F218
:1047E00000031B68002B0CD044F63413C2F2000304
:1047F0001B6803F1010244F63413C2F200031A608D
:104800000BE044F63413C2F200031B6803F1FF32DD
:1048100044F63413C2F200031A6040F61473C2F275
:1048200000031A6841F21873C2F200031A6098BDBF
:1048300080B400AF44F63413C2F200031B684FEAA1
:10484000D372D3184FEA63031846BD4680BC704745
:1048500098B500AF40F62163C2F200031B78002B2D
:1048600000F0C48503F0B8FC40F60813C2F2000360
:104870001B68012B00F0B881022B00F06583002B30
:1048800040F00F8540F67063C2F200031B884FEAC8
:10489000430440F67263C2F200031B889BB2A3F587
:1048A0000063184607F0DCFC02460B46104619462A
:1048B000C9A3D3E9002307F063FE02460B46104666
:1048C000194607F0F5FF024642F62C73C2F20003C8
:1048D0004FEA84015B181A6040F67063C2F200036D
:1048E0001B884FEA430303F1010440F6D453C2F29C
:1048F00000031B889BB2A3F50063184607F0B0FCC9
:1049000002460B4610461946B3A3D3E9002307F02D
:1049100037FE02460B461046194607F0C9FF02460D
:1049200042F62C73C2F200034FEA84015B181A604E
:1049300040F67263C2F200031B889AB240F6E003AD
:10494000C2F200031B889A420AD940F67263C2F28F
:1049500000031B889AB240F6E003C2F200031A80FB
:1049600040F6D453C2F200031B889AB240F6E0032B
:10497000C2F200031B889A420AD940F6D453C2F20D
:1049800000031B889AB240F6E003C2F200031A80CB
:1049900040F67063C2F200031B884FEA430241F203
:1049A0002073C2F200034FEA82029B1893ED007A53
:1049B00040F6F003C2F20003D3ED007AB4EEE77ADA
:1049C000F1EE10FAD4BF00230123DBB2002B13D089
:1049D00040F67063C2F200031B884FEA430241F2C3
:1049E0002073C2F200034FEA82029B181A6840F655
:1049F000F003C2F200031A6040F67063C2F20003D3
:104A00001B884FEA430303F1010241F22073C2F213
:104A100000034FEA82029B1893ED007A40F6F00300
:104A2000C2F20003D3ED007AB4EEE77AF1EE10FAA9
:104A3000D4BF00230123DBB2002B15D040F67063F6
:104A4000C2F200031B884FEA430303F1010241F263
:104A50002073C2F200034FEA82029B181A6840F6E4
:104A6000F003C2F200031A6040F67063C2F2000362
:104A70001B884FEA430241F22073C2F200034FEA5F
:104A800082029B1893ED007ADFED557A27EE277AA4
:104A900040F21003C2F20003D3ED007A27EE277A2A
:104AA000DFED507A77EE277AFCEEE77A17EE903A50
:104AB0009BB2184602F020FD40F67063C2F200037C
:104AC0001B884FEA430303F1010241F22073C2F253
:104AD00000034FEA82029B1893ED007ADFED407AE3
:104AE00027EE277A40F21003C2F20003D3ED007ADA
:104AF00027EE277ADFED3B7A77EE277AFCEEE77A2E
:104B000017EE903A9BB2184602F010FD40F6706323
:104B1000C2F200031B881A4640F21C03C2F20003D3
:104B20001B88C3F1FF039A4240F3B68340F67063DB
:104B3000C2F200031B881A4640F21C03C2F20003B3
:104B40001B88A3F58073D3184FEA430140F67063C6
:104B5000C2F200031B884FEA430242F62C73C2F2F2
:104B600000034FEA82029B181A6844F2A073C2F253
:104B700000034FEA81015B181A6040F67063C2F2CD
:104B800000031B881A4640F21C03C2F200031B8874
:104B9000A3F58073D3184FEA430303F1010140F6F4
:104BA0007063C2F200031B884FEA430303F1010262
:104BB00042F62C73C2F200034FEA82029B181A6875
:104BC00044F2A073C2F200034FEA81015B181A603D
:104BD00062E300BFAFF30080000000000000B040BF
:104BE000000080450000004540F67063C2F20003FB
:104BF0001B884FEA430440F67263C2F200031B882D
:104C00009BB2A3F50063184607F02AFB02460B4649
:104C100010461946C8A3D3E9002307F0B1FC0246A9
:104C20000B461046194607F043FE024641F2207338
:104C3000C2F200034FEA84015B181A6040F6706309
:104C4000C2F200031B884FEA430303F1010440F65C
:104C5000D453C2F200031B889BB2A3F5006318462D
:104C600007F0FEFA02460B4610461946B2A3D3E9F6
:104C7000002307F085FC02460B461046194607F054
:104C800017FE024641F22073C2F200034FEA84018C
:104C90005B181A6040F67263C2F200031B889AB276
:104CA00040F6E003C2F200031B889A420AD940F69C
:104CB0007263C2F200031B889AB240F6E003C2F2AC
:104CC00000031A8040F6D453C2F200031B889AB244
:104CD00040F6E003C2F200031B889A420AD940F66C
:104CE000D453C2F200031B889AB240F6E003C2F22A
:104CF00000031A8040F67063C2F200031B884FEA7B
:104D0000430241F62073C2F200034FEA82029B186D
:104D100093ED007A40F6F003C2F20003D3ED007A7F
:104D2000B4EEE77AF1EE10FAD4BF00230123DBB230
:104D3000002B13D040F67063C2F200031B884FEAC9
:104D4000430241F62073C2F200034FEA82029B182D
:104D50001A6840F6F003C2F200031A6040F670636E
:104D6000C2F200031B884FEA430303F1010241F63C
:104D70002073C2F200034FEA82029B1893ED007A7F
:104D800040F6F003C2F20003D3ED007AB4EEE77A06
:104D9000F1EE10FAD4BF00230123DBB2002B15D0B3
:104DA00040F67063C2F200031B884FEA430303F12D
:104DB000010241F62073C2F200034FEA82029B18FF
:104DC0001A6840F6F003C2F200031A6040F67063FE
:104DD000C2F200031B884FEA430241F62073C2F27D
:104DE00000034FEA82029B1893ED007ADFED547ABC
:104DF00027EE277A40F21003C2F20003D3ED007AC7
:104E000027EE277ADFED4F7A77EE277AFCEEE77A06
:104E100017EE903A9BB2184602F06EFB40F67063B4
:104E2000C2F200031B884FEA430303F1010241F67B
:104E30002073C2F200034FEA82029B1893ED007ABE
:104E4000DFED3F7A27EE277A40F21003C2F200032B
:104E5000D3ED007A27EE277ADFED3A7A77EE277ADC
:104E6000FCEEE77A17EE903A9BB2184602F05EFB32
:104E700040F67063C2F200031B881A4640F21C031E
:104E8000C2F200031B88C3F1FF039A4240F306827B
:104E900040F67063C2F200031B881A4640F21C03FE
:104EA000C2F200031B88A3F58073D3184FEA4301B5
:104EB00040F67063C2F200031B884FEA430241F2DE
:104EC0002073C2F200034FEA82029B181A6844F270
:104ED000A073C2F200034FEA81015B181A6040F62A
:104EE0007063C2F200031B881A4640F21C03C2F230
:104EF00000031B88A3F58073D3184FEA430303F123
:104F0000010140F67063C2F200031B884FEA4303BD
:104F100003F1010241F22073C2F200034FEA820260
:104F20009B181A6844F2A073C2F200034FEA810191
:104F30005B181A60B2E100BF000000000000B04042
:104F4000000080450000004540F67063C2F2000397
:104F50001B884FEA430440F67263C2F200031B88C9
:104F60009BB2A3F50063184607F07AF902460B4698
:104F7000104619460FF28843D3E9002307F000FBDF
:104F800002460B461046194607F092FC024641F6CF
:104F90002073C2F200034FEA84015B181A6040F6E6
:104FA0007063C2F200031B884FEA430303F101045C
:104FB00040F6D453C2F200031B889BB2A3F50063F2
:104FC000184607F04DF902460B46104619460FF2F7
:104FD0003043D3E9002307F0D3FA02460B461046CC
:104FE000194607F065FC024641F62073C2F2000341
:104FF0004FEA84015B181A6040F67263C2F2000344
:105000001B889AB240F6E003C2F200031B889A4262
:105010000AD940F67263C2F200031B889AB240F6C6
:10502000E003C2F200031A8040F6D453C2F2000338
:105030001B889AB240F6E003C2F200031B889A4232
:105040000AD940F6D453C2F200031B889AB240F644
:10505000E003C2F200031A8040F67063C2F200035C
:105060001B884FEA430242F62C73C2F200034FEA58
:1050700082029B1893ED007A40F6F003C2F200031F
:10508000D3ED007AB4EEE77AF1EE10FAD4BF002344
:105090000123DBB2002B13D040F67063C2F2000391
:1050A0001B884FEA430242F62C73C2F200034FEA18
:1050B00082029B181A6840F6F003C2F200031A60DD
:1050C00040F67063C2F200031B884FEA430303F10A
:1050D000010242F62C73C2F200034FEA82029B18CF
:1050E00093ED007A40F6F003C2F20003D3ED007AAC
:1050F000B4EEE77AF1EE10FAD4BF00230123DBB25D
:10510000002B15D040F67063C2F200031B884FEAF3
:10511000430303F1010242F62C73C2F200034FEA8B
:1051200082029B181A6840F6F003C2F200031A606C
:1051300040F67063C2F200031B884FEA430242F656
:105140002C73C2F200034FEA82029B1893ED007A9F
:10515000DFEDA97A27EE277A40F21003C2F20003AE
:10516000D3ED007A27EE277ADFEDA47A77EE277A5F
:10517000FCEEE77A17EE903A9BB2184602F0BCF9C3
:1051800040F67063C2F200031B884FEA430303F149
:10519000010242F62C73C2F200034FEA82029B180E
:1051A00093ED007ADFED947A27EE277A40F2100330
:1051B000C2F20003D3ED007A27EE277ADFED8F7A73
:1051C00077EE277AFCEEE77A17EE903A9BB2184614
:1051D00002F0ACF940F67063C2F200031B881A4675
:1051E00040F21C03C2F200031B88C3F1FF039A4282
:1051F00056DD40F67063C2F200031B881A4640F287
:105200001C03C2F200031B88A3F58073D3184FEA76
:10521000430140F67063C2F200031B884FEA430269
:1052200041F62073C2F200034FEA82029B181A680B
:1052300044F2A073C2F200034FEA81015B181A60C6
:1052400040F67063C2F200031B881A4640F21C034A
:10525000C2F200031B88A3F58073D3184FEA4303FF
:1052600003F1010140F67063C2F200031B884FEAAC
:10527000430303F1010241F62073C2F200034FEA37
:1052800082029B181A6844F2A073C2F200034FEA2C
:1052900081015B181A6003E000BF02E000BF00E07C
:1052A00000BF40F6F003C2F200031B68184606F088
:1052B000E9FF02460B46104619464DA3D3E90023E9
:1052C00007F034F802460B461046194607F0F0FA8C
:1052D000024640F6F003C2F200031A6040F6706323
:1052E000C2F200031B8803F101039AB240F6706317
:1052F000C2F200031A8040F67063C2F200031B88FA
:105300001A4640F21C03C2F200031B884FEA530303
:105310009BB2C3F580739A4266DB40F61963C2F212
:1053200000034FF001021A7040F21C03C2F20003A6
:105330001B884FEA53039AB240F67063C2F200032F
:105340001A8040F60813C2F200031B68012B1BD021
:10535000022B31D0002B47D140F6F803C2F20003F4
:105360004FF001021A6040F60813C2F200034FF03A
:1053700001021A6045F20943C0F6000341F22070B1
:10538000C2F2000098472FE040F6FC03C2F200038F
:105390004FF001021A6040F60813C2F200034FF00A
:1053A00002021A6045F20943C0F6000341F620707C
:1053B000C2F20000984717E040F60013C2F2000363
:1053C0004FF001021A6040F60813C2F200034FF0DA
:1053D00000021A6045F20943C0F6000342F62C7041
:1053E000C2F20000984700BF02F036FF98BD00BF30
:1053F0001EA7E8482EFFEF3F000080450000004553
:10540000000000000000B04080B485B000AF7860BC
:105410004FF00003FB8112E0FB894FEA83037A68B7
:10542000D218F98944F2A073C2F200034FEA810155
:105430005B181B681360FB8903F10103FB8140F2D9
:105440001C03C2F200031B88FA899A42E4D30AE0E3
:10545000FB894FEA83037A68D318084A1A60FB89EC
:1054600003F10103FB81FA8940F2FF139A42EFD95D
:1054700007F11407BD4680BC704700BF0000000064
:1054800080B586B000AF78603960FEF72BFB40F640
:10549000E033C0F60103FB6040F6F433C0F60103CD
:1054A000BB60FFF72BF802F073F8FEF76BFC02F01D
:1054B000CDFF02F0F7FF4FF40060C4F202004FF49A
:1054C00000514FF00102FDF721FA40F22C03C2F225
:1054D00000031B881AB240F6EC03C2F200031B88DB
:1054E0001BB2D21A40F6EC03C2F200031B881BB2B7
:1054F00010464FF000011A46FEF77EFD47F2D93301
:10550000C0F600039847FFF771F803F0E1F84FF099
:10551000030003F00DFE4FF0000003F099FE4FF082
:10552000000003F095FE4FF0030004F0EBF94FF09C
:10553000010004F015FA4FF6FF704FF0000104F07F
:10554000F7F94FF0C8004FF078014FF0000203F078
:10555000ADFD02F085FC40F62163C2F200034FF07E
:1055600001021A7002F078FE47F26523C0F60003CC
:1055700098474FF000024FF00003C7E9042345F6B7
:105580002143C0F600034FF00100984745F2B16394
:10559000C0F60003984745F62143C0F600034FF0DC
:1055A0000000984746F26963C0F60003984745F249
:1055B000C153C0F600039847E8E700BF00000000B1
:1055C00080B584B002AF40F60C13C2F2000393ED35
:1055D000007ADFED357A27EE277AF7EE007A77EE5C
:1055E000277A17EE900A06F04DFE02460B4643EC72
:1055F000102B06F031F953EC102B1046194628A356
:10560000D3E9002306F092FE02460B4610461946E7
:1056100007F026F903467B6040F61013C2F2000340
:105620001B687A689A4219DD40F61013C2F2000333
:105630001B6803F1960240F61013C2F200031B68C8
:105640007968CB1A4FF47841009110464FF09C01D5
:105650001A464FF0030303F0D7FD14E07B6803F113
:10566000960240F61013C2F2000319687B68CB1A49
:105670004FF00001009110464FF09C011A464FF088
:10568000030303F0C1FD40F61013C2F200037A6871
:105690001A6007F10807BD4680BD00BFAFF3008068
:1056A000000000000000244000247449AFF3008093
:1056B00080B500AF40F6E203C2F200031B880A2B5C
:1056C00000F2598201A050F823F000BFF9560008FB
:1056D00017570008355700084F570008695700084A
:1056E000835700089D570008B7570008D75800088F
:1056F000F7590008835A000840F22403C2F200035D
:1057000044F24022C0F20F021A6046F67573C0F6EA
:105710000003984738E240F22403C2F2000348F243
:10572000A062C0F201021A6046F67573C0F600036B
:10573000984729E240F22403C2F2000342F21072B9
:105740001A6046F67573C0F6000398471CE240F2F3
:105750002403C2F200034FF47A721A6046F675739E
:10576000C0F6000398470FE240F22403C2F20003A0
:105770004FF064021A6046F67573C0F6000398474E
:1057800002E240F22403C2F200034FF00A021A6060
:1057900046F67573C0F600039847F5E140F224031E
:1057A000C2F200034FF001021A6046F67573C0F6AC
:1057B00000039847E8E1FFF73BF8024643F6987389
:1057C000C2F200031A6043F69873C2F200031A682B
:1057D00042F62873C2F200031B689A4200F0CD81A2
:1057E00042F62873C2F200031B689AB243F698731C
:1057F000C2F200031B689BB2D31A9AB240F6EC03C4
:10580000C2F200031B889BB2D3189BB29AB240F637
:10581000EC03C2F200031A8040F6EC03C2F200036C
:105820001B881BB2002B06DC40F6EC03C2F200031F
:105830004FF000021A8040F6EC03C2F200031B880E
:105840001BB2C72B06DD40F6EC03C2F200034FF09B
:1058500064021A8040F6EC03C2F200031A8840F298
:105860002C03C2F200031B8812B21BB29A420EDB59
:1058700040F22C03C2F200031B889BB203F1FF33FA
:105880009BB29AB240F6EC03C2F200031A8043F6D0
:105890009873C2F200031A6842F62873C2F200033A
:1058A0001A6040F22C03C2F200031B881AB240F6C1
:1058B000EC03C2F200031B881BB2D21A40F6EC03C1
:1058C000C2F200031B881BB210464FF000011A46BB
:1058D000FEF792FB51E1FEF7ABFF024643F69873E9
:1058E000C2F200031A6043F69873C2F200031A680A
:1058F00042F62873C2F200031B689A4200F03F810F
:1059000042F62873C2F200031B689AB243F69873FA
:10591000C2F200031B689BB2D31A9AB240F22C0366
:10592000C2F200031B889BB2D3189BB29AB240F21A
:105930002C03C2F200031A8040F22C03C2F20003CF
:105940001B881BB2002B06DC40F22C03C2F20003C2
:105950004FF000021A8040F22C03C2F200031B88B1
:105960001BB2C72B06DD40F22C03C2F200034FF03E
:1059700064021A8040F22C03C2F200031A8840F637
:10598000EC03C2F200031B8812B21BB29A420EDC77
:1059900040F6EC03C2F200031B889BB203F1010343
:1059A0009BB29AB240F22C03C2F200031A8043F673
:1059B0009873C2F200031A6842F62873C2F2000319
:1059C0001A6040F22C03C2F200031B881AB240F6A0
:1059D000EC03C2F200031B881BB2D21A40F6EC03A0
:1059E000C2F200031B881BB210464FF000011A469A
:1059F000FEF702FBC3E0FEF71BFF024643F6987377
:105A0000C2F200031A6043F69873C2F200031A68E8
:105A100042F62873C2F200031B689A4200F0B1807C
:105A200040F6EE03C2F200031B781A4642F62873D2
:105A3000C2F20003196843F69873C2F200031B68B0
:105A4000CB1AD11845F25653C5F2555383FB0102C8
:105A50004FEAE173D21A13464FEA43039B18CA1A5E
:105A6000D2B240F6EE03C2F200031A7043F6987306
:105A7000C2F200031A6842F62873C2F200031A60E9
:105A80007FE0FEF7D5FE024643F69873C2F20003AC
:105A90001A6043F69873C2F200031A6842F628733C
:105AA000C2F200031B689A426DD042F62873C2F21C
:105AB00000031A6843F69873C2F200031B68D31AF6
:105AC00007EE903AB8EEE77A40F21403C2F2000310
:105AD000D3ED007A27EE277A40F21003C2F20003DA
:105AE000D3ED007A77EE277A40F21003C2F200037A
:105AF000C3ED007A40F21003C2F2000393ED007A86
:105B000040F21803C2F20003D3ED007AB4EEE77A54
:105B1000F1EE10FAD4BF00230123DBB2002B09D031
:105B200040F21803C2F200031A6840F21003C2F2F6
:105B300000031A6040F21003C2F20003D3ED007AB2
:105B4000F5EEC07AF1EE10FA8CBF00230123DBB230
:105B5000002B05D040F21003C2F200030B4A1A607A
:105B600043F69873C2F200031A6842F62873C2F231
:105B700000031A6007E000BF06E000BF04E000BFBA
:105B800002E000BF00E000BF80BD00BF00000000D9
:105B900080B586B000AF786039601F4B3B614FF035
:105BA00000037B6119E07B694FEA83037A68D318AD
:105BB00093ED007A7B694FEA83037A68D318D3EDBB
:105BC000007A67EE277A97ED047A77EE277AC7EDA9
:105BD000047A7B6903F101037B617A693B689A422D
:105BE000E1DB3B6807EE103AF8EEC77A97ED047AEE
:105BF000C7EE277AC7ED047A07F10C0397ED040A84
:105C00001846FEF7CDF9FB6807EE903AB0EE670A4A
:105C100007F11807BD4680BD00000000000000002D
:105C200090B589B004AF0346FB71FB79002B00F0FF
:105C300087804FF0140300934FF6FF7301934FF0EA
:105C4000B4004FF0020140F61842C0F601024FF0D6
:105C5000560303F075FC4FF00C0300934FF6FF73EF
:105C600001934FF096004FF05A0141F68812C0F6AA
:105C700001024FF0280303F063FC4FF08803009308
:105C80004FF0720301934FF6FF7302934FF07E00C3
:105C90004FF077014FF088024FF07C0303F0F6FAE3
:105CA0004FF00C0300934FF6FF7301934FF09600F3
:105CB0004FF0880143F6C442C0F601024FF02F03B3
:105CC00003F03EFC47F26104C0F600044FF02E00E2
:105CD0004FF0AE014FF06C024FF6FF73A04747F252
:105CE0006104C0F600044FF02E004FF0EE014FF0BB
:105CF0006C024FF6FF73A0474FF00A0300934FF674
:105D0000FF7301934FF08E004FF0A20145F258123D
:105D1000C0F601024FF09B0303F012FC4FF02E037C
:105D200000934FF6FF73019340F211104FF0C00142
:105D300044F22C12C0F601024FF02D0303F000FCD8
:105D400040F22803C2F200031B6840F63050C2F252
:105D5000000040F60841C0F601011A4607F0F6F8C7
:105D600040F63053C2F200031A7840F23C03C2F20C
:105D700000031B7852B25BB29A421CD1FB79002B14
:105D800019D140F6E203C2F200031A8840F21E0362
:105D9000C2F200031B889A4229D040F6E203C2F205
:105DA00000031B88002B06D040F21E03C2F2000342
:105DB0001B88002B1BD147F26104C0F6000440F69B
:105DC0003053C2F200031B785AB240F6E203C2F22B
:105DD00000031B88002B02D14FF4784301E04FF6FB
:105DE000FF7310464FF08E014FF06C02A04740F653
:105DF0003053C2F200035A7840F23C03C2F200036F
:105E00005B7852B25BB29A421CD1FB79002B19D15C
:105E100040F6E203C2F200031A8840F21E03C2F207
:105E200000031B889A4229D040F6E203C2F2000325
:105E30001B88002B06D040F21E03C2F200031B8811
:105E4000002B1BD147F26104C0F6000440F630532A
:105E5000C2F200035B785AB240F6E203C2F20003DA
:105E60001B88002B02D14FF4784301E04FF6FF73FB
:105E700010464FF09E014FF06C02A04740F63053A1
:105E8000C2F200039A7840F23C03C2F200039B780E
:105E900052B25BB29A421CD1FB79002B19D140F669
:105EA000E203C2F200031A8840F21E03C2F20003AA
:105EB0001B889A4229D040F6E203C2F200031B88F5
:105EC000012B06D040F21E03C2F200031B88012BF7
:105ED0001BD147F26104C0F6000440F63053C2F211
:105EE00000039B785AB240F6E203C2F200031B881B
:105EF000012B02D14FF4784301E04FF6FF731046B7
:105F00004FF0BE014FF06C02A04740F63053C2F292
:105F10000003DA7840F23C03C2F20003DB7852B2AD
:105F20005BB29A421CD1FB79002B19D140F6E203F7
:105F3000C2F200031A8840F21E03C2F200031B885B
:105F40009A4229D040F6E203C2F200031B88022BDA
:105F500006D040F21E03C2F200031B88022B1BD1A5
:105F600047F26104C0F6000440F63053C2F2000369
:105F7000DB785AB240F6E203C2F200031B88022B20
:105F800002D14FF4784301E04FF6FF7310464FF013
:105F9000CE014FF06C02A04740F63053C2F200032E
:105FA0001A7940F23C03C2F200031B7952B25BB291
:105FB0009A421CD1FB79002B19D140F6E203C2F2C0
:105FC00000031A8840F21E03C2F200031B889A42A3
:105FD00029D040F6E203C2F200031B88032B06D04F
:105FE00040F21E03C2F200031B88032B1BD147F2B1
:105FF0006104C0F6000440F63053C2F200031B797E
:106000005AB240F6E203C2F200031B88032B02D10E
:106010004FF4784301E04FF6FF7310464FF0DE0176
:106020004FF06C02A04740F63053C2F200035A7999
:1060300040F23C03C2F200035B7952B25BB29A4277
:106040001CD1FB79002B19D140F6E203C2F2000308
:106050001A8840F21E03C2F200031B889A4229D01C
:1060600040F6E203C2F200031B88042B06D040F284
:106070001E03C2F200031B88042B1BD147F26104EC
:10608000C0F6000440F63053C2F200035B795AB206
:1060900040F6E203C2F200031B88042B02D14FF446
:1060A000784301E04FF6FF7310464FF0FE014FF0CA
:1060B0006C02A04740F63053C2F200039A7940F2D6
:1060C0003C03C2F200039B7952B25BB29A421CD1EC
:1060D000FB79002B19D140F6E203C2F200031A88C3
:1060E00040F21E03C2F200031B889A4229D040F6F8
:1060F000E203C2F200031B88052B06D040F21E0308
:10610000C2F200031B88052B1BD147F26104C0F6C5
:10611000000440F63053C2F200039B795AB240F6B5
:10612000E203C2F200031B88052B02D14FF478432F
:1061300001E04FF6FF7310464FF487714FF06C0289
:10614000A04740F63053C2F20003DA7940F23C0334
:10615000C2F20003DB7952B25BB29A421CD1FB79E6
:10616000002B19D140F6E203C2F200031A8840F274
:106170001E03C2F200031B889A4229D040F6E203B4
:10618000C2F200031B88062B06D040F21E03C2F2A7
:1061900000031B88062B1BD147F26104C0F60004E4
:1061A00040F63053C2F20003DB795AB240F6E20304
:1061B000C2F200031B88062B02D14FF4784301E0A2
:1061C0004FF6FF7310464FF48F714FF06C02A047EB
:1061D00040F22803C2F200031A6840F6E803C2F254
:1061E00000031A6040F23C00C2F2000040F6305159
:1061F000C2F2000106F0D2FE40F6EC03C2F2000348
:106200001A8840F23003C2F200031B8812B21BB29C
:106210009A421ED1FB79002B1BD140F6E203C2F259
:1062200000031A8840F21E03C2F200031B889A4240
:1062300000F0998040F6E203C2F200031B88072BAE
:1062400007D040F21E03C2F200031B88072B40F068
:106250008A8040F6EC03C2F200031B881AB2134690
:106260004FEA83039B184FEAC30340F63050C2F253
:10627000000040F60C41C0F601011A4606F066FE29
:106280004FF0020003F03EFB40F6E203C2F20003CF
:106290001B88072B02D14FF4784301E04FF6FF73C0
:1062A00018464FF0000103F043FB4FF0C8004FF0D9
:1062B000870103F00FFB4FF00003FB600EE040F698
:1062C0003053C2F20003FA689B181B78DBB2184601
:1062D00003F084F9FB6803F10103FB60FB68032B07
:1062E000EDDD4FF0000300934FF079004FF078019F
:1062F0004FF003024FF0640302F086FF40F6EC0318
:10630000C2F200031B881BB24FEAD372D3184FEAC4
:1063100063039BB21BB203F1780240F22C03C2F27A
:1063200000031B8819B240F6EC03C2F200031B887D
:106330001BB2CB1A4FEAD371CB184FEA63034FF667
:10634000FF7100914FF0790011464FF0030202F007
:106350005BFF40F6EC03C2F200031A8840F2300300
:10636000C2F200031A8040F22C03C2F200031A8822
:1063700040F22E03C2F200031B8812B21BB29A42F3
:106380001ED1FB79002B1BD140F6E203C2F20003C1
:106390001A8840F21E03C2F200031B889A4200F0E2
:1063A000998040F6E203C2F200031B88082B07D055
:1063B00040F21E03C2F200031B88082B40F08A80C3
:1063C00040F22C03C2F200031B881AB213464FEAB4
:1063D00083039B184FEAC30340F63050C2F200001B
:1063E00040F61041C0F601011A4606F0AFFD4FF02D
:1063F000020003F087FA40F6E203C2F200031B88B2
:10640000082B02D14FF4784301E04FF6FF73184692
:106410004FF0000103F08CFA40F209104FF08701B1
:1064200003F058FA4FF00003BB600EE040F6305323
:10643000C2F20003BA689B181B78DBB2184603F05F
:10644000CDF8BB6803F10103BB60BB68032BEDDD36
:106450004FF0000300934FF079004FF078014FF0B8
:1064600003024FF0640302F0CFFE40F6EC03C2F2E9
:1064700000031B881BB24FEAD372D3184FEA6303A1
:106480009BB21BB203F1780240F22C03C2F200036C
:106490001B8819B240F6EC03C2F200031B881BB242
:1064A000CB1A4FEAD371CB184FEA63034FF6FF7153
:1064B00000914FF0790011464FF0030202F0A4FE64
:1064C00040F22C03C2F200031A8840F22E03C2F2FB
:1064D00000031A8040F6EE03C2F200031A7840F27D
:1064E0003203C2F200031B789A421CD1FB79002BC5
:1064F00019D140F6E203C2F200031A8840F21E03EB
:10650000C2F200031B889A4279D040F6E203C2F23D
:1065100000031B88092B06D040F21E03C2F20003C1
:106520001B88092B6BD140F6EE03C2F200031B78E7
:10653000012B20D0022B3BD0002B56D140F6E2039A
:10654000C2F200031B88092B02D14FF4784301E00B
:106550004FF6FF734FF00902009201934FF0C40011
:106560004FF05B0141F64852C0F601024FF01C03A8
:1065700002F0E6FF39E040F6E203C2F200031B88B6
:10658000092B02D14FF4784301E04FF6FF734FF02F
:106590000902009201934FF0C4004FF05B0141F6F5
:1065A0004072C0F601024FF01C0302F0C9FF1CE06C
:1065B00040F6E203C2F200031B88092B02D14FF41C
:1065C000784301E04FF6FF734FF009020092019308
:1065D0004FF0C4004FF05B0142F23812C0F60102E6
:1065E0004FF01C0302F0ACFF00BF40F6EE03C2F216
:1065F00000031A7840F23203C2F200031A7040F22C
:106600001003C2F200031B68184605F03BFE024669
:106610000B461046194610A3D3E9002305F086FE69
:1066200002460B46104619460DA3D3E9002306F097
:10663000E5F80346002B09D140F6E203C2F200035D
:106640001A8840F21E03C2F200031A8007F11407F1
:10665000BD4690BDAFF30080AE47E17A14AEEF3F88
:106660000000000000000000B0B584B000AF42F2AE
:106670002870C2F2000040F62011C2F200014FF46F
:10668000807205F007F8DFF84034FB60DFF83C3437
:10669000BB604FF00103FB712DE0FA7940F6201347
:1066A000C2F200034FEA82029B181B683B6097ED21
:1066B000007AD7ED037AB4EEE77AF1EE10FAD4BFA0
:1066C00000230123DBB2002B01D03B68FB6097ED78
:1066D000007AD7ED027AB4EEE77AF1EE10FA54BF01
:1066E00000230123DBB2002B01D03B68BB60FB79A8
:1066F00003F10103FB71FB79FF2BCED140F6205350
:10670000C2F20003D3ED007A97ED037AB4EEE77A94
:10671000F1EE10FAD4BF00230123DBB2002B27D007
:1067200040F62053C2F200031B68184605F0AAFD8C
:1067300004460D46F86805F0A5FD02460B461046D6
:106740001946D9A3D3E9002305F0F0FD02460B4614
:106750002046294605F038FC02460B4610461946ED
:1067600006F0A6F8024640F62053C2F200031A6073
:1067700040F62053C2F200031B68184605F082FD64
:1067800002460B4643EC102B05F066F853EC102B39
:1067900010461946C6A3D3E9002305F0F1FE0246D0
:1067A0000B461046194606F083F8024640F624537D
:1067B000C2F200031A6040F62053C2F200031B68C5
:1067C000184605F05FFD02460B4610461946BAA36F
:1067D000D3E9002305F0AAFD02460B4610461946F0
:1067E00006F066F8024640F62053C2F200031A6033
:1067F00040F62053C2F2000393ED007A40F23403D6
:10680000C2F20003D3ED007AB4EEE77AF1EE10FAAB
:10681000D4BF00230123DBB2002B09D040F23403A4
:10682000C2F200031A6840F62053C2F200031A6055
:1068300040F62053C2F2000393ED007A40F2380391
:10684000C2F20003D3ED007AB4EEE77AF1EE10FA6B
:1068500054BF00230123DBB2002B09D040F23803E0
:10686000C2F200031A6840F62053C2F200031A6015
:106870004FF00103FB7170E0FA7940F62013C2F289
:1068800000034FEA82029B1893ED007AF7EE007A3C
:1068900077EE277A17EE900A05F0F4FC02460B46D5
:1068A00043EC102B04F0D8FF53EC102B1046194684
:1068B0007FA3D3E9002305F063FE02460B4614468E
:1068C0001D4640F62053C2F200031B68184605F02F
:1068D000D9FC02460B462046294605F051FE0246E9
:1068E0000B461046194676A3D3E9002305F01EFD9A
:1068F00002460B461046194605F0DAFF024640F6FE
:106900002853C2F200031A6040F62C53C2F200036F
:106910001B781946FB799BB2C3F178039BB29AB2FC
:1069200040F62853C2F20003D3ED007AFCEEE77A7A
:1069300017EE903ADBB2184643F6C433C0F60103B3
:1069400033F8103009B212B2084611461A4602F066
:10695000B7F8FB7903F10103FB71FB79772B8BD936
:106960004FF08703FB7170E0FA7940F62013C2F212
:1069700000034FEA82029B1893ED007AF7EE007A4B
:1069800077EE277A17EE900A05F07CFC02460B465C
:1069900043EC102B04F060FF53EC102B104619460B
:1069A00043A3D3E9002305F0EBFD02460B46144652
:1069B0001D4640F62053C2F200031B68184605F03E
:1069C00061FC02460B462046294605F0D9FD0246E9
:1069D0000B46104619463AA3D3E9002305F0A6FC5E
:1069E00002460B461046194605F062FF024640F685
:1069F0002853C2F200031A6040F62C53C2F200037F
:106A00001B781946FB799BB2C3F5BB739BB29AB254
:106A100040F62853C2F20003D3ED007AFCEEE77A89
:106A200017EE903ADBB2184643F6C433C0F60103C2
:106A300033F8103009B212B2084611461A4602F075
:106A40003FF8FB7903F10103FB71FB79FF2B8BD13D
:106A500040F62C53C2F200031B7803F10103DAB2B3
:106A600040F62C53C2F200031A7040F62C53C2F2C7
:106A700000031B78772B06D940F62C53C2F2000393
:106A80004FF000021A7040F62C53C2F200031B783C
:106A9000C3F59E7303F10303184602F0EDFA07F104
:106AA0001007BD46B0BD00BF9A9999999999B93F11
:106AB000EF39FAFE422EE63FAE47E17A14AEEF3FE1
:106AC0000000000000005940000000000000C84223
:106AD00080B588B000AF40F61963C2F200031B789E
:106AE000DBB2002B00F03C8240F6F803C2F2000358
:106AF0001B68012B40F0CE804FF40060C4F202000E
:106B00004FF400514FF00102FBF700FF07F10403BF
:106B100018464FF480714FF000024FF0010302F06D
:106B20002FFF07F10403184642F62C71C2F2000150
:106B300004F022FB40F60413C2F200031B78012B81
:106B40001ED04FF00003FB8315E0F98BFA8B42F661
:106B50002C73C2F200034FEA82029B181A6842F2B9
:106B60002873C2F200034FEA81015B181A60FB8BA5
:106B700003F10103FB83FA8B40F2FF139A42E4D93D
:106B800040F6F403C2F200031B6842F62C70C2F216
:106B900000001946FDF7E4FB07F1040318464FF423
:106BA00080714FF001024FF0010302F0E9FE07F19E
:106BB0000403184642F62C71C2F2000104F0DCFA1C
:106BC00040F6EE03C2F200031B78022B40D142F6DE
:106BD0002C70C2F2000043F22C71C2F200014FF49B
:106BE000807204F057FD4FF00003BB832DE0BB8B98
:106BF0004FEA4301BA8B43F22C73C2F200034FEA0F
:106C000082029B181A6842F62C73C2F200034FEA04
:106C100081015B181A60BB8B4FEA430303F101014A
:106C2000BA8B43F22C73C2F200034FEA82029B1824
:106C30001A6842F62C73C2F200034FEA81015B1816
:106C40001A60BB8B03F10103BB83BB8BFF2BCED937
:106C500042F62C70C2F200004FF40071FEF798FF6C
:106C6000F0EE407A40F60C13C2F20003C3ED007A56
:106C700040F6F803C2F200034FF000021A604FF42E
:106C80000060C4F202004FF400514FF00002FBF725
:106C90003DFE5EE140F6FC03C2F200031B68012BDF
:106CA00040F0A8804FF40060C4F202004FF400519D
:106CB0004FF00102FBF72AFE07F1040318464FF4D8
:106CC00080714FF000024FF0010302F059FE07F10E
:106CD0000403184641F22071C2F2000104F04CFA9C
:106CE00040F6F403C2F200031B6841F22070C2F2C6
:106CF00000001946FDF734FB07F1040318464FF472
:106D000080714FF001024FF0010302F039FE07F1EC
:106D10000403184641F22071C2F2000104F02CFA7B
:106D200040F6EE03C2F200031B78022B40D141F281
:106D30002070C2F2000043F22C71C2F200014FF445
:106D4000807204F0A7FC4FF000037B832DE07B8B67
:106D50004FEA43017A8B43F22C73C2F200034FEAED
:106D600082029B181A6841F22073C2F200034FEAB4
:106D700081015B181A607B8B4FEA430303F1010129
:106D80007A8B43F22C73C2F200034FEA82029B1803
:106D90001A6841F22073C2F200034FEA81015B18C6
:106DA0001A607B8B03F101037B837B8BFF2BCED996
:106DB00041F22070C2F200004FF40071FEF7E8FECD
:106DC000F0EE407A40F60C13C2F20003C3ED007AF5
:106DD00040F6FC03C2F200034FF000021A604FF4C9
:106DE0000060C4F202004FF400514FF00002FBF7C4
:106DF0008DFDAEE040F60013C2F200031B68012BCC
:106E000040F0A7804FF40060C4F202004FF400513C
:106E10004FF00102FBF77AFD07F1040318464FF427
:106E200080714FF000024FF0010302F0A9FD07F15D
:106E30000403184641F62071C2F2000104F09CF9E7
:106E400040F6F403C2F200031B6841F62070C2F260
:106E500000001946FDF784FA07F1040318464FF4C1
:106E600080714FF001024FF0010302F089FD07F13C
:106E70000403184641F62071C2F2000104F07CF9C7
:106E800040F6EE03C2F200031B78022B40D141F61C
:106E90002070C2F2000043F22C71C2F200014FF4E4
:106EA000807204F0F7FB4FF000033B832DE03B8B37
:106EB0004FEA43013A8B43F22C73C2F200034FEACC
:106EC00082029B181A6841F62073C2F200034FEA4F
:106ED00081015B181A603B8B4FEA430303F1010108
:106EE0003A8B43F22C73C2F200034FEA82029B18E2
:106EF0001A6841F62073C2F200034FEA81015B1861
:106F00001A603B8B03F101033B833B8BFF2BCED9F4
:106F100041F62070C2F200004FF40071FEF738FE17
:106F2000F0EE407A40F60C13C2F20003C3ED007A93
:106F300040F60013C2F200034FF000021A604FF453
:106F40000060C4F202004FF400514FF00002FBF762
:106F5000DDFC40F61963C2F200034FF000021A7024
:106F600040F6DC50C2F20000F9F7F6FC07F120070A
:106F7000BD4680BD80B500AFFDF75AFC024643F622
:106F80009873C2F200031A6043F69873C2F20003CA
:106F90001A6842F62873C2F200031B689A424AD06C
:106FA00042F62873C2F200031A6843F69873C2F2DD
:106FB00000031B68D31A1A4640F22403C2F20003EE
:106FC0001B6803FB02F240F22803C2F200031B68B5
:106FD000D3181A4640F22803C2F200031A6040F2A6
:106FE0002803C2F200031B68002B06DC40F22803D2
:106FF000C2F200034FF001021A6040F22803C2F20D
:1070000000031A6843F26043C0F23C239A4208DD51
:1070100040F22803C2F2000343F26042C0F23C2275
:107020001A6043F69873C2F200031A6842F6287396
:10703000C2F200031A6040F22803C2F200031A6889
:1070400040F6E803C2F200031B689A4207D040F200
:107050002803C2F200031B68184600F059FE80BDE9
:1070600080B584B002AFF871B9807A803B8097F91F
:107070000730A3F12E030B2B00F2E28001A252F89D
:1070800023F000BFB5700008417200081D720008AF
:10709000D9700008FD7000082171000845710008D2
:1070A000697100088D710008B1710008D571000880
:1070B000F9710008BA887B8839884FF01300009076
:1070C00001911046194642F23032C0F601024FF0EB
:1070D0000F0302F035FAC0E0BA887B8839884FF098
:1070E0001300009001911046194642F26C52C0F60E
:1070F00001024FF00F0302F023FAAEE0BA887B885A
:1071000039884FF01300009001911046194642F261
:10711000A872C0F601024FF00F0302F011FA9CE0D2
:10712000BA887B8839884FF013000090019110468F
:10713000194642F6E412C0F601024FF00F0302F0C6
:10714000FFF98AE0BA887B8839884FF013000090F5
:1071500001911046194642F62042C0F601024FF056
:107160000F0302F0EDF978E0BA887B8839884FF098
:107170001300009001911046194642F65C62C0F679
:1071800001024FF00F0302F0DBF966E0BA887B885A
:1071900039884FF01300009001911046194643F2D0
:1071A0009802C0F601024FF00F0302F0C9F954E053
:1071B000BA887B8839884FF01300009001911046FF
:1071C000194643F2D422C0F601024FF00F0302F039
:1071D000B7F942E0BA887B8839884FF013000090F5
:1071E00001911046194643F21052C0F601024FF0C9
:1071F0000F0302F0A5F930E0BA887B8839884FF098
:107200001300009001911046194643F24C72C0F6EB
:1072100001024FF00F0302F093F91EE0BA887B8859
:1072200039884FF01300009001911046194643F63B
:107230008812C0F601024FF00F0302F081F90CE052
:10724000BA887B884FF000010091104619464FF034
:107250000F024FF0130301F0D7FF07F10807BD46F7
:1072600080BD00BF80B500AF40F20C03C2F2000346
:107270001A684DF62913C6F24263A3FB02134FEAC4
:10728000136303F1FF3240F61413C2F200031A60D5
:107290004FF46053C4F202034FF46052C4F202028E
:1072A000126C42F002021A6440F67463C2F20003E8
:1072B0004FF48062C4F200021A6040F67463C2F2B6
:1072C00000034FF000029A6040F67463C2F20003BC
:1072D00040F21A42DA6040F61413C2F200031A6850
:1072E00040F67463C2F200035A6040F67463C2F25F
:1072F00000034FF000021A6140F67460C2F2000011
:10730000F9F792F840F67460C2F20000F9F76AF9F2
:107310004FF01D004FF000014FF00102FBF754FE4B
:107320004FF01D00FBF784FE4FF46053C4F20203DC
:107330004FF46052C4F20202126C42F004021A646A
:1073400040F6DC53C2F200034FF40062C4F20002C4
:107350001A6040F6DC53C2F200034FF000029A605C
:1073600040F6DC53C2F2000340F21A42DA6040F603
:107370001413C2F200031A6840F6DC53C2F2000391
:107380005A6040F6DC53C2F200034FF000021A616B
:1073900040F6DC50C2F20000F9F746F840F6DC5047
:1073A000C2F20000F9F71EF94FF01E004FF0020183
:1073B0004FF00402FBF708FE4FF01E00FBF738FE0B
:1073C00080BD00BF80B582B000AF7860FDF740FAA5
:1073D00007F10807BD4680BD80B500AF4FF460538C
:1073E000C4F202034FF46052C4F20202126C42F083
:1073F00000521A6443F68473C2F200034FF4E84269
:10740000C4F200021A6043F68470C2F20000FBF777
:10741000E1FA0346002B01D0FDF7A6F840F6181359
:10742000C2F200034FF000021A6040F61813C2F2D5
:1074300000034FF000025A6043F68470C2F200006D
:1074400040F61811C2F200014FF00002FBF780FB7A
:107450000346002B01D0FDF787F843F68470C2F293
:10746000000040F61811C2F200014FF01002FBF7C5
:107470006FFB0346002B01D0FDF776F843F68470CE
:10748000C2F200004FF000014FF008024FF08803F5
:10749000FBF734FC0346002B01D0FDF765F843F6FB
:1074A0008470C2F200004FF010014FF008024FF05C
:1074B0008803FBF723FC0346002B01D0FDF754F8AB
:1074C00043F68470C2F200004FF00001FBF7C2FAED
:1074D0000346002B01D0FDF747F843F68470C2F253
:1074E00000004FF01001FBF7B5FA0346002B01D066
:1074F000FDF73AF880BD00BF80B582B000AF03460B
:10750000FB80FB884FEA03534FEA1353FB80FB8851
:1075100043F68470C2F200004FF000014FF0000209
:10752000FBF7ECFB07F10807BD4680BD80B582B0D4
:1075300000AF0346FB80FB884FEA03534FEA135327
:10754000FB80FB8843F68470C2F200004FF010010C
:107550004FF00002FBF7D2FB07F10807BD4680BDE4
:1075600080B483B000AF786040F6D853C2F2000315
:107570007A681A6000BF40F6D853C2F200031B6855
:10758000002BF8D107F10C07BD4680BC704700BF47
:1075900080B586B000AF45F67453C0F601039B88F2
:1075A0007B604FF002033B614FF00203BB604FF082
:1075B0000203FB604FF001037B6145F67453C0F694
:1075C00001031A6807F1040310461946FAF7C4FDCF
:1075D00045F67C53C0F601039B887B604FF00203A5
:1075E0003B614FF00203BB604FF00203FB604FF0C2
:1075F00001037B6145F67C53C0F601031A6807F16D
:10760000040310461946FAF7A7FD45F68C53C0F659
:1076100001039B887B604FF002033B614FF0010345
:10762000BB604FF000037B614FF00003FB6045F649
:107630008C53C0F601031A6807F10403104619467B
:10764000FAF78AFD45F69453C0F601039B887B60E8
:107650004FF002033B614FF00103BB604FF00003AA
:107660007B614FF00003FB6045F69453C0F60103C5
:107670001A6807F1040310461946FAF76DFD45F63E
:107680008453C0F601039B887B604FF002033B618B
:107690004FF00303BB604FF00003FB604FF00003AB
:1076A0007B6145F68453C0F601031A6807F10403B1
:1076B00010461946FAF750FD45F6FC53C0F6010393
:1076C0009B887B604FF002033B614FF00003BB607F
:1076D0004FF00103FB604FF000037B6145F6FC5364
:1076E000C0F601031A6807F1040310461946FAF7B9
:1076F00033FD45F60463C0F601039B887B604FF0C1
:1077000002033B614FF00003BB604FF00103FB60DD
:107710004FF000037B6145F60463C0F601031A686D
:1077200007F1040310461946FAF716FD45F60C63F7
:10773000C0F601039B887B604FF002033B614FF072
:107740000003BB604FF00103FB604FF000037B615F
:1077500045F60C63C0F601031A6807F104031046EE
:107760001946FAF7F9FC45F61463C0F601039B8845
:107770007B604FF002033B614FF00303BB604FF0AF
:107780000003FB604FF000037B6145F61463C0F615
:1077900001031A6807F1040310461946FAF7DCFCE6
:1077A00045F61C63C0F601039B887B604FF0020323
:1077B0003B614FF00303BB604FF00003FB604FF0F1
:1077C00000037B6145F61C63C0F601031A6807F1EC
:1077D000040310461946FAF7BFFC45F6A453C0F659
:1077E00001039B887B604FF00103BB604FF00203F5
:1077F0003B614FF00103FB6045F6A453C0F6010363
:107800001A6807F1040310461946FAF7A5FC45F675
:10781000A453C0F601031A6845F6A453C0F6010349
:107820009B88104619464FF00002FBF76FF845F6AB
:10783000AC53C0F601039B887B604FF00103BB6033
:107840004FF002033B614FF00103FB6045F6AC5380
:10785000C0F601031A6807F1040310461946FAF747
:107860007BFC45F6AC53C0F601031A6845F6AC53F1
:10787000C0F601039B88104619464FF00002FBF743
:1078800045F845F6B453C0F601039B887B604FF082
:107890000103BB604FF002033B614FF00103FB604B
:1078A00045F6B453C0F601031A6807F10403104605
:1078B0001946FAF751FC45F6B453C0F601031A68AD
:1078C00045F6B453C0F601039B88104619464FF0A5
:1078D0000002FBF71BF845F6C453C0F601039B8872
:1078E0007B604FF00103BB604FF002033B614FF040
:1078F0000103FB6045F6C453C0F601031A6807F1A3
:10790000040310461946FAF727FC45F6C453C0F69F
:1079100001031A6845F6C453C0F601039B8810465C
:1079200019464FF00102FAF7F1FF45F6BC53C0F6D5
:1079300001039B887B604FF00103BB604FF00203A3
:107940003B614FF00103FB6045F6BC53C0F60103F9
:107950001A6807F1040310461946FAF7FDFB45F6CD
:10796000BC53C0F601031A6845F6BC53C0F60103C8
:107970009B88104619464FF00102FAF7C7FF45F6FB
:10798000CC53C0F601039B887B604FF00103BB60C2
:107990004FF002033B614FF00103FB6045F6CC530F
:1079A000C0F601031A6807F1040310461946FAF7F6
:1079B000D3FB45F6CC53C0F601031A6845F6CC5309
:1079C000C0F601039B88104619464FF00002FAF7F3
:1079D0009DFF45F6DC53C0F601039B887B604FF0AA
:1079E0000103BB604FF002033B614FF00103FB60FA
:1079F00045F6DC53C0F601031A6807F1040310468C
:107A00001946FAF7A9FB45F6DC53C0F601031A68DC
:107A100045F6DC53C0F601039B88104619464FF02B
:107A20000102FAF773FF45F6D453C0F601039B88B1
:107A30007B604FF00103BB604FF002033B614FF0EE
:107A40000103FB6045F6D453C0F601031A6807F141
:107A5000040310461946FAF77FFB45F6D453C0F6E7
:107A600001031A6845F6D453C0F601039B881046FB
:107A700019464FF00102FAF749FF45F62463C0F6B4
:107A800001039A8845F62C63C0F601039B881343D3
:107A90009BB27B604FF00303BB604FF00003FB60C1
:107AA00045F62463C0F601031A6807F10403104683
:107AB0001946FAF751FB07F11807BD4680BD00BF14
:107AC00080B500AF45F6C453C0F601031A6845F609
:107AD000C453C0F601039B88104619464FF00102BB
:107AE000FAF714FF45F6DC53C0F601031A6845F6B1
:107AF000DC53C0F601039B88104619464FF0010283
:107B0000FAF704FF45F6BC53C0F601031A6845F6C0
:107B1000BC53C0F601039B88104619464FF0000283
:107B2000FAF7F4FE45F6D453C0F601031A6845F699
:107B3000D453C0F601039B88104619464FF000024B
:107B4000FAF7E4FE80BD00BF80B584B000AF024606
:107B50000B46FA80BB804FF00003FB6075E045F6F2
:107B6000B453C0F60103196845F6B453C0F60103D7
:107B70009A88F888FB68C3F10F0340FA03F3DBB27D
:107B800003F00103DBB2084611461A46FAF7BEFEBF
:107B900045F6CC53C0F60103196845F6CC53C0F640
:107BA00001039A88B888FB68C3F10F0340FA03F316
:107BB000DBB203F00103DBB2084611461A46FAF7BE
:107BC000A5FE45F6C453C0F601031A6845F6C45332
:107BD000C0F601039B88104619464FF00002FAF7E1
:107BE00095FE45F6DC53C0F601031A6845F6DC53F2
:107BF000C0F601039B88104619464FF00002FAF7C1
:107C000085FE45F6C453C0F601031A6845F6C45311
:107C1000C0F601039B88104619464FF00102FAF79F
:107C200075FE45F6DC53C0F601031A6845F6DC53D1
:107C3000C0F601039B88104619464FF00102FAF77F
:107C400065FEFB6803F10103FB60FB680F2B86DD1B
:107C500007F11007BD4680BD80B500AF45F6BC53A7
:107C6000C0F601031A6845F6BC53C0F601039B88B1
:107C7000104619464FF00102FAF748FE45F6D45374
:107C8000C0F601031A6845F6D453C0F601039B8879
:107C9000104619464FF00102FAF738FE80BD00BFCA
:107CA00080B588B000AFC7E9000117A3D3E900236E
:107CB000C7E906234FF080524FF00003C7E90423C1
:107CC0007B683A6902FB03F27B69396801FB03F3C5
:107CD000D1183A683B69A2FB0323C9180B46C7E9D0
:107CE0000223C7E90223D7E90201D7E9062304F0FA
:107CF0002FFE02460B461046194607F12007BD46E7
:107D000080BD00BFAFF30080C068780400000000B1
:107D10002DE9B04384B000AF786079680A464FEA35
:107D2000E27310461946FFF7BBFF02460B46C7E950
:107D3000022345F6A453C0F601031A6845F6A4537E
:107D4000C0F601039B88104619464FF00102FAF76E
:107D5000DDFDFFF7B5FE4FF408504FF40851FFF773
:107D6000F3FEFFF779FF45F6A453C0F601031A6846
:107D700045F6A453C0F601039B88104619464FF000
:107D80000102FAF7C3FDFFF79BFE3B894FEA8343ED
:107D90004FEA93439BB243F480439BB29AB23B8930
:107DA0004FEA83434FEA93439BB243F480439BB231
:107DB0009BB210461946FFF7C7FEFFF74DFFFFF7CE
:107DC0007FFEFB684FEA8343BA684FEA923843EA82
:107DD0000808FB684FEAA3391FFA88F34FEA834388
:107DE0004FEA93439BB243F480439BB29AB2FB6841
:107DF0004FEA8343B9684FEA91341C43FB684FEA6A
:107E0000A335A3B24FEA83434FEA93439BB243F4B3
:107E100080439BB29BB210461946FFF795FEFFF7D1
:107E20001BFFFFF74DFE4FF440404FF44C41FFF76E
:107E30008BFEFFF711FF45F6A453C0F601031A6845
:107E400045F6A453C0F601039B88104619464FF02F
:107E50000002FAF75BFD07F11007BD46BDE8B083ED
:107E600080B500AF40F67263C2F200034FF000022B
:107E70001A8040F6D453C2F200034FF000021A8079
:107E800040F62163C2F200034FF000021A7040F680
:107E90007063C2F200034FF000021A8040F61963CB
:107EA000C2F200034FF000021A7040F61863C2F2EB
:107EB00000034FF000021A704FF46053C4F2020343
:107EC0004FF46052C4F20202526C42F480725A645F
:107ED0004FF46053C4F202034FF46052C4F2020242
:107EE000526C42F400725A644FF46053C4F20203BD
:107EF0004FF46052C4F20202126B42F001021A63A4
:107F00004FF46053C4F202034FF46052C4F2020211
:107F1000526A42F480725A624FF46053C4F2020310
:107F20004FF46052C4F20202526A22F480725A6222
:107F300040F62463C2F200034FF40052C4F201027F
:107F40001A6040F62463C2F200034FF000025A6048
:107F500040F62463C2F200034FF000029A6040F63C
:107F60002463C2F200034FF000021A6140F624635A
:107F7000C2F200034FF001029A6140F62463C2F29C
:107F800000034FF000025A6240F62463C2F200037D
:107F90004FF000029A6240F62463C2F200034FF0F1
:107FA0000002DA6240F62463C2F200034FF00002DE
:107FB0001A6340F62463C2F200034FF00002DA6055
:107FC00040F62463C2F200034FF001021A6240F649
:107FD0002463C2F200034FF00002DA6140F624632A
:107FE000C2F200034FF000025A6140F62460C2F270
:107FF0000000FBF739F80346002B0CD040F618635D
:10800000C2F200031B7803F10103DAB240F61863F1
:10801000C2F200031A7040F69053C2F200034FF40C
:108020000452C4F201021A6040F69053C2F20003F7
:108030004FF000025A6040F69053C2F200034FF036
:1080400000029A6040F69053C2F200034FF0000223
:108050001A6140F69053C2F200034FF001029A6198
:1080600040F69053C2F200034FF000025A6240F60D
:108070009053C2F200034FF000029A6240F6905310
:10808000C2F200034FF00002DA6240F69053C2F2EF
:1080900000034FF000021A6340F69053C2F200034F
:1080A0004FF00002DA6040F69053C2F200034FF046
:1080B00001021A6240F69053C2F200034FF0000230
:1080C000DA6140F69053C2F200034FF000025A61A9
:1080D00040F69050C2F20000FAF7C6FF0346002BAC
:1080E0000CD040F61863C2F200031B7803F10103C1
:1080F000DAB240F61863C2F200031A7040F67C53FD
:10810000C2F200034FF001021A6040F67C53C2F243
:1081100000034FF001025A6040F67C53C2F20003A4
:108120004FF000029A6040F67C53C2F200034FF019
:108130000002DA6040F6B063C2F200034FF00202C0
:108140001A6040F6B063C2F200034FF001025A60B9
:1081500040F6B063C2F200034FF000029A6040F6AE
:10816000B063C2F200034FF00002DA6040F6246010
:10817000C2F2000040F67C51C2F20001FBF7DCF9CC
:108180000346002B0CD040F61863C2F200031B78A4
:1081900003F10103DAB240F61863C2F200031A7069
:1081A00040F69050C2F2000040F6B061C2F2000109
:1081B000FBF7C2F90346002B0CD040F61863C2F25D
:1081C00000031B7803F10103DAB240F61863C2F230
:1081D00000031A7080BD00BF80B500AF40F6246078
:1081E000C2F200004FF00A01FBF756F940F690503A
:1081F000C2F200004FF00A01FBF74EF940F624608E
:10820000C2F20000FBF754FB0346152B22D140F6C7
:108210009050C2F20000FBF74BFB0346152B19D11F
:1082200040F62460C2F20000FBF778F903469AB2E8
:1082300040F67263C2F200031A8040F69050C2F218
:108240000000FBF76BF903469AB240F6D453C2F232
:1082500000031A8080BD00BF80B500AF40F62460E7
:10826000C2F20000FBF778F80346002B0CD040F672
:108270001863C2F200031B7803F10103DAB240F67F
:108280001863C2F200031A7040F69050C2F2000068
:10829000FBF762F80346002B0CD040F61863C2F2DD
:1082A00000031B7803F10103DAB240F61863C2F24F
:1082B00000031A7080BD00BF80B500AFFBF7D2FC91
:1082C0004FF46D43CEF200034FF46D42CEF2000244
:1082D000D2F8882042F47002C3F88820FBF702FC31
:1082E00000F002F880BD00BF80B592B000AF4FF43F
:1082F0006053C4F202034FF46052C4F20202126CE3
:1083000042F080521A644FF4E043C4F200034FF489
:10831000E042C4F20002126842F440421A604FF098
:1083200001037B604FF00103BB604FF00203FB6170
:108330004FF480033B624FF018037B624FF4A87345
:10834000BB624FF00203FB624FF007033B6307F190
:1083500004031846F8F7C6FF4FF00F037B634FF096
:108360000203BB634FF00003FB634FF4A0533B6475
:108370004FF480537B6407F1340318464FF0050136
:10838000F9F768FB07F14807BD4680BD80B483B0AC
:1083900000AF03463960FB7197F90730002B10DA04
:1083A0004FF46D43CEF20003FA7902F00F02A2F10E
:1083B00004013A68D2B24FEA0212D2B25B181A76BE
:1083C0000DE04FF46143CEF2000397F907103A68CD
:1083D000D2B24FEA0212D2B25B1883F8002307F13F
:1083E0000C07BD4680BC704780B582B000AF786096
:1083F0007B6803F1FF326FF07F439A4202D94FF05E
:1084000001031DE04EF21003CEF200037A6802F180
:10841000FF325A604FF0FF304FF00F01FFF7B6FF09
:108420004EF21003CEF200034FF000029A604EF2BB
:108430001003CEF200034FF007021A604FF0000362
:10844000184607F10807BD4680BD00BF80B500AFE4
:1084500040F20C03C2F200031A6844F6D353C1F28F
:108460006203A3FB02134FEA93131846FFF7BCFF06
:1084700080BD00BF80B400AF44F63813C2F20003E1
:108480001B68002B0BD044F63813C2F200031B68A4
:1084900003F1FF3244F63813C2F200031A60BD46FE
:1084A00080BC704780B586B000AF4FF46053C4F213
:1084B00002034FF46052C4F20202126B42F0040253
:1084C0001A634FF400537B604FF00103BB604FF021
:1084D00002033B614FF00103FB6007F104034FF41B
:1084E0000060C4F202001946F9F736FE4FF400604E
:1084F000C4F202004FF400514FF00002FAF706FAFE
:1085000007F11807BD4680BDF0B595B012AF034620
:10851000FB7145F68C53C0F601031A6845F68C537F
:10852000C0F601039B88104619464FF00002FAF787
:10853000EDF945F6F453C0F601031A6845F6F45315
:10854000C0F601039B88104619464FF00002FAF767
:10855000DDF945F69C53C0F601031A6845F69C53B5
:10856000C0F601039B88104619464FF00002FAF747
:10857000CDF944F63C13C2F20003FA791A7040F6C2
:10858000C466C2F2000644F64013C2F200030F9321
:1085900044F63C13C2F2000310934FF00103119311
:1085A0006C4606F110050FCD0FC40FCD0FC40FCDD3
:1085B0000FC495E8070084E8070096E80F00FBF772
:1085C000D7FC45F69C53C0F601031A6845F69C5348
:1085D000C0F601039B88104619464FF00102FAF7D6
:1085E00095F907F10C07BD46F0BD00BFF0B595B099
:1085F00012AF0346FB7145F68C53C0F601031A68AF
:1086000045F68C53C0F601039B88104619464FF07F
:108610000102FAF77BF945F6F453C0F601031A6834
:1086200045F6F453C0F601039B88104619464FF0F7
:108630000002FAF76BF945F69C53C0F601031A687D
:1086400045F69C53C0F601039B88104619464FF02F
:108650000002FAF75BF944F63C13C2F20003FA7920
:108660001A7040F6C466C2F2000644F64013C2F225
:1086700000030F9344F63C13C2F2000310934FF033
:10868000010311936C4606F110050FCD0FC40FCDF9
:108690000FC40FCD0FC495E8070084E8070096E8E3
:1086A0000F00FBF765FC45F69C53C0F601031A6802
:1086B00045F69C53C0F601039B88104619464FF0BF
:1086C0000102FAF723F907F10C07BD46F0BD00BF20
:1086D00080B500AF45F69453C0F601031A6845F61D
:1086E0009453C0F601039B88104619464FF00102CF
:1086F000FAF70CF94FF00500FEF732FF45F69453F8
:10870000C0F601031A6845F69453C0F601039B882E
:10871000104619464FF00002FAF7F8F84FF014002F
:10872000FEF71EFF45F69453C0F601031A6845F69E
:108730009453C0F601039B88104619464FF001027E
:10874000FAF7E4F84FF09600FEF70AFF45F69C535F
:10875000C0F601031A6845F69C53C0F601039B88D6
:10876000104619464FF00002FAF7D0F84FF0EF002C
:10877000FFF7CAFE4FF00300FFF738FF4FF080000D
:10878000FFF734FF4FF00200FFF730FF4FF0CF004C
:10879000FFF7BAFE4FF00000FFF728FF4FF0C100CF
:1087A000FFF724FF4FF03000FFF720FF4FF0ED0000
:1087B000FFF7AAFE4FF06400FFF718FF4FF0030029
:1087C000FFF714FF4FF01200FFF710FF4FF081008A
:1087D000FFF70CFF4FF0E800FFF796FE4FF0850023
:1087E000FFF704FF4FF00000FFF700FF4FF07800A5
:1087F000FFF7FCFE4FF0CB00FFF786FE4FF039008D
:10880000FFF7F4FE4FF02C00FFF7F0FE4FF00000F2
:10881000FFF7ECFE4FF03400FFF7E8FE4FF00200E8
:10882000FFF7E4FE4FF0F700FFF76EFE4FF0200079
:10883000FFF7DCFE4FF0EA00FFF766FE4FF00000A6
:10884000FFF7D4FE4FF00000FFF7D0FE4FF0C0005E
:10885000FFF75AFE4FF02300FFF7C8FE4FF0C100AC
:10886000FFF752FE4FF01000FFF7C0FE4FF0C500BB
:10887000FFF74AFE4FF03E00FFF7B8FE4FF028002A
:10888000FFF7B4FE4FF0C700FFF73EFE4FF0860043
:10889000FFF7ACFE4FF03600FFF736FE4FF0480012
:1088A000FFF7A4FE4FF03A00FFF72EFE4FF0550001
:1088B000FFF79CFE4FF0B100FFF726FE4FF00000DF
:1088C000FFF794FE4FF01800FFF790FE4FF0B60050
:1088D000FFF71AFE4FF00800FFF788FE4FF0820006
:1088E000FFF784FE4FF02700FFF780FE4FF0F20005
:1088F000FFF70AFE4FF00000FFF778FE4FF026006A
:10890000FFF702FE4FF00100FFF770FE4FF0E000AE
:10891000FFF7FAFD4FF00F00FFF768FE4FF0310050
:10892000FFF764FE4FF02B00FFF760FE4FF00C00E6
:10893000FFF75CFE4FF00E00FFF758FE4FF0080007
:10894000FFF754FE4FF04E00FFF750FE4FF0F100DE
:10895000FFF74CFE4FF03700FFF748FE4FF00700DF
:10896000FFF744FE4FF01000FFF740FE4FF003000A
:10897000FFF73CFE4FF00E00FFF738FE4FF0090006
:10898000FFF734FE4FF00000FFF730FE4FF0E1003C
:10899000FFF7BAFD4FF00000FFF728FE4FF00E0082
:1089A000FFF724FE4FF01400FFF720FE4FF0030006
:1089B000FFF71CFE4FF01100FFF718FE4FF0070005
:1089C000FFF714FE4FF03100FFF710FE4FF0C1002B
:1089D000FFF70CFE4FF04800FFF708FE4FF00800CD
:1089E000FFF704FE4FF00F00FFF700FE4FF00C0002
:1089F000FFF7FCFD4FF03100FFF7F8FD4FF03600B8
:108A0000FFF7F4FD4FF00F00FFF7F0FD4FF01100FE
:108A1000FFF77AFD4FF07800FEF7A2FD4FF0290036
:108A2000FFF772FD80BD00BF80B582B000AFF88057
:108A3000B9807A803B804FF02A00FFF765FDFB8804
:108A40004FEA13239BB2DBB21846FFF7CFFDFB883A
:108A5000DBB21846FFF7CAFD7B884FEA13239BB2AF
:108A6000DBB21846FFF7C2FD7B88DBB21846FFF782
:108A7000BDFD4FF02B00FFF747FDBB884FEA1323E6
:108A80009BB2DBB21846FFF7B1FDBB88DBB21846DC
:108A9000FFF7ACFD3B884FEA13239BB2DBB21846CD
:108AA000FFF7A4FD3B88DBB21846FFF79FFD4FF0B0
:108AB0002C00FFF729FD07F10807BD4680BD00BF68
:108AC000F0B599B012AF13460246FA800A46BA8052
:108AD0007B80B7F90630002B7BDB40F66863C2F27F
:108AE00000031B88B7F906201BB29A4271DAB7F966
:108AF0000430002B6DDB40F66E63C2F200031B886E
:108B0000B7F904201BB29A4263DAF888B988FB8867
:108B100003F101039AB2BB8803F101039BB2FFF793
:108B200083FF45F68C53C0F601031A6845F68C5353
:108B3000C0F601039B88104619464FF00102F9F771
:108B4000E5FE45F69C53C0F601031A6845F69C53B2
:108B5000C0F601039B88104619464FF00002F9F752
:108B6000D5FE7B884FEA13239BB2DBB23B727B8836
:108B7000DBB27B7240F6C466C2F2000607F10C035A
:108B80000F9307F1080310934FF0020311936C4603
:108B900006F110050FCD0FC40FCD0FC40FCD0FC4BC
:108BA00095E8070084E8070096E80F00FBF7E0F976
:108BB00045F69C53C0F601031A6845F69C53C0F66F
:108BC00001039B88104619464FF00102F9F79EFEFB
:108BD00000E000BF07F11C07BD46F0BDF0B599B03D
:108BE00012AFF880B9807A803B8040F66863C2F2A9
:108BF00000031B88B7F906201BB29A4280F29880C6
:108C000040F66E63C2F200031B88B7F904201BB262
:108C10009A4280F28D80B7F90420B7F90230D31858
:108C200003F1FF3240F66E63C2F200031B881BB2F1
:108C30009A4209DB40F66E63C2F200031B889AB2C7
:108C4000BB88D31A9BB27B80F888B988FA88BC8825
:108C50007B88E3189BB203F1FF339BB2FFF7E4FE7E
:108C60003B884FEA13239BB2FB753B88BB7545F6E7
:108C70008C53C0F601031A6845F68C53C0F6010305
:108C80009B88104619464FF00102F9F73FFE45F662
:108C90009C53C0F601031A6845F69C53C0F60103C5
:108CA0009B88104619464FF00002F9F72FFE21E08D
:108CB000FB7D3B72BB7D7B7240F6C466C2F2000650
:108CC00007F10C030F9307F1080310934FF0020311
:108CD00011936C4606F110050FCD0FC40FCD0FC4D4
:108CE0000FCD0FC495E8070084E8070096E80F0051
:108CF000FBF73EF9B7F90230002B0CBF002301232C
:108D0000DBB27A8802F1FF327A80002BD0D145F6AF
:108D10009C53C0F601031A6845F69C53C0F6010344
:108D20009B88104619464FF00102F9F7EFFD00E06D
:108D300000BF07F11C07BD46F0BD00BFF0B597B0FE
:108D400012AFF880B9807A803B8040F66863C2F247
:108D500000031B88B7F906201BB29A4280F2A48058
:108D600040F66E63C2F200031B88B7F904201BB201
:108D70009A4280F29980B7F90620B7F90230D318E9
:108D800003F1FF3240F66863C2F200031B881BB296
:108D90009A4209DB40F66863C2F200031B889AB26C
:108DA000FB88D31A9BB27B80F888B988FA887B88C5
:108DB000D3189BB203F1FF339AB2BB88FFF734FE9E
:108DC0003B884FEA13239BB2FB733B88BB7345F68A
:108DD0008C53C0F601031A6845F68C53C0F60103A4
:108DE0009B88104619464FF00102F9F78FFD45F6B2
:108DF0009C53C0F601031A6845F69C53C0F6010364
:108E00009B88104619464FF00002F9F77FFD2DE0D0
:108E100044F63C13C2F20003FA7B1A7044F63C138A
:108E2000C2F20003BA7B5A7040F6C466C2F2000672
:108E300044F64013C2F200030F9344F63C13C2F20F
:108E4000000310934FF0020311936C4606F11005D6
:108E50000FCD0FC40FCD0FC40FCD0FC495E8070081
:108E600084E8070096E80F00FBF782F8B7F90230B4
:108E7000002B0CBF00230123DBB27A8802F1FF3202
:108E80007A80002BC4D145F69C53C0F601031A68C2
:108E900045F69C53C0F601039B88104619464FF0D7
:108EA0000102F9F733FD00E000BF07F11407BD46EA
:108EB000F0BD00BFF0B597B012AFF880B9807A80EE
:108EC0003B8040F66863C2F200031B88B7F90620B6
:108ED0001BB29A4280F2CB8040F66E63C2F200036E
:108EE0001B88B7F904201BB29A4280F2C080B7F900
:108EF0000620B7F90230D31803F1FF3240F6686359
:108F0000C2F200031B881BB29A4209DB40F6686379
:108F1000C2F200031B889AB2FB88D31A9BB27B80F3
:108F2000B7F90420B7F90030D31803F1FF3240F647
:108F30006E63C2F200031B881BB29A4209DB40F643
:108F40006E63C2F200031B889AB2BB88D31A9BB22D
:108F50003B80F888B988FA887B88D3189BB203F1E4
:108F6000FF339AB2BC883B88E3189BB203F1FF330E
:108F70009BB2FFF759FD3B8D4FEA13239BB2FB7366
:108F80003B8DBB7345F68C53C0F601031A6845F65A
:108F90008C53C0F601039B88104619464FF001021E
:108FA000F9F7B4FC45F69C53C0F601031A6845F680
:108FB0009C53C0F601039B88104619464FF00002EF
:108FC000F9F7A4FC3B88BB803CE07B88FB8031E068
:108FD00044F63C13C2F20003FA7B1A7044F63C13C9
:108FE000C2F20003BA7B5A7040F6C466C2F20006B1
:108FF00044F64013C2F200030F9344F63C13C2F24E
:10900000000310934FF0020311936C4606F1100514
:109010000FCD0FC40FCD0FC40FCD0FC495E80700BF
:1090200084E8070096E80F00FAF7A2FFFB8803F137
:10903000FF33FB80B7F90630002BC9DCBB8803F196
:10904000FF33BB80B7F90430002BBEDC45F69C53E0
:10905000C0F601031A6845F69C53C0F601039B88CD
:10906000104619464FF00102F9F750FC00E000BF2E
:1090700007F11407BD46F0BD80B582B000AF0346CE
:10908000FB804FF03700FFF73FFAFB884FEA1323CE
:109090009BB2DBB21846FFF7A9FAFB88DBB2184691
:1090A000FFF7A4FA07F10807BD4680BD80B582B07E
:1090B00000AF13460246FA800A46BA807B80FA88DF
:1090C000BB88D2187B88D318B3F5A07F2BD14FF083
:1090D0003300FFF719FAFB884FEA13239BB2DBB288
:1090E0001846FFF783FAFB88DBB21846FFF77EFAD3
:1090F000BB884FEA13239BB2DBB21846FFF776FA20
:10910000BB88DBB21846FFF771FA7B884FEA13235E
:109110009BB2DBB21846FFF769FA7B88DBB21846D0
:10912000FFF764FA00E000BF07F10807BD4680BD05
:1091300080B584B000AF0346FB714FF03600FFF7F7
:10914000E3F9FB7903F00303FB60FB68032B57D8BB
:1091500001A252F823F000BF699100088F91000826
:10916000B5910008DB9100084FF04800FFF73EFA88
:1091700040F66863C2F200034FF0F0021A8040F636
:109180006E63C2F200034FF4A0721A8038E04FF011
:109190002800FFF72BFA40F66863C2F200034FF491
:1091A000A0721A8040F66E63C2F200034FF0F00224
:1091B0001A8025E04FF08800FFF718FA40F6686340
:1091C000C2F200034FF0F0021A8040F66E63C2F262
:1091D00000034FF4A0721A8012E04FF0E800FFF78E
:1091E00005FA40F66863C2F200034FF4A0721A80D9
:1091F00040F66E63C2F200034FF0F0021A8000BF27
:1092000007F11007BD4680BD80B584B000AFF8807F
:10921000B9807A803B80FB88FB810CE0B7F90E00B7
:10922000B7F90410B7F900203B8BFFF7D7FCFB8997
:1092300003F10103FB81B7F90E20B7F90610B7F966
:109240000230CB189A42E9DB07F11007BD4680BD1A
:1092500080B584B002AF0346FB8040F66863C2F27B
:1092600000031A8840F66E63C2F200031B8812B234
:109270001BB2F98800914FF000004FF00001FFF79A
:1092800019FE07F10807BD4680BD00BF80B58CB050
:1092900000AFF880B9807A803B80B7F90420B7F935
:1092A00000309A420BDDBB887B843B88BB807B8C83
:1092B0003B80FB883B847B88FB803B8C7B80B7F9C1
:1092C0000020B7F93C309A420BDDBB8FFB833B8813
:1092D000BB87FB8B3B803B8FBB837B883B87BB8BF8
:1092E0007B80B7F90420B7F900309A420BDDBB88C8
:1092F0007B833B88BB807B8B3B80FB883B837B886D
:10930000FB803B8B7B80B7F90420B7F93C309A4255
:1093100037D1FB88BB85BB8DFB85B7F90220B7F938
:109320002E309A4202DA7B88FB8507E0B7F90220EB
:10933000B7F92C309A4201DD7B88BB85B7F938201C
:10934000B7F92E309A4202DA3B8FFB8507E0B7F976
:109350003820B7F92C309A4201DD3B8FBB85BA8D9E
:10936000FB8DD31A9BB203F101039BB29BB2B7F9F9
:109370002E00B7F904101AB2B7F84030FFF7DEFC40
:10938000D9E07A88FB88D31A9BB2FB823A88BB88E3
:10939000D31A9BB2BB823A8FFB88D31A9BB27B82D3
:1093A000BA8FBB88D31A9BB23B823A8F7B88D31A81
:1093B0009BB2FB81BA8F3B88D31A9BB2BB814FF023
:1093C0000003FB844FF00003BB84B7F90020B7F91A
:1093D0003C309A4202D13B883B8504E03B8803F154
:1093E000FF339BB23B85BB887B8540E0B7F92620E5
:1093F000B7F9143092FBF3F39AB2FB88D3189BB2FF
:10940000FB85B7F92420B7F9103092FBF3F39AB239
:10941000FB88D3189BB2BB85FA8CFB8AD3189BB20E
:10942000FB84BA8C7B8AD3189BB2BB84B7F92E20FD
:10943000B7F92C309A4205DDFB8D7B81BB8DFB8516
:109440007B89BB85BA8DFB8DD31A9BB203F10103D7
:109450009BB29BB2B7F92E00B7F92A101AB2B7F82F
:109460004030FFF76BFC7B8D03F101037B85B7F97F
:109470002A20B7F928309A42B8DDB7F92A20B7F97F
:109480000030D31A9BB2FA8902FB03F39BB2FB8430
:10949000B7F92A20B7F90430D31A9BB27A8A02FBB3
:1094A00003F39BB2BB8440E0B7F92620B7F90C3038
:1094B00092FBF3F39AB27B88D3189BB2FB85B7F982
:1094C0002420B7F9103092FBF3F39AB2FB88D3183B
:1094D0009BB2BB85FA8CFB89D3189BB2FB84BA8CF8
:1094E0007B8AD3189BB2BB84B7F92E20B7F92C30F6
:1094F0009A4205DDFB8D3B81BB8DFB853B89BB859E
:10950000BA8DFB8DD31A9BB203F101039BB29BB2C0
:10951000B7F92E00B7F92A101AB2B7F84030FFF7A2
:109520000DFC7B8D03F101037B85B7F92A20B7F988
:109530003C309A42B8DD07F13007BD4680BD00BF20
:1095400080B586B000AFBA600246FA810A46BA8199
:10955000FB804FF00003BB8235E04FF00003FB823D
:1095600027E0FB88BA8A02FB03F39AB2FB8AD3187E
:109570009BB27B82FA89FB8AD3189BB299B2BA89D3
:10958000BB8AD3189BB29AB2B7F912304FEA4303A1
:10959000B868C3181888BB8C03409BB209B212B2DA
:1095A000084611461A46FFF78BFAFB8A03F10103BE
:1095B000FB82B7F91620B7F906309A42D1DBBB8A95
:1095C00003F10103BB82B7F91420B7F920309A42A6
:1095D000C3DB07F11807BD4680BD00BFB0B584B03E
:1095E00002AF0346FB71FB790A2B1DD140F66D6378
:1095F000C2F200031B784FEAC3039AB240F68C53C1
:10960000C2F200031B889BB2D3189BB29AB240F6F9
:109610008C53C2F200031A8040F66A63C2F2000360
:109620004FF000021A807FE0FB790D2B7CD040F6D2
:109630006A63C2F20003198840F68C53C2F2000339
:109640001A8840F6C263C2F200031C8840F6C06369
:10965000C2F200031D8840F66D63C2F20003187861
:1096600009B212B2FB7900950190084611461A46DC
:10967000234600F05DF840F66D63C2F200031B78EC
:109680001A464FEA4202D3184FEA43039AB240F611
:109690006A63C2F200031B889BB2D3189BB29AB2D2
:1096A00040F66A63C2F200031A8040F66C63C2F2AD
:1096B00000031B78002B37D040F66A63C2F2000328
:1096C0001B8819B240F66863C2F200031B8818B207
:1096D00040F66D63C2F200031B781A4613464FEA48
:1096E00082029B1A4FEA4303C31899421CDD40F6DD
:1096F0006D63C2F200031B784FEAC3039AB240F6CF
:109700008C53C2F200031B889BB2D3189BB29AB24F
:1097100040F68C53C2F200031A8040F66A63C2F22C
:1097200000034FF000021A8007F10807BD46B0BDE4
:1097300090B587B002AFF880B980FA703B804FF0E7
:109740000003FB73BDE097F90F30052B03D14FF0F9
:109750000003BB730FE0FA7813464FEA83039B18AC
:109760001A4697F90F30D21845F63463C0F6010354
:10977000D3181B78BB734FF000037B7398E0BB7B5F
:1097800003F00103DBB2002B43D097F82430012B08
:1097900016D197F90F309AB2FB88D3189BB29AB2C0
:1097A00097F90D3099B2BB88CB189BB29BB211B21E
:1097B0001AB23B88084611461A46FFF781F96FE056
:1097C00097F90F309BB297F8242092B202FB03F373
:1097D0009AB2FB88D3189BB298B297F90D309BB21E
:1097E00097F8242092B202FB03F39AB2BB88D318F5
:1097F0009BB299B297F824309AB297F824309BB272
:1098000000B209B212B21BB23C880094FFF7FCFC14
:1098100046E03A8C3B889A4242D097F82430012B9C
:1098200016D197F90F309AB2FB88D3189BB29AB22F
:1098300097F90D3099B2BB88CB189BB29BB211B28D
:109840001AB23B8C084611461A46FFF739F927E051
:1098500097F90F309BB297F8242092B202FB03F3E2
:109860009AB2FB88D3189BB298B297F90D309BB28D
:1098700097F8242092B202FB03F39AB2BB88D31864
:109880009BB299B297F824309AB297F824309BB2E1
:1098900000B209B212B21BB23C8C0094FFF7B4FCC8
:1098A000BB7B4FEA5303BB737B7B03F101037B73E9
:1098B00097F90D30072B7FF762AFFB7B03F10103B4
:1098C000FB7397F90F30052B7FF73DAF07F11407B6
:1098D000BD4690BD80B483B000AF02460B46FA800F
:1098E000BB8040F66A63C2F20003FA881A8040F631
:1098F0008C53C2F20003BA881A8007F10C07BD46E8
:1099000080BC704780B483B000AF0346FB71FB7925
:10991000002B01D0FA7901E04FF0010240F66D63AF
:10992000C2F200031A7007F10C07BD4680BC7047F5
:1099300080B483B000AF02460B46FA80BB8040F68D
:10994000C263C2F20003FA881A8040F6C063C2F212
:109950000003BA881A8007F10C07BD4680BC704727
:1099600080B483B000AF0346FB7140F66C63C2F273
:109970000003FA791A7007F10C07BD4680BC7047E6
:1099800080B485B000AF786079807A703B704FF01A
:109990000003FB737B687A881A807A6846F6407306
:1099A000C0F6010353607B687A789A707B683A78D6
:1099B000DA707B681B88B3F5807F2ED0B3F5807F8B
:1099C00004DC102B47D0402B36D053E0B3F5806F2A
:1099D00014D0B3F5805F4DD17B684FF001029A81BE
:1099E0007B684FF00102DA817A6846F24073C0F674
:1099F000010393607B68294A1A613FE07B684FF05E
:109A000004029A817B684FF00402DA817B681F4A66
:109A10009A607B68224A1A6130E07B684FF010023E
:109A20009A817B684FF01002DA817B68184A9A604D
:109A30007B681C4A1A6121E07B684FF040029A81E2
:109A40007B684FF04002DA817B68124A9A607B683B
:109A5000154A1A6112E07B684FF480729A817B6824
:109A60004FF48072DA817B680B4A9A607B680F4AF8
:109A70001A6103E04FF0FF03FB7300BFFB7B5BB297
:109A8000184607F11407BD4680BC704746670108B9
:109A90005E670108BE6701083E6901080000803961
:109AA0000000803A0000803B0000803C0000803DC8
:109AB00080B4C1B000AFF8607A600A467A813B8119
:109AC0007B89C7F8F430D7F8F430C7F8E430D7F81A
:109AD000F4304FEA9303C7F8F4304FF00003C7F8AF
:109AE000F8304FF00003C7F8FC30D7F8F430C7F86F
:109AF000F030D7F8F820D7F8F430D318C7F8E030B2
:109B0000D7F8E020D7F8F430D318C7F8DC30D7F80E
:109B1000DC20D7F8F430D318C7F8D830D7F8F830AD
:109B20004FEAC303FA68D3181B68C7F8D430D7F8D4
:109B3000F8304FEAC30303F10403FA68D3181B6833
:109B4000C7F8D030D7F8E0304FEAC303FA68D3182B
:109B50001B68C7F8CC30D7F8E0304FEAC30303F1F5
:109B60000403FA68D3181B68C7F8C830D7F8DC308C
:109B70004FEAC303FA68D3181B68C7F8C430D7F894
:109B8000DC304FEAC30303F10403FA68D3181B68FF
:109B9000C7F8C030D7F8D8304FEAC303FA68D318F3
:109BA0001B68C7F8BC30D7F8D8304FEAC30303F1BD
:109BB0000403FA68D3181B68C7F8B83097ED357AF4
:109BC000D7ED317A77EE277AC7ED2D7A97ED337A94
:109BD000D7ED2F7A77EE277AC7ED2C7A97ED347A86
:109BE000D7ED307A77EE277AC7ED2B7A97ED327A78
:109BF000D7ED2E7A77EE277AC7ED2A7AD7F8FC20B0
:109C0000D7F8FC30D318C7F8A430D7F8A4304FEAFF
:109C1000C3037A68D3181B68C7F8A030D7F8A430FC
:109C20004FEAC30303F104037A68D3181B68C7F82B
:109C30009C3097ED357AD7ED317A77EE677AC7EDBC
:109C4000267A97ED337AD7ED2F7A77EE677AC7EDDC
:109C5000257A97ED347AD7ED307A77EE677AC7EDCB
:109C6000247A97ED327AD7ED2E7A77EE677AC7EDC0
:109C7000237AD7F8F8304FEAC303FA68D31897ED80
:109C80002D7AD7ED2C7A77EE277AC3ED007AD7F8C4
:109C9000F8304FEAC30303F10403FA68D31897EDD1
:109CA0002B7AD7ED2A7A77EE277AC3ED007A97EDF3
:109CB000267AD7ED237A77EE277AC7ED227A97EDC9
:109CC000247AD7ED257A77EE677AC7ED217A97ED7A
:109CD0002D7AD7ED2C7A77EE677AC7ED207A97ED5B
:109CE0002B7AD7ED2A7A77EE677AC7ED1F7A97ED50
:109CF000267AD7ED237A77EE677AC7ED1E7A97ED4D
:109D0000257AD7ED247A77EE277AC7ED1D7AD7F832
:109D1000FC304FEAC3037A68D3181B683B67D7F857
:109D2000FC304FEAC30303F104037A68D3181B68BD
:109D3000FB66D7F8A420D7F8FC30D318BB66BB6EFF
:109D40004FEAC3037A68D3181B687B66BB6E4FEA81
:109D5000C30303F104037A68D3181B683B6697EDCD
:109D6000227AD7ED1C7A67EE277AC7ED177A97ED3E
:109D7000217AD7ED1C7A67EE277AC7ED167A97ED30
:109D8000207AD7ED287A67EE277AC7ED157A97ED16
:109D90001F7AD7ED287A67EE277AC7ED147A97ED08
:109DA0001E7AD7ED197A67EE277AC7ED137A97ED09
:109DB0001D7AD7ED197A67EE277AC7ED127A97EDFB
:109DC000217AD7ED1B7A67EE277AC7ED117A97EDE6
:109DD000227AD7ED1B7A67EE277AC7ED107A97EDD6
:109DE0001F7AD7ED277A67EE277AC7ED0F7A97EDBE
:109DF000207AD7ED277A67EE277AC7ED0E7A97EDAE
:109E00001D7AD7ED187A67EE277AC7ED0D7A97EDB0
:109E10001E7AD7ED187A67EE277AC7ED0C7A97EDA0
:109E2000177AD7ED117A77EE277AC7ED177A97ED83
:109E3000167AD7ED107A77EE677AC7ED167A97ED36
:109E4000157AD7ED0F7A77EE277AC7ED157A97ED69
:109E5000147AD7ED0E7A77EE677AC7ED147A97ED1C
:109E6000137AD7ED0D7A77EE277AC7ED137A97ED4F
:109E7000127AD7ED0C7A77EE677AC7ED127AD7F8B7
:109E8000E0304FEAC303FA68D3187A6D1A60D7F846
:109E9000E0304FEAC30303F10403FA68D3183A6DC4
:109EA0001A60D7F8DC304FEAC303FA68D318FA6DAA
:109EB0001A60D7F8DC304FEAC30303F10403FA68F1
:109EC000D318BA6D1A60D7F8D8304FEAC303FA68CE
:109ED000D318FA6C1A60D7F8D8304FEAC30303F1ED
:109EE0000403FA68D318BA6C1A603B89D7F8FC20CF
:109EF000D318C7F8FC30D7F8F83003F10103C7F8DE
:109F0000F830D7F8F03003F1FF33C7F8F030D7F866
:109F1000F030002B7FF4EDAD3B894FEA83033B81AA
:109F20007B894FEA93039BB2C7F8EC303DE2D7F848
:109F3000F430C7F8E430D7F8F4304FEA9303C7F8A9
:109F4000F4304FF00003C7F8FC304FF00003C7F8BF
:109F5000F030D7F8FC20D7F8FC30D318C7F8A4307D
:109F6000D7F8A420D7F8FC30D318BB66D7F8FC305C
:109F70004FEAC3037A68D3181B683B67D7F8FC30F5
:109F80004FEAC30303F104037A68D3181B68FB6626
:109F9000D7F8A4304FEAC3037A68D3181B68C7F810
:109FA000A030D7F8A4304FEAC30303F104037A6862
:109FB000D3181B68C7F89C30BB6E4FEAC3037A689E
:109FC000D3181B687B66BB6E4FEAC30303F104031F
:109FD0007A68D3181B683B663B89D7F8FC20D318F6
:109FE000C7F8FC30D7F8F030C7F8F830D7F8F820C9
:109FF000D7F8F430D318C7F8E030D7F8E020D7F816
:10A00000F430D318C7F8DC30D7F8DC20D7F8F430B8
:10A01000D318C7F8D830D7F8F8304FEAC303FA6836
:10A02000D3181B68C7F8D430D7F8F8304FEAC30309
:10A0300003F10403FA68D3181B68C7F8D030D7F8C7
:10A04000E0304FEAC303FA68D3181B68C7F8CC3076
:10A05000D7F8E0304FEAC30303F10403FA68D318DA
:10A060001B68C7F8C830D7F8DC304FEAC303FA687A
:10A07000D3181B68C7F8C430D7F8DC304FEAC303E5
:10A0800003F10403FA68D3181B68C7F8C030D7F887
:10A09000D8304FEAC303FA68D3181B68C7F8BC303E
:10A0A000D7F8D8304FEAC30303F10403FA68D31892
:10A0B0001B68C7F8B83097ED357AD7ED317A77EE6F
:10A0C000677AC7ED267A97ED337AD7ED2F7A77EE58
:10A0D000677AC7ED257A97ED347AD7ED307A77EE47
:10A0E000677AC7ED247A97ED327AD7ED2E7A77EE3C
:10A0F000677AC7ED237A97ED357AD7ED317A77EE27
:10A10000277AC7ED2D7A97ED337AD7ED2F7A77EE50
:10A11000277AC7ED2C7A97ED347AD7ED307A77EE3F
:10A12000277AC7ED2B7A97ED327AD7ED2E7A77EE34
:10A13000277AC7ED2A7A97ED267AD7ED237A77EE3C
:10A14000277AC7ED227A97ED247AD7ED257A77EE34
:10A15000677AC7ED217A97ED2D7AD7ED2C7A77EED5
:10A16000677AC7ED207A97ED2B7AD7ED2A7A77EECA
:10A17000677AC7ED1F7A97ED267AD7ED237A77EEC7
:10A18000677AC7ED1E7A97ED257AD7ED247A77EEB8
:10A19000277AC7ED1D7AD7F8F8304FEAC303FA687B
:10A1A000D31897ED2D7AD7ED2C7A77EE277AC3ED79
:10A1B000007AD7F8F8304FEAC30303F10403FA68D2
:10A1C000D31897ED2B7AD7ED2A7A77EE277AC3ED5D
:10A1D000007A97ED227AD7ED1C7A67EE277AC7EDE1
:10A1E000177A97ED217AD7ED1C7A67EE277AC7EDBB
:10A1F000167A97ED207AD7ED287A67EE277AC7EDA1
:10A20000157A97ED1F7AD7ED287A67EE277AC7ED92
:10A21000147A97ED1E7AD7ED197A67EE277AC7ED93
:10A22000137A97ED1D7AD7ED197A67EE277AC7ED85
:10A23000127A97ED217AD7ED1B7A67EE277AC7ED70
:10A24000117A97ED227AD7ED1B7A67EE277AC7ED60
:10A25000107A97ED1F7AD7ED277A67EE277AC7ED48
:10A260000F7A97ED207AD7ED277A67EE277AC7ED38
:10A270000E7A97ED1D7AD7ED187A67EE277AC7ED3B
:10A280000D7A97ED1E7AD7ED187A67EE277AC7ED2B
:10A290000C7A97ED177AD7ED117A77EE277AC7ED1A
:10A2A000177A97ED167AD7ED107A77EE677AC7EDC1
:10A2B000167A97ED157AD7ED0F7A77EE277AC7EDF4
:10A2C000157A97ED147AD7ED0E7A77EE677AC7EDA7
:10A2D000147A97ED137AD7ED0D7A77EE277AC7EDDA
:10A2E000137A97ED127AD7ED0C7A77EE677AC7ED8D
:10A2F000127AD7F8E0304FEAC303FA68D3187A6DC0
:10A300001A60D7F8E0304FEAC30303F10403FA6898
:10A31000D3183A6D1A60D7F8DC304FEAC303FA68F5
:10A32000D318FA6D1A60D7F8DC304FEAC30303F193
:10A330000403FA68D318BA6D1A60D7F8D8304FEA18
:10A34000C303FA68D318FA6C1A60D7F8D8304FEA0A
:10A35000C30303F10403FA68D318BA6C1A60D7F880
:10A36000F820D7F8E430D318C7F8F8307A89D7F84E
:10A37000F8309A423FF63AAED7F8F03003F10103D5
:10A38000C7F8F030D7F8F43003F1FF32D7F8F030E7
:10A390009A42BFF4DEAD3B894FEA83033B81D7F895
:10A3A000EC304FEA9303C7F8EC30D7F8EC30042BCD
:10A3B0003FF6BDAD7B894FEA93039BB2C7F8F030FF
:10A3C000FB68C7F8E830D7F8E8301B68C7F8D43026
:10A3D000D7F8E8305B68C7F8D030D7F8E8309B682A
:10A3E000C7F8CC30D7F8E830DB68C7F8C830D7F802
:10A3F000E8301B69C7F8C430D7F8E8305B69C7F8A4
:10A40000C030D7F8E8309B69C7F8BC30D7F8E830DF
:10A41000DB69C7F8B83097ED357AD7ED317A77EE4A
:10A42000277AC7ED2D7A97ED357AD7ED317A77EE29
:10A43000677AC7ED267A97ED347AD7ED307A77EEE2
:10A44000277AC7ED2B7A97ED347AD7ED307A77EE0D
:10A45000677AC7ED247A97ED337AD7ED2F7A77EEC6
:10A46000277AC7ED2C7A97ED327AD7ED2E7A77EEF0
:10A47000277AC7ED2A7A97ED337AD7ED2F7A77EEE0
:10A48000677AC7ED257A97ED327AD7ED2E7A77EE97
:10A49000677AC7ED237A97ED2D7AD7ED2C7A77EE90
:10A4A000277AC7ED0B7A97ED2B7AD7ED2A7A77EEDC
:10A4B000277AC7ED0A7A97ED2D7AD7ED2C7A77EEC9
:10A4C000677AC7ED097A97ED2B7AD7ED2A7A77EE7E
:10A4D000677AC7ED087A97ED267AD7ED237A77EE7B
:10A4E000277AC7ED077A97ED247AD7ED257A77EEAC
:10A4F000677AC7ED067A97ED267AD7ED237A77EE5D
:10A50000677AC7ED057A97ED257AD7ED247A77EE4D
:10A51000277AC7ED047AD7F8E830FA6A1A60D7F8D4
:10A52000E83003F10403BA6A1A60D7F8E83003F19F
:10A5300008037A6A1A60D7F8E83003F10C033A6A24
:10A540001A60D7F8E83003F11003FA691A60D7F8F7
:10A55000E83003F11403BA691A60D7F8E83003F160
:10A5600018037A691A60D7F8E83003F11C033A69D6
:10A570001A60D7F8E83003F12003C7F8E830D7F8BD
:10A58000F03003F1FF33C7F8F030D7F8F030002B8C
:10A590007FF419AF07F58277BD4680BC704700BFD6
:10A5A00080B4C3B000AFF86007F1040002601A463F
:10A5B0003B4683ED000A0B467B8107F108031A80B6
:10A5C0007B89C7F8FC30D7F8FC30C7F8EC30D7F8F7
:10A5D000FC304FEA9303C7F8FC304FF00003C7F894
:10A5E00000314FF00003C7F80431D7F8FC30C7F84A
:10A5F000F830D7F80021D7F8FC30D318C7F8E83086
:10A60000D7F8E820D7F8FC30D318C7F8E430D7F8EB
:10A61000E420D7F8FC30D318C7F8E030D7F8003181
:10A620004FEAC303FA68D3181B68C7F8DC30D7F8C1
:10A6300000314FEAC30303F10403FA68D3181B681F
:10A64000C7F8D830D7F8E4304FEAC303FA68D31814
:10A650001B68C7F8D430D7F8E4304FEAC30303F1DE
:10A660000403FA68D3181B68C7F8D030D7F8E8306D
:10A670004FEAC303FA68D3181B68C7F8CC30D7F881
:10A68000E8304FEAC30303F10403FA68D3181B68E8
:10A69000C7F8C830D7F8E0304FEAC303FA68D318D8
:10A6A0001B68C7F8C430D7F8E0304FEAC30303F1A2
:10A6B0000403FA68D3181B68C7F8C03097ED377ADF
:10A6C000D7ED357A77EE277AC7ED2F7A97ED337A83
:10A6D000D7ED317A77EE277AC7ED2E7A97ED367A75
:10A6E000D7ED347A77EE277AC7ED2D7A97ED327A67
:10A6F000D7ED307A77EE277AC7ED2C7AD7F8042198
:10A70000D7F80431D318C7F8AC30D7F8AC304FEADB
:10A71000C30307F104021268D3181B68C7F8A830F6
:10A72000D7F8AC304FEAC30303F1040307F1040286
:10A730001268D3181B68C7F8A43097ED377AD7EDA5
:10A74000357A77EE677AC7ED287A97ED337AD7EDC9
:10A75000317A77EE677AC7ED277A97ED367AD7EDBB
:10A76000347A77EE677AC7ED267A97ED327AD7EDAD
:10A77000307A77EE677AC7ED257AD7F800314FEA5D
:10A78000C303FA68D31897ED2F7AD7ED2E7A77EEB8
:10A79000277AC3ED007AD7F800314FEAC30303F1FB
:10A7A0000403FA68D31897ED2D7AD7ED2C7A77EE5B
:10A7B000277AC3ED007A97ED287AD7ED257A77EEE0
:10A7C000677AC7ED247A97ED267AD7ED277A77EE68
:10A7D000277AC7ED237A97ED2F7AD7ED2E7A77EE89
:10A7E000677AC7ED227A97ED2D7AD7ED2C7A77EE3E
:10A7F000677AC7ED217A97ED287AD7ED257A77EE3B
:10A80000277AC7ED207A97ED267AD7ED277A77EE6B
:10A81000677AC7ED1F7AD7F804314FEAC30307F10F
:10A8200004021268D3181B68BB67D7F804314FEADB
:10A83000C30303F1040307F104021268D3181B6871
:10A840007B67D7F8AC20D7F80431D3183B673B6F50
:10A850004FEAC30307F104021268D3181B68FB66B2
:10A860003B6F4FEAC30303F1040307F104021268CC
:10A87000D3181B68BB6697ED247AD7ED1E7A67EE76
:10A88000277AC7ED197A97ED237AD7ED1E7A67EE0E
:10A89000277AC7ED187A97ED227AD7ED2A7A67EEF4
:10A8A000277AC7ED177A97ED217AD7ED2A7A67EEE6
:10A8B000277AC7ED167A97ED207AD7ED1B7A67EEE7
:10A8C000277AC7ED157A97ED1F7AD7ED1B7A67EED9
:10A8D000277AC7ED147A97ED237AD7ED1D7A67EEC4
:10A8E000277AC7ED137A97ED247AD7ED1D7A67EEB4
:10A8F000277AC7ED127A97ED217AD7ED297A67EE9C
:10A90000277AC7ED117A97ED227AD7ED297A67EE8B
:10A91000277AC7ED107A97ED1F7AD7ED1A7A67EE8E
:10A92000277AC7ED0F7A97ED207AD7ED1A7A67EE7E
:10A93000277AC7ED0E7A97ED197AD7ED137A77EE6D
:10A94000677AC7ED197A97ED187AD7ED127A77EE14
:10A95000277AC7ED187A97ED177AD7ED117A77EE47
:10A96000677AC7ED177A97ED167AD7ED107A77EEFA
:10A97000277AC7ED167A97ED157AD7ED0F7A77EE2D
:10A98000677AC7ED157A97ED147AD7ED0E7A77EEE0
:10A99000277AC7ED147AD7F8E8304FEAC303FA688C
:10A9A000D318FA6D1A60D7F8E8304FEAC30303F101
:10A9B0000403FA68D318BA6D1A60D7F8E4304FEA86
:10A9C000C303FA68D3187A6E1A60D7F8E4304FEAF6
:10A9D000C30303F10403FA68D3183A6E1A60D7F878
:10A9E000E0304FEAC303FA68D3187A6D1A60D7F8DB
:10A9F000E0304FEAC30303F10403FA68D3183A6D59
:10AA00001A6007F108031B88D7F80421D318C7F888
:10AA10000431D7F8003103F10103C7F80031D7F84A
:10AA2000F83003F1FF33C7F8F830D7F8F830002BCF
:10AA30007FF4DFAD07F1080307F1080212884FEA3F
:10AA400082021A807B894FEA93039BB2C7F8F430E5
:10AA50004FE2D7F8FC30C7F8EC30D7F8FC304FEABB
:10AA60009303C7F8FC304FF00003C7F804314FF0F0
:10AA70000003C7F8F830D7F80421D7F80431D31809
:10AA8000C7F8AC30D7F8AC20D7F80431D3183B67FF
:10AA9000D7F804314FEAC30307F104021268D31850
:10AAA0001B68BB67D7F804314FEAC30303F1040303
:10AAB00007F104021268D3181B687B67D7F8AC3023
:10AAC0004FEAC30307F104021268D3181B68C7F8E2
:10AAD000A830D7F8AC304FEAC30303F1040307F101
:10AAE00004021268D3181B68C7F8A4303B6F4FEA02
:10AAF000C30307F104021268D3181B68FB663B6F9F
:10AB00004FEAC30303F1040307F104021268D318E8
:10AB10001B68BB6607F108031B88D7F80421D3180C
:10AB2000C7F80431D7F8F830C7F80031D7F800215A
:10AB3000D7F8FC30D318C7F8E830D7F8E820D7F8B2
:10AB4000FC30D318C7F8E430D7F8E420D7F8FC304D
:10AB5000D318C7F8E030D7F800314FEAC303FA68DA
:10AB6000D3181B68C7F8DC30D7F800314FEAC303AD
:10AB700003F10403FA68D3181B68C7F8D830D7F874
:10AB8000E8304FEAC303FA68D3181B68C7F8CC3023
:10AB9000D7F8E8304FEAC30303F10403FA68D31887
:10ABA0001B68C7F8C830D7F8E4304FEAC303FA6827
:10ABB000D3181B68C7F8D430D7F8E4304FEAC30382
:10ABC00003F10403FA68D3181B68C7F8D030D7F82C
:10ABD000E0304FEAC303FA68D3181B68C7F8C430E3
:10ABE000D7F8E0304FEAC30303F10403FA68D3183F
:10ABF0001B68C7F8C03097ED377AD7ED357A77EE16
:10AC0000677AC7ED287A97ED337AD7ED317A77EE08
:10AC1000677AC7ED277A97ED367AD7ED347A77EEF3
:10AC2000677AC7ED267A97ED327AD7ED307A77EEEC
:10AC3000677AC7ED257A97ED377AD7ED357A77EED3
:10AC4000277AC7ED2F7A97ED337AD7ED317A77EE01
:10AC5000277AC7ED2E7A97ED367AD7ED347A77EEEC
:10AC6000277AC7ED2D7A97ED327AD7ED307A77EEE5
:10AC7000277AC7ED2C7A97ED287AD7ED257A77EEEB
:10AC8000677AC7ED247A97ED267AD7ED277A77EEA3
:10AC9000277AC7ED237A97ED2F7AD7ED2E7A77EEC4
:10ACA000677AC7ED227A97ED2D7AD7ED2C7A77EE79
:10ACB000677AC7ED217A97ED287AD7ED257A77EE76
:10ACC000277AC7ED207A97ED267AD7ED277A77EEA7
:10ACD000677AC7ED1F7AD7F800314FEAC303FA68E5
:10ACE000D31897ED2F7AD7ED2E7A77EE277AC3ED2A
:10ACF000007AD7F800314FEAC30303F10403FA687E
:10AD0000D31897ED2D7AD7ED2C7A77EE277AC3ED0D
:10AD1000007A97ED247AD7ED1E7A67EE277AC7ED91
:10AD2000197A97ED237AD7ED1E7A67EE277AC7ED69
:10AD3000187A97ED227AD7ED2A7A67EE277AC7ED4F
:10AD4000177A97ED217AD7ED2A7A67EE277AC7ED41
:10AD5000167A97ED207AD7ED1B7A67EE277AC7ED42
:10AD6000157A97ED1F7AD7ED1B7A67EE277AC7ED34
:10AD7000147A97ED237AD7ED1D7A67EE277AC7ED1F
:10AD8000137A97ED247AD7ED1D7A67EE277AC7ED0F
:10AD9000127A97ED217AD7ED297A67EE277AC7EDF7
:10ADA000117A97ED227AD7ED297A67EE277AC7EDE7
:10ADB000107A97ED1F7AD7ED1A7A67EE277AC7EDEA
:10ADC0000F7A97ED207AD7ED1A7A67EE277AC7EDDA
:10ADD0000E7A97ED197AD7ED137A77EE677AC7ED89
:10ADE000197A97ED187AD7ED127A77EE277AC7EDB0
:10ADF000187A97ED177AD7ED117A77EE677AC7ED63
:10AE0000177A97ED167AD7ED107A77EE277AC7ED95
:10AE1000167A97ED157AD7ED0F7A77EE677AC7ED48
:10AE2000157A97ED147AD7ED0E7A77EE277AC7ED7B
:10AE3000147AD7F8E8304FEAC303FA68D318FA6DEA
:10AE40001A60D7F8E8304FEAC30303F10403FA6845
:10AE5000D318BA6D1A60D7F8E4304FEAC303FA6822
:10AE6000D3187A6E1A60D7F8E4304FEAC30303F1BF
:10AE70000403FA68D3183A6E1A60D7F8E0304FEA44
:10AE8000C303FA68D3187A6D1A60D7F8E0304FEA36
:10AE9000C30303F10403FA68D3183A6D1A60D7F8B4
:10AEA0000021D7F8EC30D318C7F800317A89D7F8E9
:10AEB00000319A423FF63AAED7F8F83003F1010379
:10AEC000C7F8F830D7F8FC3003F1FF32D7F8F83084
:10AED0009A42BFF4D0AD07F1080307F108021288C7
:10AEE0004FEA82021A80D7F8F4304FEA9303C7F88A
:10AEF000F430D7F8F430042B3FF6ABAD7B894FEA42
:10AF000093039BB2C7F8F830FB68C7F8F030D7F866
:10AF1000F0301B68C7F8DC30D7F8F0305B68C7F852
:10AF2000D830D7F8F0309B68C7F8CC30D7F8F0307D
:10AF3000DB68C7F8C830D7F8F0301B69C7F8D430E1
:10AF4000D7F8F0305B69C7F8D030D7F8F0309B699C
:10AF5000C7F8C430D7F8F030DB69C7F8C03097EDD8
:10AF6000377AD7ED357A77EE277AC7ED2F7A97EDD6
:10AF7000377AD7ED357A77EE677AC7ED287A97ED8D
:10AF8000367AD7ED347A77EE277AC7ED2D7A97EDBA
:10AF9000367AD7ED347A77EE677AC7ED267A97ED71
:10AFA000337AD7ED317A77EE277AC7ED2E7A97ED9F
:10AFB000327AD7ED307A77EE277AC7ED2C7A97ED93
:10AFC000337AD7ED317A77EE677AC7ED277A97ED46
:10AFD000327AD7ED307A77EE677AC7ED257A97ED3A
:10AFE0002F7AD7ED2E7A77EE277AC7ED0D7A97ED87
:10AFF0002D7AD7ED2C7A77EE277AC7ED0C7A97ED7C
:10B000002F7AD7ED2E7A77EE677AC7ED0B7A97ED28
:10B010002D7AD7ED2C7A77EE677AC7ED0A7A97ED1D
:10B02000287AD7ED257A77EE677AC7ED097A97ED1A
:10B03000267AD7ED277A77EE277AC7ED087A97ED4B
:10B04000287AD7ED257A77EE277AC7ED077A97ED3C
:10B05000267AD7ED277A77EE677AC7ED067A3B46F0
:10B0600097ED0D7AD3ED007A67EE277AC7ED137A64
:10B070003B4697ED0C7AD3ED007A67EE277AC7ED61
:10B08000127A3B4697ED0B7AD3ED007A67EE277A7A
:10B09000C7ED117A3B4697ED0A7AD3ED007A67EE59
:10B0A000277AC7ED107A3B4697ED097AD3ED007AFF
:10B0B00067EE277AC7ED0F7A3B4697ED087AD3ED16
:10B0C000007A67EE277AC7ED0E7A3B4697ED077A4E
:10B0D000D3ED007A67EE277AC7ED057A3B4697ED08
:10B0E000067AD3ED007A67EE277AC7ED047AD7F8AF
:10B0F000F030FA6C1A60D7F8F03003F10403BA6C40
:10B100001A60D7F8F03003F108037A6C1A60D7F8A8
:10B11000F03003F10C033A6C1A60D7F8F03003F109
:10B120001003FA6B1A60D7F8F03003F11403BA6B0E
:10B130001A60D7F8F03003F118037A691A60D7F86B
:10B14000F03003F11C033A691A60D7F8F03003F1CC
:10B150002003C7F8F030D7F8F83003F1FF33C7F811
:10B16000F830D7F8F830002B7FF4D1AE07F58677AA
:10B17000BD4680BC704700BF80B582B000AF78602C
:10B1800039607B689B78012B0ED17B6819887B68BE
:10B190005A687B689B897868D0ED047A3868B0EE8D
:10B1A000670AFFF7FDF908E07B6819887B685A6831
:10B1B0007B689B893868FEF77BFC7B68DB78012B1A
:10B1C00008D17B6819887B68DA897B689B68386856
:10B1D00000F004F807F10807BD4680BD80B489B0CF
:10B1E00000AFF8607B600B467B8113463B814FF0DC
:10B1F0000003BB837B894FEA53037B837B894FEA40
:10B2000053039BB203F101033B834FF00003FB8325
:10B21000E5E0FA8BBB8B9A4280F08880FB8B4FEA8B
:10B22000C303FA68D3181B687B61FB8B4FEAC30327
:10B23000FA68D318BA8B4FEAC202F9688A18126802
:10B240001A60BB8B4FEAC303FA68D3187A691A6095
:10B25000FB8B4FEAC30303F10403FA68D3181B689E
:10B260007B61FB8B4FEAC30303F10403FA68D31835
:10B27000BA8B4FEAC20202F10402F9688A18126816
:10B280001A60BB8B4FEAC30303F10403FA68D318B7
:10B290007A691A60FA8B3B8BD3184FEAC303FA68BA
:10B2A000D3181B687B61FA8B3B8BD3184FEAC3031F
:10B2B000FA68D318B98B3A8B8A184FEAC202F96838
:10B2C0008A1812681A60BA8B3B8BD3184FEAC303F3
:10B2D000FA68D3187A691A60FA8B3B8BD3184FEA55
:10B2E000C30303F10403FA68D3181B687B61FA8B6C
:10B2F0003B8BD3184FEAC30303F10403FA68D31856
:10B30000B98B3A8B8A184FEAC20202F10402F9683B
:10B310008A1812681A60BA8B3B8BD3184FEAC303A2
:10B3200003F10403FA68D3187A691A60FB8B03F1FE
:10B3300001034FEAC303FA68D3181B687B61FB8BD8
:10B3400003F101034FEAC303FA68D318B98B7A8B70
:10B350008A184FEAC202F9688A1812681A60BA8B12
:10B360007B8BD3184FEAC303FA68D3187A691A6043
:10B37000FB8B03F101034FEAC30303F10403FA68F3
:10B38000D3181B687B61FB8B03F101034FEAC303F6
:10B3900003F10403FA68D318B98B7A8B8A184FEA41
:10B3A000C20202F10402F9688A1812681A60BA8BA4
:10B3B0007B8BD3184FEAC30303F10403FA68D31855
:10B3C0007A691A607B681B88BB833B894FEA430319
:10B3D0007A68D3187B60FB8B03F10203FB83FA8B43
:10B3E0007B8BA3F102039A427FF613AF07F1240788
:10B3F000BD4680BC704700BF80B49BB000AF87EDF6
:10B40000010A4FF48073FB6597ED017ADFED887ACE
:10B4100067EE277AC7ED167AD7ED167AFDEEE77A52
:10B4200017EE903A3B66D7ED017AF5EEC07AF1EE71
:10B4300010FA54BF00230123DBB2002B03D03B6E74
:10B4400003F1FF333B663B6E06EE903AF8EEE67A88
:10B4500097ED167A77EE677AC7ED167AFB6D07EEF1
:10B46000903AB8EE677AD7ED167A67EE277AFCEE57
:10B47000E77A17EE903A7B66FB6D06EE903AB8EEEF
:10B48000667AD7ED167A27EE277A7B6E06EE903A2B
:10B49000F8EEE67A77EE677AC7ED157A7B6E002BC9
:10B4A00003DA4FF000037B6606E07B6EB3F5807F26
:10B4B00002DD4FF480737B667B6E4FEA830246F2B7
:10B4C0003033C0F60103D3183B653B6D1B68FB644A
:10B4D0003B6D5B68BB643B6D9B687B643B6DDB686D
:10B4E0003B6497ED157AD7ED157A67EE277AC7EDAD
:10B4F0000F7A97ED157AF6EE007A67EE277AC7EDA8
:10B500000E7A97ED157ADFED4B7A67EE277AC7ED65
:10B510000D7A97ED157ADFED487A67EE277AC7ED59
:10B520000C7A97ED0F7AF6EE007A67EE277AC7ED80
:10B530000B7A97ED0E7AD7ED0F7A67EE277AC7ED83
:10B540000A7A97ED0D7AD7ED0F7A67EE277AC7ED75
:10B55000097AB7EE007AD7ED0E7A77EE677AC7ED03
:10B56000087A97ED0B7AD7ED0C7A77EE677AC7ED0C
:10B57000077A97ED0B7AD7ED157A77EE277AC7ED34
:10B58000067A97ED077AD7ED097A77EE677AC7EDF5
:10B59000057A97ED0A7AD7ED0F7A77EE677AC7EDDD
:10B5A000077A97ED057AD7ED137A67EE277AC7ED1C
:10B5B000047A97ED067AD7ED0A7A77EE677AC7EDC7
:10B5C000067A97ED097AD7ED0D7A77EE677AC7EDAF
:10B5D000037A97ED077AD7ED087A77EE277AC7EDE9
:10B5E000077A97ED127AD7ED077A27EE277AD7ED0B
:10B5F000047A37EE277AD7ED116AD7ED067A66EE30
:10B60000A76A97ED106AD7ED037A66EE277A76EE91
:10B61000A77A77EE277AC7ED047A3B6907EE903A6E
:10B62000B0EE670A07F16C07BD4680BC704700BFEB
:10B6300083F9223EABAA2A3EABAAAA3E80B582B0CD
:10B6400000AF87ED010A3860D7ED017AF5EEC07AD8
:10B65000F1EE10FAD4BF00230123DBB2002B0BD094
:10B6600097ED010A00F07EF9F0EE407A3B68C3EDF9
:10B67000007A4FF0000304E03B68054A1A604FF07F
:10B68000FF035BB2184607F10807BD4680BD00BF47
:10B690000000000080B588B000AFF860B9607A6043
:10B6A0007B684FEA9303FB619BE0FB681B68BB610F
:10B6B000FB6803F10403FB60FB681B687B61FB68AC
:10B6C00003F10403FB6097ED067AD7ED067A27EEC7
:10B6D000277AD7ED056AD7ED057A66EEA77A77EE79
:10B6E000277ABB68BA6802F10402BA60B0EE670A52
:10B6F0001846FFF7A3FFFB681B68BB61FB6803F1FB
:10B700000403FB60FB681B687B61FB6803F10403B7
:10B71000FB6097ED067AD7ED067A27EE277AD7ED0C
:10B72000056AD7ED057A66EEA77A77EE277ABB68C9
:10B73000BA6802F10402BA60B0EE670A1846FFF771
:10B740007DFFFB681B68BB61FB6803F10403FB60C2
:10B75000FB681B687B61FB6803F10403FB6097EDEA
:10B76000067AD7ED067A27EE277AD7ED056AD7ED68
:10B77000057A66EEA77A77EE277ABB68BA6802F197
:10B780000402BA60B0EE670A1846FFF757FFFB687D
:10B790001B68BB61FB6803F10403FB60FB681B686B
:10B7A0007B61FB6803F10403FB6097ED067AD7ED3C
:10B7B000067A27EE277AD7ED056AD7ED057A66EE89
:10B7C000A77A77EE277ABB68BA6802F10402BA60FA
:10B7D000B0EE670A1846FFF731FFFB6903F1FF334C
:10B7E000FB61FB69002B7FF460AF7B6803F0030310
:10B7F000FB6129E0FB681B68BB61FB6803F1040384
:10B80000FB60FB681B687B61FB6803F10403FB6062
:10B8100097ED067AD7ED067A27EE277AD7ED056AF7
:10B82000D7ED057A66EEA77A77EE277ABB68BA6815
:10B8300002F10402BA60B0EE670A1846FFF7FEFE96
:10B84000FB6903F1FF33FB61FB69002BD2D107F1E8
:10B850002007BD4680BD00BFD0B52DED048BB0EEF6
:10B86000408AF0EE608A3C4C8AB000F0D5F894F93A
:10B870000030B0EE409AF0EE609A013335D0B0EE71
:10B88000480AF0EE680A00F029FB00282DD051ECA0
:10B89000180B0022002300F0D9FF30BB2F4B247877
:10B8A0000193002308938DED028B8DED048B002C0A
:10B8B00023D000270026CFF6F07751EC180B00229A
:10B8C0000023CDE9066700F099FF002825D0022368
:10B8D0009C42009336D0684600F038FB002831D0F7
:10B8E000089B002B27D19DED069BB0EE490AF0EE98
:10B8F000690A0AB0BDEC048BD0BD4FF6FF774FF05C
:10B900006046CCF2EF7751EC180B00220023CDE912
:10B91000066700F073FF0028D9D10123022C0093A1
:10B9200015D0684600F012FB88B10D4800F010FBFE
:10B930008DED060BD4E701F003FB089B9DED069B04
:10B940000360D2E701F0FCFA22230360C8E701F0AC
:10B95000F7FA21230360E8E74C00002040EF0108DC
:10B9600080EF010810B52DED028B294C8AB0B0EEA6
:10B97000408A00F065FA94F900300133F0EE408A15
:10B980002FD0B0EE480A00F0EBFA50B3B5EEC08A03
:10B99000F1EE10FA25D5012300931E4B18EE100A84
:10B9A00001930023089300F06DFC2478CDE9040195
:10B9B000CDE90201DCB10020002102460B4600F077
:10B9C000DFFD022CCDE9060117D101F0B9FA2123E0
:10B9D0000360089BBBB9DDE9060100F069FF08EED2
:10B9E000900AB0EE680A0AB0BDEC028B10BD0022CE
:10B9F000002343EC172B8DED067B684600F0A6FA7A
:10BA00000028E6D1E1E701F09BFA089B0360E2E73A
:10BA10004C00002044EF01082DE9F04F53EC102BAF
:10BA2000B3F5801F87B0194667DA23F0004313434C
:10BA300000F00B81002951EC100BC0F2948100231F
:10BA40000022C4F2503300F071FC4FF6FF720B4637
:10BA5000C7F6EF72934241EC100B6FF0350753DCE1
:10BA600023F07F4445F6647624F47004C0F209069E
:10BA7000A61906F4801686F07E521D1582F4E002A7
:10BA8000002351EC100BC3F6F07342EA04010022CC
:10BA900000F098FAA5F57E75A31C073D23F470030A
:10BAA000ED190022022B05EB165582468B4636DC3B
:10BAB000002300F0A3FE002800F0D280002D00F04B
:10BAC0005D81284600F0CCFBC9A3D3E900230446DE
:10BAD0000D4600F02BFCC8A3D3E9002306460F4611
:10BAE0002046294600F022FC02460B4630463946E5
:10BAF00000F06AFA41EC100B0EE04FF6FF72C7F649
:10BB0000EF7200279342ABDD51EC100B02460B465F
:10BB100000F05AFA41EC100B07B0BDE8F08F4FF07F
:10BB2000804300F051FA02460B465046594600F059
:10BB300027FDCDE90001284600F092FBCDE9020186
:10BB4000DDE9000102460B4600F0F0FB02460B4621
:10BB50008046894600F0EAFBA9A3D3E90023064604
:10BB60000F4600F0E3FBA8A3D3E9002300F02CFA72
:10BB700032463B4600F0DAFBA5A3D3E9002300F0F0
:10BB800023FA32463B4600F0D1FBA3A3D3E90023BE
:10BB900000F01AFA42464B4600F0C8FBA0A3D3E9D6
:10BBA0000023804689463046394600F0BFFB9EA3FD
:10BBB000D3E9002300F008FA32463B4600F0B6FB1A
:10BBC0009BA3D3E9002300F0FFF932463B4600F087
:10BBD000ADFB02460B464046494600F0F5F94EF6ED
:10BBE00086334BF65102CFF6F973C0F20602E31822
:10BBF000121B1343002B06460F465BDD0023002279
:10BC0000C3F6E0735046594600F090FB52465B463F
:10BC100000F08CFB80468946002D6FD132463B46B2
:10BC200000F0D2F9DDE9002300F080FB02460B466C
:10BC30004046494600F0C6F902460B465046594672
:10BC400000F0C0F941EC100B66E700210020CCF2B7
:10BC500050310022002300F093FC41EC100B5BE715
:10BC600052465B465046594600F060FB72A3D3E94A
:10BC7000002306460F465046594600F057FB0B4638
:10BC800000210246C3F6E071002000F09BF9024655
:10BC90000B463046394600F049FB06460F46002D5C
:10BCA0006FD15046594632463B4600F08BF941EC85
:10BCB000100B31E7002D00F08A804DA3D3E900235B
:10BCC000DDE9020100F032FB32463B468046894600
:10BCD0005046594600F076F9DDE9002300F026FBD6
:10BCE00045A3D3E9002304460D46DDE9020100F037
:10BCF0001DFB02460B462046294659E03CA3D3E9EA
:10BD00000023DDE9020100F011FB3246CDE9040118
:10BD10003B464046494600F057F9DDE9002300F074
:10BD200005FB35A3D3E9002304460D46DDE90201F6
:10BD300000F0FCFA02460B462046294600F044F982
:10BD400002460B464046494600F03CF952465B46E7
:10BD500000F038F902460B46DDE9040100F032F943
:10BD600041EC100BD8E602460B4600F02BF90022FE
:10BD7000002300F005FC41EC100BCDE69FED1A0B03
:10BD8000CAE6284600F06CFA19A3D3E9002304465A
:10BD90000D4600F0CBFA18A3D3E90023804689466C
:10BDA0002046294600F0C2FA02460B463046394684
:10BDB00000F008F952465B4600F004F902460B46D3
:10BDC0004046494600F0FEF841EC100BA4E632462E
:10BDD0003B465046594600F0F5F8DDE9002300F0F7
:10BDE000A5FA29E7AFF30080000000000000000082
:10BDF0000000E0FE422EE63F763C7935EF39EA3D21
:10BE000044523EDF12F1C23FDE03CB966446C73F89
:10BE1000599322942449D23F935555555555E53FA2
:10BE20009FC678D0099AC33FAF788E1DC571CC3FAD
:10BE300004FA97999999D93F555555555555D53F78
:10BE400010EE103A23F00042B2F1FF4F70B42FD23F
:10BE500062B3002B3ADBD915B2F5000F2BD323F0D8
:10BE60007F43A1F17F0223F40003D10743F40003D1
:10BE700048BF5B00002556105B0019212C464FF08F
:10BE80008072A018984202DC84181B1AAD185B005F
:10BE900052080139F5D113B105F001035D196D1098
:10BEA00005F17C5505EBC65500EE105A70BC704785
:10BEB00000EE000AFAE713F400020CD15B00013235
:10BEC0001802FBD5C2F101028918C8E730EE400A1A
:10BED00080EE000AEAE701228918C0E753EC102B34
:10BEE00010461A4663B1B3F1004F09D04FF6FF7305
:10BEF000A2F58011C7F6DF73994205D80420704778
:10BF00000028F3D10220704702F1FE4101F57001D3
:10BF10009942F3D94FF6FF73C0F20F039A4201D84A
:10BF20000320704702F100419942F9D90023C7F676
:10BF3000F0739A4204D012F5801F01D000207047A0
:10BF4000D0F1010038BF0020704700BF00207047CB
:10BF50009FED010B704700BF000000000000F87F5C
:10BF600010EE103A0BB902207047B3F1004FFAD02F
:10BF7000A3F500016FF00142914201D804207047FF
:10BF800003F1FF419142F9D94FF6FE72591EC0F2FA
:10BF90007F02914201D80320704703F1004101392B
:10BFA0009142F8D9B3F1FF4F05D013F5000F14BF3C
:10BFB0000020012070470120704700BF81F0004140
:10BFC00002E000BF83F0004330B54FEA41044FEA7E
:10BFD000430594EA050F08BF90EA020F1FBF54EA19
:10BFE000000C55EA020C7FEA645C7FEA655C00F0B5
:10BFF000E2804FEA5454D4EB5555B8BF6D420CDD86
:10C000002C4480EA020281EA030382EA000083EA08
:10C01000010180EA020281EA0303362D88BF30BDA8
:10C0200011F0004F4FEA01314FF4801C4CEA1131FE
:10C0300002D0404261EB410113F0004F4FEA03335D
:10C040004CEA133302D0524263EB430394EA050FE8
:10C0500000F0A780A4F10104D5F1200E0DDB02FA57
:10C060000EFC22FA05F2801841F1000103FA0EF2EB
:10C07000801843FA05F359410EE0A5F120050EF1B1
:10C08000200E012A03FA0EFC28BF4CF0020C43FAE2
:10C0900005F3C01851EBE37101F0004507D54FF0EF
:10C0A000000EDCF1000C7EEB00006EEB0101B1F53F
:10C0B000801F1BD3B1F5001F0CD349085FEA300085
:10C0C0004FEA3C0C04F101044FEA445212F5800F90
:10C0D00080F09A80BCF1004F08BF5FEA500C50F12D
:10C0E000000041EB045141EA050130BD5FEA4C0C10
:10C0F000404141EB010111F4801FA4F10104E9D199
:10C1000091F0000F04BF01460020B1FA81F308BF8F
:10C110002033A3F10B03B3F120020CDA0C3208DD5B
:10C1200002F1140CC2F10C0201FA0CF021FA02F136
:10C130000CE002F11402D8BFC2F1200C01FA02F1A6
:10C1400020FA0CFCDCBF41EA0C019040E41AA2BFCB
:10C1500001EB0451294330BD6FEA04041F3C1CDA93
:10C160000C340EDC04F11404C4F1200220FA04F0B3
:10C1700001FA02F340EA030021FA04F345EA03015D
:10C1800030BDC4F10C04C4F1200220FA02F001FA1F
:10C1900004F340EA0300294630BD21FA04F02946A1
:10C1A00030BD94F0000F83F4801306BF81F480113A
:10C1B0000134013D4EE77FEA645C18BF7FEA655CAD
:10C1C00029D094EA050F08BF90EA020F05D054EA7F
:10C1D000000C04BF1946104630BD91EA030F1EBF84
:10C1E0000021002030BD5FEA545C05D14000494188
:10C1F00028BF41F0004130BD14F580043CBF01F57B
:10C20000801130BD01F0004545F0FE4141F4700160
:10C210004FF0000030BD7FEA645C1ABF194610463B
:10C220007FEA655C1CBF0B46024650EA013406BF3C
:10C2300052EA033591EA030F41F4002130BD00BFFB
:10C2400090F0000F04BF0021704730B54FF48064B8
:10C2500004F132044FF000054FF0000150E700BF39
:10C2600090F0000F04BF0021704730B54FF4806498
:10C2700004F1320410F0004548BF40424FF0000185
:10C280003EE700BF42004FEAE2014FEA31014FEAC8
:10C2900002701FBF12F07F4393F07F4F81F0605117
:10C2A000704792F0000F14BF93F07F4F704730B586
:10C2B0004FF4607401F0004521F0004120E700BF19
:10C2C00050EA010208BF704730B54FF000050AE0A0
:10C2D00050EA010208BF704730B511F0004502D5A1
:10C2E000404261EB41014FF4806404F132045FEAA3
:10C2F000915C3FF4DCAE4FF003025FEADC0C18BF48
:10C3000003325FEADC0C18BF033202EBDC02C2F13D
:10C31000200300FA03FC20FA02F001FA03FE40EACF
:10C320000E0021FA02F11444C1E600BF70B54FF0CF
:10C33000FF0C4CF4E06C1CEA11541DBF1CEA1355B1
:10C3400094EA0C0F95EA0C0F00F0DEF82C4481EA19
:10C35000030621EA4C5123EA4C5350EA013518BF39
:10C3600052EA033541F4801143F4801338D0A0FB26
:10C3700002CE4FF00005E1FB02E506F00042E0FBD3
:10C3800003E54FF00006E1FB03569CF0000F18BFD9
:10C390004EF0010EA4F1FF04B6F5007F64F5407481
:10C3A00004D25FEA4E0E6D4146EB060642EAC62114
:10C3B00041EA55514FEAC52040EA5E504FEACE2E81
:10C3C000B4F1FD0C88BFBCF5E06F1ED8BEF1004F84
:10C3D00008BF5FEA500E50F1000041EB045170BD00
:10C3E00006F0004646EA010140EA020081EA030144
:10C3F000B4EB5C04C2BFD4EB0C0541EA045170BD40
:10C4000041F480114FF0000E013C00F3AB8014F1B9
:10C41000360FDEBF002001F0004170BDC4F1000402
:10C42000203C35DA0C341BDC04F11404C4F1200583
:10C4300000FA05F320FA04F001FA05F240EA0200DE
:10C4400001F0004221F0004110EBD37021FA04F614
:10C4500042EB06015EEA430E08BF20EAD37070BDCE
:10C46000C4F10C04C4F1200500FA04F320FA05F02D
:10C4700001FA04F240EA020001F0004110EBD3702F
:10C4800041F100015EEA430E08BF20EAD37070BD9F
:10C49000C4F1200500FA05F24EEA020E20FA04F378
:10C4A00001FA05F243EA020321FA04F001F0004127
:10C4B00021FA04F220EA020000EBD3705EEA430E98
:10C4C00008BF20EAD37070BD94F0000F0FD101F0C7
:10C4D0000046400041EB010111F4801F08BF013C00
:10C4E000F7D041EA060195F0000F18BF704703F03E
:10C4F0000046520043EB030313F4801F08BF013DC5
:10C50000F7D043EA0603704794EA0C0F0CEA135580
:10C5100018BF95EA0C0F0CD050EA410618BF52EA3A
:10C520004306D1D181EA030101F000414FF0000040
:10C5300070BD50EA410606BF1046194652EA43064E
:10C5400019D094EA0C0F02D150EA013613D195EAC2
:10C550000C0F05D152EA03361CBF104619460AD10A
:10C5600081EA030101F0004141F0FE4141F4700114
:10C570004FF0000070BD41F0FE4141F4780170BD04
:10C5800070B54FF0FF0C4CF4E06C1CEA11541DBF69
:10C590001CEA135594EA0C0F95EA0C0F00F0A7F86B
:10C5A000A4EB050481EA030E52EA03354FEA013198
:10C5B00000F088804FEA03334FF0805545EA1313AB
:10C5C00043EA12634FEA022245EA111545EA106573
:10C5D0004FEA00260EF000419D4208BF964244F10A
:10C5E000FD0404F5407402D25B084FEA3202B61A29
:10C5F00065EB03055B084FEA32024FF480104FF4FD
:10C60000002CB6EB020E75EB030E22BFB61A754670
:10C6100040EA0C005B084FEA3202B6EB020E75EB03
:10C62000030E22BFB61A754640EA5C005B084FEA6B
:10C630003202B6EB020E75EB030E22BFB61A754638
:10C6400040EA9C005B084FEA3202B6EB020E75EB43
:10C65000030E22BFB61A754640EADC0055EA060E04
:10C6600018D04FEA051545EA16754FEA06164FEA47
:10C67000C30343EA52734FEAC2025FEA1C1CC0D1F3
:10C6800011F4801F0BD141EA00014FF000004FF080
:10C69000004CB6E711F4801F04BF01430020B4F141
:10C6A000FD0C88BFBCF5E06F3FF6AFAEB5EB030CF9
:10C6B00004BFB6EB020C5FEA500C50F1000041EBF6
:10C6C000045170BD0EF0004E4EEA113114EB5C04C3
:10C6D000C2BFD4EB0C0541EA045170BD41F4801196
:10C6E0004FF0000E013C90E645EA060E8DE60CEA9E
:10C6F000135594EA0C0F08BF95EA0C0F3FF43BAFBB
:10C7000094EA0C0F0AD150EA01347FF434AF95EA71
:10C710000C0F7FF425AF104619462CE795EA0C0F55
:10C7200006D152EA03353FF4FDAE1046194622E722
:10C7300050EA410618BF52EA43067FF4C5AE50EAFC
:10C7400041047FF40DAF52EA43057FF4EBAE12E7EC
:10C750004FF0FF3C06E000BF4FF0010C02E000BFCD
:10C760004FF0010C4DF804CD4FEA410C7FEA6C5CB0
:10C770004FEA430C18BF7FEA6C5C1BD001B050EA53
:10C78000410C0CBF52EA430C91EA030F02BF90EA3E
:10C79000020F0020704710F1000F91EA030F58BFFD
:10C7A000994208BF90422CBFD8176FEAE37040F05F
:10C7B000010070474FEA410C7FEA6C5C02D150EAFD
:10C7C000013C07D14FEA430C7FEA6C5CD6D152EAB8
:10C7D000033CD3D05DF8040B704700BF844610467D
:10C7E00062468C461946634600E000BF01B5FFF77C
:10C7F000B7FF002848BF10F1000F01BD4DF808ED4C
:10C80000FFF7F4FF0CBF012000205DF808FB00BF1C
:10C810004DF808EDFFF7EAFF34BF012000205DF876
:10C8200008FB00BF4DF808EDFFF7E0FF94BF0120C3
:10C8300000205DF808FB00BF4DF808EDFFF7CEFFC4
:10C8400094BF012000205DF808FB00BF4DF808ED03
:10C85000FFF7C4FF34BF012000205DF808FB00BFD4
:10C860004FEA410212F5001215D211D56FF4787318
:10C87000B3EB625212D94FEAC12343F0004343EABB
:10C88000505311F0004F23FA02F018BF4042704796
:10C890004FF00000704750EA013005D111F0004020
:10C8A00008BF6FF0004070474FF00000704700BFB6
:10C8B0004FEA4102B2F1E04324BFB3F5001CDCF1C2
:10C8C000FE5C0DD901F0004C4FEAC0024CEA5070FA
:10C8D000B2F1004F40EB830008BF20F00100704729
:10C8E00011F0804F21D113F13872BCBF01F000402C
:10C8F000704741F480114FEA5252C2F11802C2F15E
:10C90000200C10FA0CF320FA02F018BF40F00100DE
:10C910004FEAC1234FEAD32303FA0CFC40EA0C0090
:10C9200023FA02F34FEA4303CCE77FEA625307D1CD
:10C9300050EA01331EBF4FF0FE4040F44000704704
:10C9400001F0004040F0FE4040F40000704700BF9E
:10C9500073B96AB9002908BF0028BCBF00204FF096
:10C960000041C4BF6FF000414FF0FF3000F038B815
:10C9700082B0EC462DE9005000F006F8DDF804E046
:10C9800002B00CBC704700BFF8B5144606460F460F
:10C990001D4600F027F804FB01F300FB0535A4FB5E
:10C9A0000023EB18069CB21A67EB0303C4E90023CB
:10C9B000F8BD00BFF8B5144606460F461D4600F008
:10C9C00075F900FB05F5A0FB042304FB0155EB18EA
:10C9D000069CB21A67EB0303C4E90023F8BD00BF4D
:10C9E000704700BF00292DE9F0071D46C0F29E8068
:10C9F0000024002DC0F2958007460D4616469C4641
:10CA0000002B3ED18A4254D9B2FA82F343B1C3F12A
:10CA1000200620FA06F501FA03F19A4029439840CE
:10CA2000160CB1FBF6F597B206FB15114FEA104C48
:10CA300007FB05F34CEA01418B4209D9891805F13E
:10CA4000FF3C80F015818B4240F21281023D891833
:10CA5000C3EB010CBCFBF6F306FB13C180B207FB72
:10CA600003F740EA0140874207D9591E821880F037
:10CA70000581974240F20281023B43EA05420023CE
:10CA800003E08B420AD900231A461046194614B116
:10CA9000404261EB4101BDE8F0077047B3FA83F310
:10CAA000002B40F087808C4501D38242ECD80122D4
:10CAB000EBE712B90123B3FBF2F2B2FA82F6002ED1
:10CAC0003AD1891A150C1FFA82FC0123B1FBF5F744
:10CAD00005FB17114FEA10480CFB07F648EA014125
:10CAE0008E4207D9891807F1FF3802D28E4200F230
:10CAF000DA804746891BB1FBF5F605FB161180B2BB
:10CB00000CFB06FC40EA0140844507D9711E8218DF
:10CB100080F0B080944540F2AD80023E46EA074284
:10CB2000B3E7E443524263EB430365E7404261EB02
:10CB300041014FF0FF345CE7B240C6F1200521FA15
:10CB400005F320FA05F701FA06F9150CB3FBF5F821
:10CB500047EA09091FFA82FC05FB18374FEA194119
:10CB60000CFB08F341EA0747B040BB420AD9BF18A3
:10CB700008F1FF3180F09580BB4240F29280A8F12D
:10CB80000208BF18FE1AB6FBF5F305FB13611FFA86
:10CB900089F90CFB03F649EA01418E4206D95F1E72
:10CBA000891878D28E4276D9023B8918891B43EACC
:10CBB00008438BE7C3F1200726FA07F80CFA03F2C3
:10CBC00048EA020C21FA07F105FA03FA4FEA1C4978
:10CBD00020FA07F5B1FBF9F845EA0A0509FB181731
:10CBE0002A0C1FFA8CFA0AFB08F142EA0747B942FD
:10CBF00006FA03F609D917EB0C0708F1FF324ED2FB
:10CC0000B9424CD9A8F1020867447F1AB7FBF9F280
:10CC100009FB1271ADB20AFB02FA45EA01418A45ED
:10CC200007D9551E11EB0C0137D28A4535D9023A86
:10CC3000614442EA08424FEA124C1FFA86F808FBA8
:10CC40000CF7360C95B208FB05F806FB057505EBED
:10CC5000184506FB0CFCAF4288BF0CF5803CCAEBC4
:10CC600001010CEB1546B14212D309D000230CE7A9
:10CC70006546EDE60E4646EA074206E70B46FCE649
:10CC80001FFA88F800FA03F308EB0545AB42EDD232
:10CC9000013A0023F9E63B4688E72A46C9E7904671
:10CCA000B3E788466EE7023F891823E72DE9F00FC6
:10CCB000144605460E46002B3FD18A424AD9B2FAA5
:10CCC00082F343B1C3F1200025FA00F201FA03F622
:10CCD0009C4016439D40210CB6FBF1F22F0CA0B2F4
:10CCE00001FB126C00FB02F347EA0C46B34208D981
:10CCF000571E361980F0FF80B34240F2FC80023AA2
:10CD00003619F61AB6FBF1F301FB1361ADB200FB65
:10CD100003F045EA0141884207D95E1E091980F0F7
:10CD2000EC80884240F2E980023B43EA0242002361
:10CD300010461946BDE8F00F70478B4243D8B3FA4E
:10CD400083F4002C42D18B42234601D382423BD84C
:10CD50000122EDE712B90123B3FBF2F4B4FA84F235
:10CD6000002A40F08A80091B260CA7B20123B1FBE0
:10CD7000F6F006FB10114FEA154C07FB00F24CEAE7
:10CD800001418A4207D9091900F1FF3C02D28A42C7
:10CD900000F2D3806046C2EB010CBCFBF6F206FB4E
:10CDA00012C1ADB207FB02F745EA0145AF4207D910
:10CDB000511E2C1980F0A380A74240F2A080023AB5
:10CDC00042EA0042B4E700231A46B1E7C4F1200763
:10CDD00022FA07F603FA04F3334321FA07FA4FEA7B
:10CDE000134C01FA04FB20FA07F141EA0B0BBAFBE2
:10CDF000FCF70CFB17A61FFA83F84FEA1B4508FB4C
:10CE000007F945EA0645A94502FA04FA04D97A1E4B
:10CE1000ED18C0F088801746C9EB0505B5FBFCF698
:10CE20000CFB16521FFA8BFB08FB06F84BEA02417B
:10CE3000884503D9721EC91870D3164646EA0742C0
:10CE4000170C1FFA8AFC0CFB07F695B24FEA1A433F
:10CE50000CFB05FC03FB056505EB1C4503FB07F319
:10CE6000AE4288BF03F58033C8EB010103EB1543E5
:10CE7000994250D347D000235AE79440C2F120088A
:10CE8000260C20FA08F721FA08F501FA02F9B5FB99
:10CE9000F6F847EA090906FB1855A7B24FEA194CFC
:10CEA0004CEA054C07FB08F3634500FA02F509D983
:10CEB0001CEB040C08F1FF323DD263453BD9A8F1CD
:10CEC0000208A444C3EB0C02B2FBF6F306FB1320EA
:10CED0001FFA89F907FB03F249EA00418A4206D9A1
:10CEE000581E091925D28A4223D9023B0919891AE9
:10CEF00043EA08433BE73A4603E7334615E70A4669
:10CF000042EA004214E71FFA8CF100FA04F001EB48
:10CF10000545A842AFD2013A002309E788458CD9DC
:10CF2000023EC9188AE7A9457FF675AF023FED18A2
:10CF300072E70346DBE79046C4E7023809192AE79F
:10CF400040F27843C2F20003186870470EB470B51F
:10CF500040F278419DB0C2F2000121AB096853F85C
:10CF6000042B6FF0004405460394069408464FF4E2
:10CF7000027601A94FF6FF741B93ADF8106001957E
:10CF80000595ADF8124000F067F8019B00221A7079
:10CF90001DB0BDE8704003B0704700BF80EA0102D9
:10CFA000844612F0030F4FD111F0030F32D14DF828
:10CFB000044D11F0040F51F8043B0BD0A3F10132E2
:10CFC0009A4312F0803F04BF4CF8043B51F8043BF5
:10CFD00016D100BF51F8044BA3F101329A4312F06D
:10CFE000803FA4F101320BD14CF8043BA24312F074
:10CFF000803F04BF51F8043B4CF8044BEAD0234671
:10D000000CF8013B13F0FF0F4FEA3323F8D15DF822
:10D01000044B704711F0010F06D011F8012B0CF8EA
:10D02000012B002A08BF704711F0020FBFD031F862
:10D03000022B12F0FF0F16BF2CF8022B8CF80020E9
:10D0400012F47F4FB3D1704711F8012B0CF8012B6C
:10D05000002AF9D1704700BF2DE9F04FBFB09346C9
:10D0600005910B93089002F0E7F900680023002275
:10D07000CDE91423109003F023F8129005988389CA
:10D080001B0603D50369002B01F03F8046F2676160
:10D09000002319AAC6F266610A933392359334933A
:10D0A000169317930793164613919BF80030002BA5
:10D0B00000F0BC80252B00F0B9805A465F4601E0A5
:10D0C000252B04D012F8013F0137002BF8D1CBEB10
:10D0D00007037BB1349C359DC6F800B00134ED18D0
:10D0E000072C73603595349400F3828008360798D6
:10D0F000C01807903B78002B00F0848000210022AC
:10D1000007F1010B7B7806918DF8F7204FF0FF3780
:10D11000039120242B200BF1010BA3F12002582AAC
:10D1200000F21782DFE812F0C10215021502AE020A
:10D13000150215021502150215021502B50284002A
:10D1400015025D0089001502A300AA00AA00AA002A
:10D15000AA00AA00AA00AA00AA00AA0015021502A5
:10D160001502150215021502150215021502150207
:10D17000BB004901150249011502150215021502ED
:10D180008401150215028B01150215021502150204
:10D190001502A30115021502B701150215021502A9
:10D1A00015021502150215021502150215024F028D
:10D1B00027024901490149014802270215021502C7
:10D1C0000A0215028A0260027302DA011502E10105
:10D1D0001502980215021502D602069B0B915B42BE
:10D1E0000693039941F0040103919BF8003092E704
:10D1F00008980599029333AA02F092FF029B40B966
:10D2000019AE74E7359B23B10898059933AA02F04B
:10D2100087FF0599079A8B8913F0400F18BF4FF0CD
:10D22000FF32079207983FB0BDE8F08F5F4661E795
:10D230008DF8F7009BF800306DE75A4612F8013B75
:10D240002A2B01F0FB80A3F13001092901F2AA8009
:10D25000002712F8013B07EB870701EB4707A3F113
:10D26000300109299346F4D947EAE77755E703994E
:10D2700041F0800103919BF800304CE759460022B1
:10D28000A3F1300C11F8013BA3F1300502EB82024F
:10D29000092D0CEB42028B46F2D906923DE70F9323
:10D2A000039B43F0100303930398850640F16881C4
:10D2B0000B99CB1D23F00703D3E9000108330B932F
:10D2C000002871F1000380468946C0F26C81012379
:10D2D000002F03DB039921F08001039158EA090232
:10D2E00040F0E882002F40F0E582002B40F03784C8
:10D2F000039AD10740F1338430238DF8CB300123DA
:10D3000009930DF1CB0A09989DF8F7300C97B842B4
:10D31000B8BF384600210490119113B10498013030
:10D320000490039B13F002030D9302D00498023083
:10D330000490039B13F084030E9340F0E28106985F
:10D340000499471A002F40F3DC81102F359D349C3F
:10D35000DFF87C8325DD23462A4644464FF010093A
:10D36000059DDDF8208003E0103F0836102F15DD05
:10D3700001331032072B86E8100235923493F3DD27
:10D380004046294633AA02F0CBFE00287FF441AF85
:10D39000103F102F359A349B19AEE9DCA046154694
:10D3A0001C460134ED19072CC6F8008077603595CE
:10D3B000349400F354840836A4E103980F930207D1
:10D3C00040F185850B99CB1D23F0070303F108027B
:10D3D0000B92D3F800805D6842462B46CDE91423BA
:10D3E00042462B4643EC102BFEF778FD012840F017
:10D3F00040854046294600220023FFF709FA00280D
:10D4000040F07E869DF8F73003200021AC4A04905E
:10D410000C910F98AB494728CCBF8A469246039996
:10D42000032221F08001002003910992119074E7FA
:10D43000039A42F0080203929BF800306BE60399CE
:10D440000F9341F010010391039A12F0200300F0B2
:10D45000D1800B98C31D23F0070303F10801D3E922
:10D4600000890B91002300208DF8F70030E7039A24
:10D470000F9342F010020392039B9B0640F1F18050
:10D480000B98C31D23F0070303F10801D3E90089BA
:10D490000B910123E7E70F93039B8B4A99061692A2
:10D4A00040F11F810B98C31D23F00703D3E90089C6
:10D4B00003F108010B910399CD0740F1818358EAEC
:10D4C000090200F07D8330238DF8F4300F9B41F08A
:10D4D00002018DF8F53003910223C4E7039B43F06A
:10D4E000200303939BF8003015E60B9A0F9300215D
:10D4F0008DF8F710D2F800A0141DBAF1000F00F05B
:10D500008E86002F5046C0F2398600213A4602F03E
:10D5100039FA002800F02987CAEB00000023B8423E
:10D5200009900C9340F3648527EAE770002104908A
:10D530009DF8F7300B9409971191EEE69BF80030B7
:10D540006C2B5A4600F04B85039A42F0100203926E
:10D55000E1E50F93002B3FF455AE01228DF8A43086
:10D56000002304928DF8F73009920DF1A40A0023EC
:10D570000C931193D5E603980F9385063FF598AE6B
:10D58000039AD00640F1AC840B98036898460B9A36
:10D590004FEAE879404649460432002871F1000319
:10D5A0000B92BFF694AE2D238DF8F730D8F100081A
:10D5B00069EB490901238BE6039B43F04003039386
:10D5C0009BF80030A7E50F930B9B0B9A1B6801207B
:10D5D0000021043204908DF8F7100B928DF8A430DE
:10D5E00009900DF1A40AC2E7039A0F9312F02003E9
:10D5F0007FF42FAF039810F0100200F059840B99BC
:10D600000A68043190464FF000090B912BE70B9B01
:10D610000B991B682D489846039B169043F0020314
:10D6200078220431039330238DF8F4308DF8F520FF
:10D630000B914FF0000902230F9214E70398800624
:10D6400040F157840B99079A0B68D1171A600B9A0F
:10D65000596004320B9228E50F93039B9B063FF51C
:10D660000FAF039AD50600F14F830399480640F1A6
:10D670004B830B9AB2F80080043201234FF000096B
:10D680000B92F0E6039A42F0010203929BF80030FD
:10D6900041E50B9B0B9A1B68111D002B0693FFF6AF
:10D6A0009CAD9BF800300B9135E59DF8F730002BD1
:10D6B00040F02B848DF8F7409BF800302BE500BF3D
:10D6C00060EF010864EF010870EF010884EF0108C2
:10D6D000A4EF01088D490F93039B169199063FF51E
:10D6E000E1AE039AD20600F1198303994B0640F18B
:10D6F00015830B9AB2F8008004320B924FF00009A8
:10D70000D9E6359D9DF8F7306BB1349C0DF1F703E8
:10D710000134336001350123072C7360359534944F
:10D7200000F3078208360D9B63B1349C3DAB013496
:10D73000336002350223072C73603595349400F36F
:10D74000038208360E9B802B00F041810C9B0998C8
:10D750001F1A002F35DD102F349CDFF8B48125DD32
:10D7600023462A4644464FF01009059DDDF82080E7
:10D7700003E0103F0836102F15DD01331032072B60
:10D7800086E8100235923493F3DD4046294633AAE9
:10D7900002F0C6FC00287FF43CAD103F102F359AF4
:10D7A000349B19AEE9DCA04615461C460134ED1940
:10D7B000072CC6F8008077603595349400F3AE816D
:10D7C00008360399CA0500F1A780349C099BC6F866
:10D7D00000A00134ED18072C7360359534945EDC9D
:10D7E0000836039A530740D5069B04981F1A002F4A
:10D7F0003BDD102F349CDFF81C8124DD23464FF0E5
:10D8000010094446DDF814A0DDF8208003E0103F45
:10D810000836102F15DD01331035072B86E810026E
:10D8200035953493F3DD4046514633AA02F078FC37
:10D8300000287FF4EEAC103F102F359D349B19AEBD
:10D84000E9DCA0461C4601347D19072CC6F800808F
:10D8500077603595349408DD0898059933AA02F06D
:10D860005FFC00287FF4D5AC359D0799049A069B90
:10D870009A42ACBF8918C9180791002D40F0448125
:10D880000020349019AE10E4A0461C460134ED1976
:10D89000072CC6F80080776035953494A0DD089891
:10D8A000059933AA02F03CFC00287FF4B2AC19AE13
:10D8B000359D96E7012B00F07381022B00F0548117
:10D8C00033AC224600E052464FEAD80343EA49739C
:10D8D0004FEAD90108F007008946984600F1300365
:10D8E00058EA090002F8013C02F1FF3AEBD1039932
:10D8F000C80706D5302B04D03023A2F1020A02F863
:10D90000023CCAEB04040994FDE400BF84EF010863
:10D9100050EF0108A4EF01080F98652840F39480A8
:10D92000DDE9140100220023FEF768FF002800F063
:10D930004D81349CA34B0134336001350123072C06
:10D9400073603595349400F3F38208363A9B0A9954
:10D950008B4203DB039AD3077FF543AF349C1298C5
:10D96000109B706001342D18072C3360359534946A
:10D9700000F3498308360A994F1E002F7FF731AF15
:10D98000102F349CDFF8408280DD23464FF01009D1
:10D990004446DDF814A0DDF8208004E00836103F8E
:10D9A000102F7FF771AF01331035072B86E8100277
:10D9B00035953493F2DD4046514633AA02F0B0FB70
:10D9C00000287FF426AC359D349B19AEE7E7069816
:10D9D0000499471A002F7FF7B9AE102F349CDFF857
:10D9E000E88125DD23462A4644464FF01009059D6F
:10D9F000DDF8208003E0103F0836102F15DD0133DD
:10DA00001032072B86E8100235923493F3DD40463E
:10DA1000294633AA02F084FB00287FF4FAAB103FBA
:10DA2000102F359A349B19AEE9DCA04615461C46EA
:10DA30000134ED19072CC6F80080776035953494D1
:10DA400000F30C82083681E60A9A349C012A40F3DE
:10DA5000D281013401350123072CC6F800A0736080
:10DA60003595349400F3E28108361298109970606D
:10DA700001342D18072C31603595349400F3E28180
:10DA80000836DDE9140100220023FEF7B7FE002866
:10DA900040F0F0800A9B01345A1EAD180AF10103D0
:10DAA000072C336072603595349421DC0836179961
:10DAB00001346D1836AB072C3360716035953494A2
:10DAC0007FF78EAE0898059933AA02F029FB00284B
:10DAD0007FF49FAB359D19AE83E6A0461C4601340A
:10DAE000ED19072CC6F80080776035953494DDDD9C
:10DAF0000898059933AA02F013FB00287FF489AB3C
:10DB000019AE359D349CD2E70898059933AA02F0E6
:10DB100007FB00283FF4B4AEFFF77BBB08980599DC
:10DB200033AA02F0FDFA00287FF473AB359D19AEDD
:10DB300047E60898059933AA02F0F2FA00287FF424
:10DB400068AB359D19AEEEE50898059933AA02F049
:10DB5000E7FA00287FF45DAB359D19AEF2E5099731
:10DB60000DF1CC0AFFF7CFBB169C0DF1CB0208F0EC
:10DB70000F004FEA181343EA09734FEA191192464E
:10DB80009846225C894658EA09018AF800200AF181
:10DB9000FF32ECD133ABCAEB03030993FFF7B3BBFE
:10DBA000B8F10A0F79F1000280F0908008F1300896
:10DBB00001238DF8CB8009930DF1CB0AFFF7A3BBAE
:10DBC000022350E4A0EF010850EF01083A9F002F14
:10DBD00040F3B981119B0A9F9F42A8BF1F460A9B31
:10DBE000002F534409930BDD349CC6F800A0013488
:10DBF000ED19072C77603595349400F3DD820836F3
:10DC0000119827EAE777C71B002F40F39A80102F5F
:10DC1000349CDFF8208540F37F8123462A46444622
:10DC20004FF01009059DDDF8208004E00836103F14
:10DC3000102F40F36E8101331032072B86E810025B
:10DC400035923493F2DD4046294633AA02F068FA51
:10DC500000287FF4DEAA359A349B19AEE7E70898CE
:10DC6000059933AA02F05CFA00287FF4D2AA359D08
:10DC700019AE47E50A98471E002F7FF718AF102FFF
:10DC8000DFF8B0847FF72BAF23464FF010094446EE
:10DC9000DDF814A0DDF8208004E00836103F102FD6
:10DCA0007FF71BAF01331035072B86E8100235953F
:10DCB0003493F2DD4046514633AA02F031FA00288F
:10DCC0007FF4A7AA359D349B19AEE7E70DF1CB048D
:10DCD000404649460A22002302F078FE3032227084
:10DCE000404649460A22002302F070FE80468946DB
:10DCF00058EA0900A24604F1FF34E9D133ABCAEB7C
:10DD000003030993FFF7FFBA0B98036804309846A2
:10DD10004FF000090B900123FFF7A5BB0B98036898
:10DD2000043098464FF000090B90FFF7C4BB0898E9
:10DD3000059933AA02F0F4F900287FF46AAA359D08
:10DD400019AE3A9B0A998B4247DB039AD10744D418
:10DD5000119809990AEB00020A988F1AC31ABB425C
:10DD6000B8BF1F46002F0ADD349C32600134ED1924
:10DD7000072C77603595349400F34382083627EA00
:10DD8000E777DF1B002F7FF72CAD102F349CDFF8D7
:10DD9000A4837FF77BAD23464FF010094446DDF89E
:10DDA00014A0DDF8208004E00836103F102F7FF724
:10DDB0006BAD01331035072B86E81002359534938F
:10DDC000F2DD4046514633AA02F0AAF900287FF45A
:10DDD00020AA359D349B19AEE7E7349C1299109820
:10DDE000716001346D18072C30603595349400F360
:10DDF000EE810836ACE7039BDA073FF52AAE013423
:10DE000001350123072CC6F800A0736035953494C2
:10DE10007FF74CAE0898059933AA02F081F90028E3
:10DE20007FF4F7A9359D349C19AE40E60898059912
:10DE300033AA02F075F900287FF4EBA9359D349CD4
:10DE400019AE12E60898059933AA02F069F900287C
:10DE50007FF4DFA9359D349C19AE12E60898059928
:10DE600033AA02F05DF900287FF4D3A9359D19AEDD
:10DE70006CE442462B4643EC102BFEF72FF80028AB
:10DE800040F0CC8003210C90A74A0F980491A74939
:10DE90009DF8F7304728CCBF8A46924603990C98E4
:10DEA00021F080010322039109921190FFF735BA06
:10DEB000039810F0400300F058810B99B1F80080EE
:10DEC000043113464FF000090B91FFF7CCBA0B98C1
:10DED000C31D23F0070303F108010B91FFF779BA83
:10DEE000039B0B9859067FF550ABB0F90080FFF704
:10DEF0004EBB039BD90640F12D810B98079903680F
:10DF000004300B901960FFF7D0B89BF80030FFF792
:10DF100002B9A04615461C460134ED19072CC6F877
:10DF200000807760359534943FF701AF083608E7F5
:10DF30000898059933AA02F0F3F800287FF469A93C
:10DF4000359D19AE02E5349C794B013433600135BF
:10DF50000123072C73603595349400F3ED80083667
:10DF60002FB90A9A1AB9039BD8077FF53AAC349CAB
:10DF700012991098716001346D18072C3060359536
:10DF8000349400F3FE8108367F42002F40F307816E
:10DF9000102FDFF8A08140F3298123462A4644460A
:10DFA0004FF01009089DDDF8148004E00836103F9A
:10DFB000102F40F3188101331032072B86E810022E
:10DFC00035923493F2DD2846414633AA02F0A8F890
:10DFD00000287FF41EA9359A349B19AEE7E7039910
:10DFE000537841F020010BF1010B0391FFF793B837
:10DFF000099820EAE070002104909DF8F7300B9416
:10E000001191FFF78AB90898059933AA02F088F8A8
:10E0100000287FF4FEA8359D19AEACE47B1C00F00F
:10E0200097800F99672900F0B981472900F0B681E0
:10E03000039A002D42F480720392C0F2BA8100204C
:10E040000C900F99662900F05281462900F04F810B
:10E05000652900F0AB81452900F0A881B946424608
:10E060002B463BAC43EC102B02214A460094089807
:10E070003AAB3CAC019400F0ABFA0F9A672A8246A7
:10E0800001D0472A03D1039BDC0740F1AD810F98F3
:10E0900046280AEB090400F03B814046294600224D
:10E0A0000023FEF7ABFB002800F046813C940F995B
:10E0B000CAEB040467290A9400F0C980472900F0DC
:10E0C000C6800F9B3A99662B40F0C980002940F327
:10E0D000AB81002F40F0A181039AD20700F19D810E
:10E0E00021EAE1730493099111910C99002900F040
:10E0F000A2802D238DF8F73000230C93FFF70EB983
:10E100002D238DF8F730FFF77FB94021089801F0F3
:10E1100099F9059908600861002800F0A181059827
:10E1200040234361FEF7B2BF68EF01086CEF0108BE
:10E13000A0EF010850EF01080898059933AA01F0F3
:10E14000EFFF00287FF465A83A9F359D19AE07E7D9
:10E1500006276DE7039A520671D50B980799036855
:10E1600004300B901980FEF7A0BF0B9802680430B2
:10E1700090464FF000090B90FFF775B901F0A0FF32
:10E18000002309900C9334E70898059933AA01F00D
:10E19000C7FF00287FF43DA8359D349C19AE0A9A2C
:10E1A000C6F800A00134AD18072C72603595349480
:10E1B0007FF716ABFFF773BB0898059933AA01F0F8
:10E1C000AFFF00287FF425A8359D19AE18E5089803
:10E1D000059933AA01F0A4FF00287FF41AA83A9BFE
:10E1E000359D19AEB4E5A04615461C460134ED191F
:10E1F000072CC6F80080776035953494C4DC083667
:10E20000CDE70898059933AA01F08AFF00287FF42A
:10E2100000A83A9B0A99359DCB1A19AEAFE5062F97
:10E2200028BF062727EAE773099704930B94DFF8C2
:10E230004CA2FFF79CB99DF8F730FFF76EB80B9A28
:10E240000798136804320B921860FEF72EBF3A99B4
:10E25000C81C01DB8F427ADA0F9A023A0F92013919
:10E260000F983A9100298DF8D800C0F2D1802B2365
:10E270008DF8D930092940F3A1800DF1E704139FEF
:10E28000204687FB0132CB17C3EBA20303EB8302CB
:10E29000A1EB420202F13005092B0246194600F8B3
:10E2A000015DEEDC3031C9B202F8021D944240F249
:10E2B000DF800DF1DA030DF1E60001E012F8011F35
:10E2C00003F8011B82421946F8D10A9836ABCB1AE3
:10E2D000179301280344099340F38880099B013375
:10E2E00023EAE3700021099304901191FDE6424670
:10E2F0002B463BAC43EC102B009408983CAC03211C
:10E300003A463AAB019400F063F9B9468246C41923
:10E310009AF80030302B02D03A9BE418BDE6404614
:10E32000294600220023FEF769FA0028F4D1C9F13A
:10E3300001033A93E418B0E63C9B9C4240F29B8078
:10E34000302203F8012BA3423C93FAD1AFE60A989E
:10E3500081423BDB039AD50753D54B1C23EAE3707C
:10E360006722099304900F92BEE60C900C999DF8D9
:10E37000F7300B9427EAE770049009971191FEF7A4
:10E38000CCBF0898059933AA01F0CAFE00287EF494
:10E3900040AF3A9F359D349C19AEF5E5002F08BF7C
:10E3A000012745E693460027FEF7B7BE07F10109AE
:10E3B00055E62D2305F100450C9342E6303130231C
:10E3C0008DF8DB108DF8DA3037A97EE700290A983E
:10E3D000D4BFC1F1020301231B1823EAE37209939E
:10E3E000672304920F937FE63C9C60E6039911F04B
:10E3F00001037FF473AF099A119322EAE272049247
:10E4000073E621EAE1736720049309910F906BE6AC
:10E410002D2349428DF8D9302CE70137CF1927EA4F
:10E42000E770099704905FE617B9039AD30713D5ED
:10E43000023727EAE7730997049355E60B9B1F6899
:10E44000191D002F9BF801300B919346BEF663AE69
:10E450004FF0FF37FEF75FBE01200490099043E6BE
:10E46000089A0C2313604FF0FF330793FEF7DABED0
:10E470000DF1DA0129E71C4619E600BF98EF010803
:10E480002DE9F04F02690B69934283B0804600F397
:10E490009B80DA1C92008F1882187E6852680136C1
:10E4A000B2FBF6F600F1140201F114055C1E04370C
:10E4B0000192002E49D04FF0000E1046F2462A4637
:10E4C000994652F804BB03681FFA8BFC4FEA1B4BBA
:10E4D00006FB0CEC06FB0BFE0EEB1C4E1AFA83FA45
:10E4E0001FFA8EFB1FFA8CFCCCEB0A0CCBEB134A09
:10E4F0000AEB2C4A1FFA8CFC4CEA0A43974240F87C
:10E50000043B4FEA1E4E4FEA2A4ADAD2201D08EB9E
:10E5100080024B46D2F804E0BEF1000F15D1DDF8C1
:10E5200004E096450FD258F8200060B96FEA0E005B
:10E53000023B8018A3EB900302E052F8040D10B9DF
:10E54000013C9C42F9D1C8F81040404601F0B8FCAB
:10E55000002835DB4FF0000C019B0136624655F870
:10E56000040B19681FFA80FC1FFA81F9000CCCEB30
:10E57000090C9444C0EB114202EB2C421FFA8CFCB4
:10E580004CEA02411214AF4243F8041BE7D2221DA9
:10E5900008EB8203596899B9019999420ED258F84B
:10E5A00022205AB9C943C91821F00301591A02E0BF
:10E5B00053F8042D12B9013C8B42F9D1C8F8104030
:10E5C000304603B0BDE8F08F0020FAE700000000FD
:10E5D0002DE9F04F9FB05BEC10AB0291016C049001
:10E5E000289D06920B9351B1436C012202FA03F26B
:10E5F0004B608A6001F074FA049C00232364BBF131
:10E600000004C0F2E58000232B6000231A46C7F601
:10E61000F073C7F6F0722340934200F0C2800023EB
:10E62000002250465946FEF7E9F856465F46012358
:10E6300090B913F0FF0F13D10B9D299C01232B6080
:10E64000002C00F0EA807C4C299D2C60013C059454
:10E6500005981FB0BDE8F08F002313F0FF0FEBD03B
:10E66000049847EC106B1DA91CAA01F0B3FCC4F37D
:10E670000A550D90002D40F0BA80DDF870801D9D88
:10E680006FF4826345449D42C0F2CA824FF60E4346
:10E69000CFF6FF7305F582625B1B023204FA03F3C7
:10E6A0002AFA02F01843FDF7CBFD0B460246CDE9EE
:10E6B0000823099B0124A3F1F873013D09931794E2
:10E6C00000230022C3F6F873DDE90801FDF77AFCA8
:10E6D00053A3D3E90023FDF729FE53A3D3E9002375
:10E6E000FDF772FC064628460F46FDF7B9FD50A31C
:10E6F000D3E90023FDF71AFE02460B4630463946A1
:10E70000FDF762FC06460F46FEF7AAF839460A9066
:10E71000002230460023FEF77BF850B10A98FDF73F
:10E720009FFD32463B46FEF769F810B90A9C013C52
:10E730000A940A9C162C00F25182404B03EBC4034E
:10E74000D3E9000152465B46FEF780F8002800F04E
:10E7500064820A9C013C0A9400241694C5EB0805C7
:10E76000B5F1010900F14682002507950A9C002CAD
:10E77000C0F237820025A14414941095029C092C04
:10E7800064D8052C40F34986043C02940026029D7F
:10E79000AB1E032B5CD8DFE813F0F903CC020604B0
:10E7A00003040B9D42F20F732B60BAF1000F15D0DA
:10E7B000234C0594299D002D3FF44AAF059CE37836
:10E7C000002B00F01A8104F10803299C23603FE725
:10E7D00024F0004401232B60A34616E7184B194A86
:10E7E000C4F31304002C18BF1A460592E2E7394619
:10E7F0003046CDE908010999DDF8708021F07F43AA
:10E8000023F4700343F07E53A5F57E7543F4E003D3
:10E8100000240993073D179452E70B4C059417E722
:10E8200061436F63A787D23FB3C8608B288AC63F16
:10E83000FB799F501344D33FA1EF0108D0EF0108AB
:10E84000C0EF0108B4EF0108A0EF01080024029412
:10E85000049D00246C642846214601F01BF94FF00A
:10E86000FF351595049D05902864012511954FF0FD
:10E87000FF350C9506941D9B002BC0F2C3800A9CAB
:10E880000E2C00F3BF805E4B03EBC40393ED007BC3
:10E89000069C002C8DED027BC0F28883DDE902230B
:10E8A00050465946FDF76CFEFDF7DAFF8046FDF74E
:10E8B000D7FCDDE90223FDF739FD059D0B46024635
:10E8C00059465046FDF77EFB08F130030C9C05F8D5
:10E8D000013B012C0E9582468B462F464BD00023E0
:10E8E0000022C4F22403FDF721FD0023002282460A
:10E8F0008B46FDF783FF0123002840F0188213F0B8
:10E90000FF0F6AD0059D0C98AC1C05EB00090EE0CA
:10E91000FDF70CFD0023002282468B46FDF76EFFBB
:10E920000134012300B1002313F0FF0F55D0DDE9BE
:10E93000022350465946FDF723FEFDF791FF80461E
:10E94000FDF78EFCDDE90223FDF7F0FC02460B46E5
:10E9500050465946FDF736FB08F130050F460023B7
:10E96000064600224C45BB46C4F2240304F8015C71
:10E97000B2462746CCD152465B4650465946FDF733
:10E9800023FB04460D462246DDE902012B46FDF736
:10E990003FFF48B9DDE9020122462B46FDF72EFF75
:10E9A000D8B118F0010F18D017F8015C3B460E9A49
:10E9B00002E013F8025C013B392D1F4640F0DC8475
:10E9C0009342F6D10E9D0A9C302305F8013C2B465C
:10E9D000013431220A9403F8012C04980D9901F0B6
:10E9E0007FF80A9D0B9C6B1C299D00223A702360C6
:10E9F000002D3FF42DAE2F602AE6059DEB1CE4E6CA
:10EA0000D0EF0108119D002D00F0FB80029C012C2D
:10EA100040F3FA820C9C651E109CAC42C0F2AD83A0
:10EA2000651B0C9C002CC0F29684079C0C9B079ADB
:10EA30000498D21801210792994401F0E9F8804620
:10EA400064B1B9F1000F09DD0798A145B4BF4B4689
:10EA50002346C01A0790E41AC3EB0909109900294C
:10EA60001ADD119A002A00F08183002D10DD414645
:10EA70002A46049801F078F9804641460D9A049898
:10EA800001F0D0F80D990646049801F029F80D968A
:10EA9000109B5A1B40F0A7820121049801F0B8F89E
:10EAA00005461498002805DD29460498149A01F0BB
:10EAB0005BF905460299012940F322810026149B47
:10EAC000002B40F02C8301234B4413F01F0300F074
:10EAD0009D80C3F12002042A40F3A2840798C3F169
:10EAE0001C03C0180790E4189944079A002A04DD13
:10EAF00004980D9901F084F90D90B9F1000F05DD2E
:10EB0000294604984A4601F07BF90546169B002BDE
:10EB100040F0ED820C98002840F30A8311980028F9
:10EB200040F08680C246119C0C9EDDF834B0059FF3
:10EB3000DDF8108006E0594640460A22002300F026
:10EB4000D9FF834629465846FFF79AFC00F1300961
:10EB500007F804900134A642EDDCD0460C9CDDF8A9
:10EB600014A0CDF834B0012CACBFA2440AF1010AC4
:10EB7000002601220D99049801F042F929460D90D2
:10EB800001F09EF9002840F334821AF8013C059CFC
:10EB9000621C03E01AF8023C0AF1FF3A392B57468F
:10EBA00040F04E839245F5D10A9C312301340A94FA
:10EBB00002F8013C0498294600F092FFB8F1000FDA
:10EBC0003FF40BAF2EB1464503D00498314600F018
:10EBD00087FF0498414600F083FFFEE60124169467
:10EBE000BCE50A9D079C641B07946C4200251094A9
:10EBF0001495C3E5C9F10009CDF81C904FF0000948
:10EC0000B4E5109D079CDDF8448019E71C230799A3
:10EC1000C9180791E418994467E7002416949DE504
:10EC20004FF6EE30CFF6FF70401B0AFA00F03AE5DF
:10EC3000002C05DD41460498224601F0E1F88046AB
:10EC4000002E40F001834446059F069546464FF04E
:10EC500001080AEA0801C146049D1091B8460D9FBB
:10EC600006993846FFF70CFC31460790384601F00C
:10EC700027F9224608900699284601F03FF9079A9D
:10EC800002F13003C2688246002A00F0CB81284698
:10EC90005146019300F024FF019B4FF0010B0898AF
:10ECA0000028C0F2838205D1029919B9109A002A6E
:10ECB00000F07C82BBF1000F00F3DD820C9808F8B5
:10ECC000013B8145C24600F0E28239460A22002318
:10ECD000284600F00FFFA642074600F0CB813146E0
:10ECE0000A220023284600F005FF214606460A2294
:10ECF0002846002300F0FEFE09F101090446AFE7B3
:10ED0000BAF1000F7FF4DAAECBF31303002B40F01F
:10ED10003083C7F6F0730BEA0303002B00F0528335
:10ED2000079A0132079209F101090126C7E600237B
:10ED3000E5E5002411940A9C069D2D1915950135D1
:10ED4000002D2C4640F32B820C9504980021172DA2
:10ED500041640AD9012204235B0003F11400114627
:10ED60000132A842F8D9049D6964049800F092FE2B
:10ED7000049D05900E2C28643FF67DAD002E3FF4D7
:10ED80007AAD0A9C002CCDE90EAB4BEC17ABCDE96C
:10ED900008AB40F33182A14B04F00F02241103EBC6
:10EDA000C203E106D3E900AB40F1EF819C4B51EC8B
:10EDB000170BD3E90823FDF7E3FBCDE90E0104F0BF
:10EDC0000F04032674B1964D50465946E20704D508
:10EDD000D5E90023FDF7AAFA013608356410F5D10C
:10EDE00082468B46DDE90E0152465B46FDF7C8FBC5
:10EDF000CDE90E01169C002C00F047810023DDE9CF
:10EE00000E010022C3F6F073FDF702FD002800F0AA
:10EE10003C810C9D002D00F0D882159C002C40F305
:10EE2000E58100230022C4F22403DDE90E01FDF791
:10EE30007DFACDE90E01701CFDF712FA02460B4671
:10EE4000DDE90E01FDF772FA00230022C4F21C0373
:10EE5000FDF7BAF804460A98DDF8548001381A9094
:10EE6000A1F15075119B002B00F019826B4B002112
:10EE700003EBC80353E902230020C3F6E071FDF75A
:10EE80007FFB22462B46FDF79DF8CDE91201DDE917
:10EE90000E01FDF7E5FC0546FDF7E2F902460B46DB
:10EEA000DDE90E01FDF78EF83035059CEDB28246A6
:10EEB0008B4604F8015BDDE9120152465B460E9475
:10EEC000FDF7C4FC0E9F002840F0748200215246DA
:10EED0005B460020C3F6F071FDF774F802460B465E
:10EEE000DDE91201FDF7B2FC002840F06782B8F1BD
:10EEF000010F40F37B81059D0E9ECDF86C90A844D8
:10EF0000CDF860800CE0FDF75DF8DDE91223FDF738
:10EF10007FFC002840F05282189CA64200F06481D9
:10EF200000230022C4F22403DDE91201FDF7FEF9FB
:10EF300000230022C4F22403CDE9120150465946B1
:10EF4000FDF7F4F989468046FDF78AFC0446FDF793
:10EF500087F902460B4640464946FDF733F8303400
:10EF6000E5B2DDE9122306F8015B8B468246FDF728
:10EF70004FFC0021044652465B460020C3F6F07168
:10EF80003746002CBFD01A9C0A9426E50024119421
:10EF9000069D002D40F3FB802C4615950C95D4E67C
:10EFA00001251195C7E601241194F1E70C9D002D70
:10EFB0003FF774AC40F0238200230022C4F2140314
:10EFC000DDE90201FDF7B2F952465B46FDF734FC7C
:10EFD0000C9DA846002800F0C080069C059FE443D5
:10EFE0000A940026E6E504980D9900F0BDFE0D9008
:10EFF00052E503D119F0010F7FF4C7AD57461AF857
:10F00000013D302BFAD0D5E5179D002D00F0AA81E7
:10F0100003F586630333109D079C08E5D0EF0108D4
:10F0200098F0010851463846019300F049FF5146D7
:10F030008346284600F054FD019BBBF1000F7FF48E
:10F040002EAE029800287FF42AAE109900297FF492
:10F0500026AE392B0D979946069D474600F0BE8097
:10F06000089B002B02DD079B03F13109A04607F83E
:10F07000019B9FE5314628460A22002300F03AFD15
:10F0800009F1010906460446EAE53046FDF7E8F8CD
:10F09000DDE90E23FDF74AF900230022C4F21C0328
:10F0A000FCF792FFA1F150750C990446002978D124
:10F0B00000230022C4F21403DDE90E01FCF782FFF5
:10F0C00022462B4682468B46FDF7C0FB06460028AB
:10F0D00040F0E280224605F1004350465946FDF7D4
:10F0E00097FB002800F082803546B04675E70D9802
:10F0F000294600F0E5FE0028BFF60CAD0D990498F6
:10F100000A22002300F0F6FC0D900A9811990138AC
:10F110000A90002940F07681159B0C93FAE42B6944
:10F1200005EB8303186900F027FDC0F12003CBE451
:10F13000029902297FF7F2AC00287FF44EAF052236
:10F1400003462946049800F0D5FC054629460D984B
:10F1500000F0B6FE00287FF740AF0A9C059F3123E0
:10F16000013407F8013B0A94002623E504980D9921
:10F17000109A00F0F9FD0D908EE4109C10952B1B59
:10F18000149CE418149400254BE402261AE601248A
:10F1900015940C940694049D00216964E5E50C9592
:10F1A000F9E70A9ADDF830801A925BE6BBF1000FAE
:10F1B0000D979946069D47467FF758AF01220D9956
:10F1C000049800F01DFE29460D9000F079FE0028FD
:10F1D00040F30E81B9F1390F7FF445AFBA463923B8
:10F1E0000AF8013BA046D2E4DDF86C90DDE90801A5
:10F1F00082468B46FFF73FBB0A9D6C42002C00F015
:10F20000AF808A4B04F00F0203EBC203DDE90E016D
:10F21000D3E90023FDF78AF82411CDE90E0100F0AF
:10F220009F80834D0226E30704D5D5E90023FDF72F
:10F230007DF8013608356410F5D1CDE90E01D9E528
:10F2400001330AF8013CB5E4D8F80410049800F042
:10F2500021FCD8F8102002320446920008F10C017B
:10F2600000F10C0000F0D0FB21460498012200F0D0
:10F27000C7FD0446E8E4392B0D979946069D47469D
:10F28000ACD003F1010907F8019BA04692E499462E
:10F290000D97069DA0466CE40025A8465DE76349EE
:10F2A00008F1FF3001EBC00122462B461290D1E954
:10F2B0000001FDF73BF8CDE91801DDE90E01FDF78E
:10F2C000CFFA0446FCF7CCFF059D0B460246DDE96C
:10F2D0000E01FCF777FE04F1300305F8013BB8F1AD
:10F2E000010F82468B460E952F461FD0059C631E4C
:10F2F000984400230022C4F22403FDF717F80F46B8
:10F300000646FDF7ADFA0546FCF7AAFF3035024682
:10F310000B4630463946FCF755FE04F8015F44457C
:10F32000E7D10E9D129C82468B462F1900230022A6
:10F33000C3F6E073DDE91801FCF746FE02460B4612
:10F3400050465946FDF782FAE0B11A9C17F8015C65
:10F350000A94FFF72BBB07980023041BFFF767BB3A
:10F36000022647E51C9B109D079CC3F13603FFF75F
:10F370005EBB5646FFF7A3BB6A1CD2B203F8012C52
:10F38000FFF72BBB0021DDE918230020C3F6E07155
:10F39000FCF718FE02460B4650465946FDF738FA70
:10F3A00000283FF423AF3B461F46013B17F8012CD2
:10F3B000302AF9D01A9D0A95FFF70FBB1A9C0A94C0
:10F3C000FFF7F4BA1E46FFF77ABB3046FCF748FF5A
:10F3D00002460B46DDE90E01FCF7A8FF00230022E0
:10F3E000C4F21C03FCF7F0FD0446A1F150755FE682
:10F3F0007FF43CAE19F0010F3FF438AEEAE6002589
:10F40000A846EAE541460A220498002300F072FB70
:10F41000159A80460C92FFF77DBB0126FFF7B7B91E
:10F420003FF463ABC3F13C03FFF7F1BBD0EF01083E
:10F4300098F00108AFF3008040F27C40C2F2000077
:10F44000704700BF2DE9F04F01F10B04162C83B07B
:10F45000054627D934F0070427D4A14225D82846E9
:10F4600000F014FBB4F5FC7F23D2B14E4FEAD40E6A
:10F4700006EBCE03DF689F4200F0D5817B68FA6817
:10F48000B96823F00303FB18CA605868916040F024
:10F4900001025A60284600F0FBFA0837384603B0EC
:10F4A000BDE8F08F1024A142D9D90C232B6000278E
:10F4B000F4E75FEA542E00F08880BEF1040F00F2FA
:10F4C00050814FEA941E0EF1380E4FEACE01984E4D
:10F4D0007118CF68B94205D10CE0002B7ADAFF68C9
:10F4E000B94207D07A6822F00302131B0F2BF4DD18
:10F4F0000EF1FF3E0EF1010E8D4A376902F1080C44
:10F50000674500F06E817B6823F00303191B0F2908
:10F5100000F354810029C2F814C0C2F810C067DAA1
:10F52000B3F5007F80F02B81DB0802EBC301D2F83A
:10F5300004808868F9609B104FF0010909FA03F311
:10F5400043EA0803B86053608F60C76001204FEA48
:10F55000AE0200FA02F0984254D8034206D12EF0CF
:10F56000030E400003420EF1040EFAD006EBCE0962
:10F570004F46F046FB689F4207D134E1002A80F2F3
:10F580005B81DB689F4200F02E81596821F0030106
:10F590000A1B0F2AF2DD1F461919D86857F808EF21
:10F5A0008A5044F0010442F00102CEF80C00C0F889
:10F5B00008E05C6071613161C1F80CC0C1F808C03D
:10F5C0004A60284600F064FA68E74FEAD40E4FEA32
:10F5D000CE017CE7BA18FB685068B96840F00100BA
:10F5E0005060CB609960284600F052FA083755E722
:10F5F000FB1828465A6842F001025A6000F048FAA7
:10F6000008374BE7B7687B6823F003094C4504D8FB
:10F61000C4EB09020F2A00F39780DFF824B1454BB1
:10F62000DBF800201B680132234400F0518103F510
:10F6300080530F3323F47E6323F01F0319462846BB
:10F64000019300F02BFDB0F1FF3F8046019B00F0DD
:10F650004A8107EB0901814200F20981DFF8E4A049
:10F66000DAF8002041451A44CAF8002000F0408131
:10F67000DBF80000013000F04B81C1EB08015218AB
:10F68000CAF8002018F0070200F00481C2F1080156
:10F69000C2F58052884402F1080B43441B051B0D40
:10F6A000C3EB0B0B2846594600F0F8FC431C00F056
:10F6B0003B81C8EB00035B4443F00103DAF8002010
:10F6C000C6F808805A44B742CAF80020C8F8043087
:10F6D00015D0B9F10F0F40F2EA807868A9F10C0358
:10F6E00023F00703F91800F0010E43EA0E0E05207F
:10F6F0000F2BC7F804E04860886000F20D810E4BC4
:10F70000B76819688A4288BF1A600C4B19688A4228
:10F7100088BF1A607A6822F00302944202D8121B52
:10F720000F2A11DC284600F0B3F90027B6E600BF27
:10F73000B40400204C0D0020480D0020440D002092
:10F74000C0080020500D00203B1942F0010244F097
:10F7500001047C6028465A60B360083700F098F9CD
:10F760009CE6BEF1140F76D9BEF1540F00F28880EA
:10F770004FEA143E0EF16E0E4FEACE01A7E65A0A8A
:10F78000042A6DD9142A00F2A58002F15B084FEA21
:10F79000C800301878498268824203D17DE09268BF
:10F7A000904204D0516821F003018B42F7D3D16815
:10F7B0007368F960BA60D7608F60C7E63B1941F0A3
:10F7C000010044F001047C60536113615860C3F888
:10F7D0000CC0C3F808C05950284600F059F9083742
:10F7E0005CE65368B2E608F10108083718F0030F29
:10F7F0007FF4C0AE4B461EF0030FA3F108020EF1DA
:10F80000FF3E00F0AA801B689342F4D0736840006A
:10F8100098423FF6F7AE00283FF4F4AE184200F0ED
:10F82000A180C646A2E607F108037F69BB427FF4C8
:10F8300025AE0EF1020E5FE659181F464868DB68D8
:10F8400057F8082F40F001004860D3609A602846BE
:10F8500000F01EF922E60EF15B0E4FEACE0136E60D
:10F860004FEA931808F138084FEAC80091E7B74209
:10F870003FF4F4AE404B9F687A6822F003024CE7F5
:10F88000BEF5AA7F19D84FEAD43E0EF1770E4FEAA3
:10F89000CE011CE64FF4805BFFE64B684FEAA808F8
:10F8A000012000FA08F003434B60114681E7012371
:10F8B000C8F80430474600222FE740F254539E45D3
:10F8C00021D84FEA944E0EF17C0E4FEACE01FEE5B0
:10F8D0001033B3E6542A2BD84FEA133808F16E08D8
:10F8E0004FEAC80055E7B7687A6822F0030214E7C8
:10F8F0000805000D00287FF4BBAEB1684B4443F00F
:10F9000001034B60FBE64FF47C714FF07E0EDEE5A9
:10F910001A4AC2F80080B5E607F10801284600F04F
:10F92000FDFC174B1A68EAE601234FF0000BC5E611
:10F93000B2F5AA7F06D84FEAD33808F177084FEA24
:10F94000C80026E740F254518A420FD84FEA934844
:10F9500008F17C084FEAC8001BE7736823EA00033C
:10F96000736054E7400008F1040857E74FF47C70D7
:10F970004FF07E080DE700BFB4040020C00800204F
:10F98000500D0020830770B4C9B211D0002A23D0D3
:10F9900003788B421ED00346013A05E0E2B113F82A
:10F9A000014F013A8C4215D0013010F0030FF5D110
:10F9B000032A13D882B103788B420BD0431C8218E0
:10F9C00003E013F8014B8C4204D0934200F1010094
:10F9D000F7D1002070BC70471046FBE741EA0126D2
:10F9E00046EA06460446043023687340A3F1013515
:10F9F00025EA030313F0803F03D1043A032AF1D828
:10FA0000D8E72046D6E700BF0F2AF0B43AD941EA3A
:10FA100000039B0738D10C460346154626681E6036
:10FA200066685E60A6689E60E668103DDE60103421
:10FA300010330F2DF2D8A2F1100424F00F0402F0BD
:10FA40000F021034032A00EB0403214411D90E469F
:10FA50001D46144656F8047B043C032C45F8047BF1
:10FA6000F8D8141F24F00304043402F00302091927
:10FA70001B192AB111F8014B013A03F8014BF9D1D6
:10FA8000F0BC70470346F4E70346F3E7704700BF56
:10FA9000704700BFC36C70B505460C464BB153F8B8
:10FAA000240078B1026843F8242000230361C36076
:10FAB00070BD0421212200F0B1FB0346E864002858
:10FAC000EDD170BD012101FA04F6721D92002846A5
:10FAD00000F0A4FB0028F4D044608660E5E700BF96
:10FAE00031B1C36C4A6853F82200086043F8221011
:10FAF000704700BFF0B50D4606460C6901F11400D1
:10FB000083B0002107681FFA87FC3F0C02FB0C330F
:10FB100002FB07F707EB13479BB203EB07430131E7
:10FB200040F8043B3B0C8C42ECDC3BB1AA689442AD
:10FB300007DA05EB8402013453612C61284603B0D7
:10FB4000F0BD6968019301313046FFF7A3FF2A69D0
:10FB5000023205F10C010746920000F10C00FFF79C
:10FB600053FF6968F26C019B52F82100286042F84B
:10FB700021503D46DDE700BF020C034616D10304C9
:10FB8000102013F07F4F01D108301B0213F0704F8B
:10FB900001D104301B0113F0404F01D102309B0012
:10FBA000002B02DB5B0003D4202070470020E8E735
:10FBB000013070470368024613F0070007D0D907E9
:10FBC0001FD498071FD49B0813600220704799B276
:10FBD00009B91B0C102013F0FF0F01D108301B0ACC
:10FBE000190701D104301B09990701D102309B0884
:10FBF000D90704D45B0801D120207047013013607D
:10FC00007047002070475B0813600120704700BFF9
:10FC100010B50C460121FFF73DFF0123446103614C
:10FC200010BD00BF2DE9F04F0F691569AF4287B0D5
:10FC30000C46924604DA3A4654462F468A46154602
:10FC4000A368616807EB050B9B45C8BF0131FFF74F
:10FC500021FF0BF1040100EB8103043300F11409CF
:10FC6000994502900491039306D203994B460022D2
:10FC700043F8042B9942FBD80AEB850504EB870770
:10FC80000AF1140A143514341437AA45019452D2D7
:10FC9000CDF814B0AB465AF8044BA5B2E5B1019AC1
:10FCA0004B46002152F8046B1C68B0B211FA84F183
:10FCB000360C240C05FB001005FB064101EB10413E
:10FCC00080B240EA0140090C97421C4643F8040BFD
:10FCD000E8D861605AF8044C240C26D0D9F800C04A
:10FCE000019B4E4661464D464FF0000800E0154628
:10FCF0001A8808EB114804FB02881FFA8CFC2A467C
:10FD00004CEA084042F8040B53F804CB56F8041FA1
:10FD10004FEA1C4C88B204FB0C0C0CEB184C9F42B5
:10FD20004FEA1C48E3D8C5F804C0D34509F10409DB
:10FD3000B1D8DDF814B0BBF1000F0DDD049A0299C3
:10FD400051F8223043B9039A131F02E053F8042DEF
:10FD500012B9BBF1010BF9D1029BC3F810B01846E0
:10FD600007B0BDE8F08F00BF12F003032DE9F041AA
:10FD70001546044688462DD1AD101DD0A76C2FB96D
:10FD800031E06D1018D03E68CEB13746E807F8D59F
:10FD900041463A462046FFF745FFB8F1000F17D01D
:10FDA000D8F80420E36C53F822106D10C8F8001046
:10FDB00043F822808046E6D14046BDE8F0813946CE
:10FDC0003A462046FFF72EFF386006600746DDE71B
:10FDD0008046D6E7013B094A52F823200023FFF76B
:10FDE00089FE8046C8E7204640F27121FFF710FFE8
:10FDF0000023A06407460360C8E700BFC0F0010805
:10FE00002DE9F84F91460A698B684FEA691707EBAD
:10FE1000020B0BF101059D420C460646496803DDC5
:10FE20005B0001319D42FBDC3046FFF733FE002FC3
:10FE300000F1140309DD002211460132BA4243F8F1
:10FE4000041BFAD100EB82031433226919F01F0955
:10FE500004EB820C04F114010CF1140C22D0C9F152
:10FE6000200A002200E03B46D1F800801F4608FA35
:10FE700009F848EA020247F8042B51F8042B8C4594
:10FE800022FA0AF2EFD85A600AB10BF10205F36CBC
:10FE9000626853F82210013D0561216043F8224059
:10FEA000BDE8F88F51F8042B8C4543F8042BEED9AC
:10FEB00051F8042B8C4543F8042BF3D8E7E700BF37
:10FEC00003460A690069801A30B40FD104329400E5
:10FED0001A19091914330432043152F8045C51F828
:10FEE000044D043AA54203D19342F6D330BC704787
:10FEF00001D30120FAE74FF0FF30F7E72DE9F04793
:10FF00000C460746114620461546FFF7D9FF002844
:10FF1000064656D050DB002661683846FFF7BAFD2A
:10FF200027692B69C66004EB870C05EB83080CF18D
:10FF3000140C08F114081434143500F114090026C7
:10FF400054F8043B55F8042B16FA83F11FFA82FA91
:10FF5000120CC2EB1346CAEB010106EB21464B46DD
:10FF600089B241EA064143F8041B3614A8452246EB
:10FF70009946E5D8A445984614D952F8045B16FA78
:10FF800085F62D0C05EB2645B6B246EA05412E1442
:10FF9000944543F8041BF0D8E343634423F0030380
:10FFA0000433434429B9043B53F8042D013F002A8C
:10FFB000FAD00761BDE8F087234601262C461D468E
:10FFC000AAE738463146FFF765FD01230361466124
:10FFD000BDE8F0872DE9F04355EC104B83B00E4699
:10FFE00001211746FFF756FD25F07F4323F47003E8
:10FFF000C5F30A5980460193B9F1000F02D043F4CA
:020000040801F1
:1000000080130193002C26D002A840F8084D6846C2
:10001000FFF7D0FD019B002833D1009AC8F81420C7
:10002000002B0CBF01240224C8F81830C8F8104077
:10003000B9F1000F1CD108EB8402A0F58663023BE6
:1000400010693360FFF798FDC0EB44143C604046F4
:1000500003B0BDE8F08301A8FFF7ACFD019B0124CC
:10006000C8F81430C8F810402030B9F1000FE2D0C1
:10007000A9F58663033B1B18C0F135003360386077
:10008000E5E7C0F12002009903FA02F20A4323FADD
:1000900000F3C8F814200193C2E700BF38B5074C3D
:1000A0000023054608462360F3F782FD431C00D079
:1000B00038BD2368002BFBD02B6038BD780D0020A5
:1000C00020F0030110F00300C0F1000051F8043BE0
:1000D00000F1040C4FEACC0C6FF000021CBF22FAB6
:1000E0000CF213434FF0010C4CEA0C2C4CEA0C4C74
:1000F000A3EB0C0222EA030212EACC1204BF51F86D
:10010000043B0430F4D013F0FF0F1FBF013013F491
:100110007F4F013013F47F0F18BF0130704700BFCD
:100120002DE9F04F83B091460190906817680D4615
:10013000002871D04FF0000A08688B685446B4B1AB
:100140009C421E46984617D22646A0464246514635
:1001500000F0ACF9D9F80820AB6828689B1B404434
:10016000141BAB602860C9F80840002C4ED0D7F8AB
:1001700000A07C680837E2E7AB8913F4906FE5D004
:100180006E69296906EB4606C1EB000806EBD676D8
:10019000601C76104044864232463CBF06463246DA
:1001A0005B0501981AD51146FFF74CF98346F0B16B
:1001B00029694246FFF728FCAB8923F4906343F09A
:1001C0008003AB81C8EB06030BEB08006E61C5F83A
:1001D00010B028602646AB60A046B7E700F006FAEC
:1001E00083460028EED12969019800F097F8019A1A
:1001F0000C231360AA89002342F04002AA814FF029
:10020000FF30C9F80830C9F8043002E0C9F80440EA
:10021000204603B0BDE8F08F5060FAE710B501FB4F
:1002200002F1FFF70FF90446D8B150F8042C22F080
:100230000302043A242A18D8132A14D900231B2AAB
:100240000360436016D9242A8360C36011BF00F1A4
:1002500010020361436100F1180200231360536030
:100260009360204610BD0246F7E7002100F076F9C2
:10027000204610BD00F10802EFE700BFF8B5244D9D
:1002800004460F46FFF702FCAB685E6826F00306E3
:1002900006F57E630F33DF1B3F0B013F3F03B7F5CE
:1002A000805F20461CDB0021FFF7F8FEAB689B193E
:1002B000984219D02046FFF7EBFB0020F8BD002143
:1002C0002046FFF7EBFEAB68C21A0F2A07DD114983
:1002D0000968401A104942F0010208605A6020463D
:1002E000FFF7D6FB0020F8BD79422046FFF7D6FE87
:1002F0000130E4D0084BAA681968F61B46F00106E5
:10030000CF1B204656601F60FFF7C2FB0120F8BDDF
:10031000B4040020C0080020500D00202DE9F04159
:100320000D460446002958D0FFF7B0FB55F8040CE1
:100330005A4EA5F1080120F00103CA18D6F808C0EA
:100340005768944527F0030765D010F00100576007
:1003500032D00020D5196D6815F0010F06D1DB19D8
:10036000956800284BD0D268EA60956043F001029E
:100370004A60CB50D8B9B3F5007F30D35A0A042A6B
:1003800064D89D093835E80086194448B268B242FD
:1003900003D161E09268964204D0506820F00300D7
:1003A0008342F7D3D368CB608A60D16099602046DE
:1003B000BDE8F041FFF76CBB55F808CCCCEB010170
:1003C00006F108088D68454563443DD0D1F80CC05E
:1003D000C5F80CC0CCF80850BCE7BDE8F081DB08DC
:1003E00006EBC30275689068CA609B10012707FA84
:1003F00003F32B43886073609160C160D7E7284F97
:10040000BD42B0D143F0010271613161CD608D60B8
:100410004A60CB50CBE7C2073B4407D455F8082CC1
:10042000891A9B188868CA68C26090601D4AB160CA
:10043000126843F0010093424860B8D31A4B20463B
:100440001968FFF71BFFB2E7012083E7142A0CD8D5
:1004500002F15B05E80097E74368AD10012606FA54
:1004600005F52B43436013469DE7542A03D81D0B23
:100470006E35E80088E7B2F5AA7F03D8DD0B773543
:10048000E80081E740F25450824203D89D0C7C354D
:10049000E80079E74FF47C707E2575E7B40400200E
:1004A000BC040020BC0800204C0D00208842F0B4A1
:1004B00012D98D18A8420FD262B151421346821848
:1004C0006D185218EC18D11814F8014C013B01F8C2
:1004D000014CF7D1F0BC70470F2A3AD941EA00032A
:1004E0009B0738D10C460346154626681E60666891
:1004F0005E60A6689E60E668103DDE6010341033D2
:100500000F2DF2D8A2F1100424F00F0402F00F0214
:100510001034032A00EB0403214411D90E461D4672
:10052000144656F8047B043C032C45F8047BF8D8A9
:10053000141F24F00304043402F0030209191B19E8
:10054000002AC7D011F8014B013A03F8014BF9D149
:10055000C0E70346F4E70346F4E700BF10F0030FDB
:1005600070B403463FD0002A3BD0CDB201E0002A50
:1005700037D003F8015B013A13F0030F1C46F6D1A4
:10058000032A28D9CDB245EA05250F2A45EA0545B3
:1005900013D923461646103E1D605D609D60DD60E8
:1005A00010330F2EF7D8A2F1100323F00F0302F03F
:1005B0000F021033032A1C440DD926461346043B70
:1005C000032B46F8045BFAD8131F23F0030304330C
:1005D00002F00302E41822B1C9B2013A04F8011B87
:1005E000FBD170BC70470446CAE700BF2DE9F04F4D
:1005F0000C4683B006469346002900F0C4800BF1F8
:100600000B05FFF743FA162D54F8042C52D810218D
:100610000D46AB4553D822F003098945A4F1080AD9
:1006200051DA8C4BD3F808C00AEB0900844500F07E
:10063000B080476827F0010E8644DEF804E01EF023
:10064000010F57D04FF0000E7046D20775D454F802
:10065000082CC2EB0A08D8F8042022F00302002874
:1006600067D0604502EB090C00F0F6800EEB0C073A
:100670008F4260DBC3688268C2469A60D360D8F854
:100680000C305AF8081FA9F10402242ACB609960A3
:1006900000F22E81132A40F2BA802368C8F808308D
:1006A00063681B2AC8F80C3000F23B8108F1100384
:1006B0000834ADE025F00705002D2946A9DA0C2302
:1006C0003360002712E04F467B1B0F2B1DD802F032
:1006D00001020AEB07031743CAF804705A6842F094
:1006E00001025A603046FFF7D3F92746384603B077
:1006F000BDE8F08F27F0030E0EEB09078F42A4DB55
:10070000C3688168CB609960DEE70AEB050102F0FF
:100710000102C818154343F00103CAF804504B60A6
:10072000436843F00103436008313046FFF7F6FDAC
:10073000D8E702EB090C8C4537DA30465946FEF70C
:1007400081FE0746D8B154F8042C22F00103A0F131
:1007500008015344994200F0C580A9F10402242AFB
:1007600074D8132A48D80346224611681960516884
:10077000596092689A6030462146FFF7CFFD3046B7
:10078000FFF786F9B2E7114603B0BDE8F04FFEF778
:1007900059BEDCF8040020F0030E0EEB090005F151
:1007A0001007B8423FDA60464FE74746D8F80C30AA
:1007B00057F8081FA9F10402242ACB60996000F2BF
:1007C000A280132A40F29D802368C8F8083063682D
:1007D0001B2AC8F80C3000F2B98008F11003083465
:1007E00022681A6062685A60A2689A603C46D8F82B
:1007F00004206746C24667E72368036063681B2AD4
:10080000436064D800F1080304F10802ADE75346E1
:1008100022681A6062685A60A2689A605446D8F8E2
:100820000420C24650E70AEB0502411B41F00101DA
:10083000516054F8041C9A6001F001031D4344F810
:10084000045C3046FFF724F927464FE72146FFF7BF
:100850002DFE90E7B4040020E64405F11002964511
:10086000CDF804E0FFF667AF4746D8F80C1057F80C
:10087000080FA9F10402242AC160886000F2888070
:10088000132A79D92168C8F8081061681B2AC8F8AA
:100890000C1000F2848008F1100208342168116005
:1008A00061685160A1689160019808EB0502411BE5
:1008B00041F001015160D8F804109A6001F0010381
:1008C0001D43C8F804503046FFF7E2F80EE7A3686E
:1008D0008360E368242AC3602FD000F1100304F181
:1008E000100242E750F8047C27F003074F44EBE680
:1008F00021465046FFF7DAFD5446D8F80420C24698
:10090000E2E63B466CE721463846CDF800C0FFF7EB
:10091000CDFDDDF800C0D8F804203C46C24667464D
:10092000D2E6A368C8F81030E368242AC8F8143067
:1009300018D008F1180310346AE72369036162696B
:1009400000F11803426104F118020EE7A368C8F829
:100950001030E368242AC8F814300FD008F11803C7
:1009600010343DE72369C8F81830626908F12003A4
:10097000C8F81C2018344BE73A468FE72369C8F8BB
:100980001830626908F12003C8F81C20183427E7E2
:10099000384621460093FFF789FD009B84E7A16854
:1009A000C8F81010E168242AC8F8141003D008F120
:1009B0001802103472E72269C8F81820616908F13A
:1009C0002002C8F81C10183468E700BF4BB942B9C0
:1009D000002908BF002802D04FF0FF310846FBF77E
:1009E000FFBF82B0EC462DE90050FBF7E3FFDDF8D6
:1009F00004E002B00CBC70472E2E5C7379737465F2
:100A00006D5C7372635C73746D333266342D686130
:100A10006C5C73746D3332663478785F68616C5FD8
:100A200074696D2E630000002E2E5C7379737465FB
:100A30006D5C7372635C73746D333266342D686100
:100A40006C5C73746D3332663478785F68616C5FA8
:100A50007370692E630000000000000001020304AF
:100A600001020304060708092E2E5C73797374656E
:100A70006D5C7372635C73746D333266342D6861C0
:100A80006C5C73746D3332663478785F68616C5F68
:100A90007263632E630000002E2E5C73797374659D
:100AA0006D5C7372635C73746D333266342D686190
:100AB0006C5C73746D3332663478785F68616C5F38
:100AC0006770696F2E6300002E2E5C7379737465F6
:100AD0006D5C7372635C73746D333266342D686160
:100AE0006C5C73746D3332663478785F68616C5F08
:100AF0006461632E630000002E2E5C73797374654D
:100B00006D5C7372635C73746D333266342D68612F
:100B10006C5C73746D3332663478785F68616C5FD7
:100B2000636F727465782E63000000002E2E5C7374
:100B3000797374656D5C7372635C73746D33326664
:100B4000342D68616C5C73746D3332663478785F11
:100B500068616C5F6164632E630000002C20667521
:100B60006E6374696F6E3A200000000000000000A0
:100B7000617373657274696F6E202225732220661B
:100B800061696C65643A2066696C65202225732270
:100B90002C206C696E65202564257325730A00007E
:100BA0006173736572745F706172616D282920666C
:100BB00061696C65643A2066696C65202225732240
:100BC0002C206C696E652025640A000061626F72DA
:100BD0007428292C2065786974696E672E2E2E0082
:100BE00048656C6C6F2041524D20576F726C6421C8
:100BF0000000000053797374656D20636C6F636B44
:100C00003A202575487A0A002538640025346400A6
:100C1000252D3464000000000000000000000000EA
:100C20000000000000003603FFFFFFFFFFFFFFFF93
:100C3000FFFFFFFFFFFFFFFFFFFFFFFFFFFFFFFFC4
:100C4000F6FF00600000000000000000000000004F
:100C50000000000000003603FFFFFFFFFFFFFFFF63
:100C6000FFFFFFFFFFFFACFD0000000000000000E1
:100C70000000000000003603FFFFFFFFFFFFFFFF43
:100C8000FFFFFFFFFFFFFFFFFFFFFFFFFFFFFBFF78
:100C9000C091000000000000000000000000000003
:100CA0003603FFFFFFFFFFFFFFFFFFFFFFFFFFFF19
:100CB000FFFFFFFFFFFFFFFFFFFFFFFFD2FE003838
:100CC0000000000000000000000000000000000024
:100CD0000000BF65FFFFFFFFFFFFFFFFFFFFFFFFFC
:100CE000FFFFFFFFFFFFFFFFFFFFFFFFFFFFFFFF14
:100CF00020B3000000000000000000000000BF65FD
:100D0000FFFFFFFFFFFFFFFFFFFFFFFFFFFFFFFFF3
:100D1000FFFFFFFFFFFF20B3000000000000000006
:100D20000000BF65FFFFFFFFFFFFFFFFFFFFFFFFAB
:100D3000FFFFFFFFFFFFFFFFFFFFFFFFFFFFD2FEF1
:100D4000003800000000000000000000BF65FFFF49
:100D5000FFFFFFFFFFFFFFFFFFFFFFFFFFFFFFFFA3
:100D6000FFFFFFFFFFFFFFFFFFFFFBFFC091000042
:100D70000000000000000000000000000C00FFB7B1
:100D8000FFFFFFFFFFFFFFFFFFFFFFFFFFFFFFFF73
:100D9000FFFFFFFFFFFFFFFFFFFFFFFFD2FE003857
:100DA000000000000000D201FFDFFFFFFFFFFFFF98
:100DB000FFFFFFFFFFFFFFFFFFFFFFFFFFFFFFFF43
:100DC000FFFFF6FF00600000000000000C00FFB70E
:100DD000FFFFFFFFFFFFFFFFFFFFFFFFFFFFFFFF23
:100DE000FFFFFFFFFFFFFFFFFFFFFFFF87DC0000AC
:100DF0000000000000000C00FFB7FFFFFFFFFFFF37
:100E0000FFFFFFFFFFFFFFFFFFFFFFFFFFFFFFFFF2
:100E1000FFFFFFFFFFFFFFFFACFD00000000000031
:100E200000000000000000003603FFFFFFFFFFFF8F
:100E3000FFFFFFFFFFFFFFFFFFFFFFFFFFFFFFFFC2
:100E4000FFFFFFFFFFFFFFFFF6FF00600000000055
:100E50000C00FFB7FFFFFFFFFFFFFFFFFFFFFFFFDC
:100E6000FFFFFFFFFFFFFFFFFFFFFFFFFFFFFFFF92
:100E700020B30000000000003603FFFFFFFFFFFF6C
:100E8000FFFFFFFFFFFFFFFFFFFFFFFFFFFFFFFF72
:100E9000FFFFFFFFFFFFFFFFF6FF00600000000005
:100EA00000003603FFFFFFFFFFFFFFFFFFFFFFFF15
:100EB000FFFFFFFFFFFFFFFFFFFFFFFFFFFFFFFF42
:100EC000FFFFFFFFD2FE003800000000000000001E
:100ED0000000000000000000000000000000000012
:100EE0000000000000000000BF65FFFFFFFFFFFFE4
:100EF000FFFFFFFFF6FF006000000700DF96FFFF27
:100F0000FFFFFFFFFFFFFBFFC091000000000C0090
:100F1000FFB7FFFFFFFFFFFFFFFFFFFF20B3000052
:100F200000000000000000000000000000000000C1
:100F30000000000000000700DF96FFFFFFFFFFFF3B
:100F4000FFFFFFFFFBFFC09100000000000000005A
:100F50000000000000000000000000000000000091
:100F600000000700DF96FFFFFFFFFFFFFFFFFFFF0F
:100F7000ACFD0000000000000000000000000000C8
:100F80000000000000000000000000000000000061
:100F9000000000003603FFFFFFFFFFFFFFFFFFFF22
:100FA000ACFD000000003603FFFFFFFFFFFFFFFF67
:100FB000FFFF20B300000000000000009B3CFFFF8B
:100FC000FFFFFFFFFFFFFBFFC091000000000000DC
:100FD0000000000000000000000000000000000011
:100FE000000000000C00FFB7FFFFFFFFFFFFFFFF47
:100FF000FBFFC091000000000000000000000000A6
:1010000000000000000000000000000000000000E0
:10101000BF65FFFFFFFFFFFFFFFFFFFF87DC000053
:10102000000000000000000000003603FFFFFFFF8B
:10103000FFFFFFFFFFFFACFD00000000000000000D
:10104000BF65FFFFFFFFFFFFFFFFFFFF20B30000B3
:1010500000009B3CFFFFFFFFFFFFFFFFFFFFF6FFCE
:101060000060000000000000000000000000000020
:10107000000000000000000000003603FFFFFFFF3B
:10108000FFFFFFFFFFFFACFD0000000000000000BD
:101090000C00FFB7FFFFFFFFFFFFFFFFFBFFC0914B
:1010A000000000003603FFFFFFFFFFFFFFFFFFFF11
:1010B000ACFD00000000000000000C00FFB7FFFFC7
:1010C000FFFFFFFFFFFFF6FF0060000000000000D1
:1010D000000000000000BF65FFFFFFFFFFFFFFFFF4
:1010E000FFFF20B3000000000700DF96FFFFFFFFB7
:1010F000FFFFFFFFFFFFD2FE003800000000BF65CA
:10110000FFFFFFFFFFFFFFFFFFFFFFFFFFFFFFFFEF
:10111000FFFFACFD00000000000000000000000028
:10112000000000000000BF65FFFFFFFFFFFFFFFFA3
:10113000FFFF20B300000000000000000C00FFB71C
:10114000FFFFFFFFFFFFFFFFF6FF00600000000052
:10115000BF65FFFFFFFFFFFFFFFFFFFF20B30000A2
:10116000000000000C00FFB7FFFFFFFFFFFFFFFFC5
:10117000FFFF87DC0000000000000000000000000E
:101180000C00FFB7FFFFFFFFFFFFFFFFFFFFFFFFA9
:10119000FFFFFFFFFFFFFFFFFFFFFFFFFFFFFFFF5F
:1011A000FBFFC0910000000000009B3CFFFFFFFF21
:1011B000FFFFFFFFFFFFFFFFFFFFFFFFFFFFFFFF3F
:1011C000FFFFFFFF20B30000000000000000000050
:1011D0000C00FFB7FFFFFFFFFFFFFFFFF6FF006000
:1011E00000000000000000003603FFFFFFFFFFFFCC
:1011F000FFFFFFFFACFD000000000C00FFB7FFFF8A
:10120000FFFFFFFFFFFFFFFFFFFFFFFFFFFFFFFFEE
:10121000FFFFFFFFFFFFFFFFFFFFFFFFACFD000031
:101220000000000000000000000000003603FFFF87
:10123000FFFFFFFFFFFFFFFFFFFFFFFFFFFFFFFFBE
:10124000FFFFFFFFFFFFFFFFFFFFFFFF20B30000D7
:101250000000000000000700DF96FFFFFFFFFFFF18
:10126000FFFFFFFFFFFFFFFFFFFFFFFFFFFFFFFF8E
:10127000FFFFACFD00000000000000003603FFFF90
:10128000FFFFFFFFFFFFFFFFACFD000000000000BD
:10129000000000009B3CFFFFFFFFFFFFFFFFFFFF81
:1012A00087DC000000003603FFFFFFFFFFFFFFFFAA
:1012B000FFFFFFFFFFFFFFFFFFFFFFFFFFFFFFFF3E
:1012C000FFFFFFFFFFFFACFD00000000000000007B
:1012D0000000000000000000BF65FFFFFFFFFFFFF0
:1012E000FFFFFFFFFFFFFFFFFFFFFFFFFFFFFFFF0E
:1012F000FFFFFFFFF6FF006000000000000000009D
:101300000000000000009B3CFFFFFFFFFFFFFFFF0E
:10131000FFFFFFFFFFFFFFFFFFFFFFFFFFFFFBFFE1
:10132000C091000000000000BF65FFFFFFFFFFFF4E
:10133000FFFFFFFF20B300000000000000000700D7
:10134000DF96FFFFFFFFFFFFFFFFFBFFC0910000E5
:101350000000BF65FFFFFFFFFFFFFFFFFFFFFFFF75
:10136000FFFFFFFFFFFFFFFFFFFFFFFFFFFFF6FF96
:10137000006000000000000000000000000000000D
:1013800000000C00FFB7FFFFFFFFFFFFFFFFFFFFA5
:10139000FFFFFFFFFFFFFFFFFFFFFFFFD2FE003851
:1013A000000000000000000000000000000000003D
:1013B0000000000000000C00FFB7FFFFFFFFFFFF71
:1013C000FFFFFFFFFFFFFFFFFFFFFFFF87DC0000C6
:1013D00000000C00FFB7FFFFFFFFFFFFFFFFF6FF5E
:1013E000006000000000000000003603FFFFFFFF68
:1013F000FFFFFFFFFFFFACFD000000000C00FFB788
:10140000FFFFFFFFFFFFFFFFFFFFFFFFFFFFFFFFEC
:10141000FFFFFFFFFFFFFFFF20B300000000000001
:101420000000000000000000000000000000360383
:10143000FFFFFFFFFFFFFFFFFFFFACFD000000000D
:10144000000000000000000000000000000000009C
:10145000000000000000000000000000000000008C
:1014600000000000000000000000BF65FFFFFFFF5C
:10147000FFFFFFFFFFFFFFFF20B300000000360368
:10148000FFFFFFFFFFFFFFFFFFFFACFD00000000BD
:10149000000000000000BF65FFFFFFFFFFFFFFFF30
:1014A000FFFF20B3000000003603FFFFFFFFFFFF38
:1014B000FFFFFFFFACFD00003603FFFFFFFFFFFF54
:1014C000FFFFFFFFFFFF87DC0000000000000000BF
:1014D00000000000000000000000BF65FFFFFFFFEC
:1014E000FFFFFFFFFFFF20B300000000000000002F
:1014F00000000000000000000000000000000000EC
:10150000BF65FFFFFFFFFFFFFFFFFBFFC091000074
:101510000000000000000700DF96FFFFFFFFFFFF55
:10152000FFFFFBFFC09100000000BF65FFFFFFFF52
:10153000FFFFFFFFFFFF20B30000000000000000DE
:10154000D201FFDFFFFFFFFFFFFFFFFFD2FE0038EA
:1015500000000000BF65FFFFFFFFFFFFFFFFFFFF71
:1015600020B300000C00FFB7FFFFFFFFFFFFFFFFEE
:10157000FFFFD2FE00380000000000000000000065
:10158000000000000C00FFB7FFFFFFFFFFFFFFFFA1
:10159000F6FF0060000000000000000000000000F6
:1015A000000000000000000000000700DF96FFFFC1
:1015B000FFFFFFFFFFFFFBFFC091000000000000E6
:1015C0000000D201FFDFFFFFFFFFFFFFFFFFACFDC9
:1015D000000000000C00FFB7FFFFFFFFFFFFFFFF51
:1015E000F6FF00600000000000000C00FFB7FFFFE6
:1015F000FFFFFFFFFFFFFBFFC091000000000C009A
:10160000FFB7FFFFFFFFFFFFFFFFF6FF00600000D7
:101610000000BF65FFFFFFFFFFFFFFFFFFFFFBFFB6
:10162000C091000000000000000000000000000069
:101630003603FFFFFFFFFFFFFFFFFFFFACFD0000D2
:10164000000000000000000000000000000000009A
:101650000000000000000700DF96FFFFFFFFFFFF14
:10166000FFFFFFFFD2FE003800000000D201FFDFC5
:10167000FFFFFFFFFFFFFFFFFBFFC0910000000027
:101680003603FFFFFFFFFFFFFFFFFFFFACFD000082
:1016900000000000D201FFDFFFFFFFFFFFFFFFFFA1
:1016A000FFFF87DC0000000000003603FFFFFFFFA4
:1016B000FFFFFFFFFFFFACFD0000000000009B3CB0
:1016C000FFFFFFFFFFFFFFFFFFFFFFFF20B3000053
:1016D000000000000000000000000000BF65FFFFE8
:1016E000FFFFFFFFFFFFFFFF20B30000000000002F
:1016F00000000000000000000000000000000000EA
:1017000000000700DF96FFFFFFFFFFFFFFFFFFFF67
:10171000FFFFFFFFFFFFFFFFFFFFFFFFFFFFFFFFD9
:10172000FFFFFFFF20B3000000000000BF65FFFFC8
:10173000FFFFFFFFFFFFFFFFFFFFFFFFFFFFFFFFB9
:10174000FFFFFFFFFFFFFFFFFFFFFFFF87DC000042
:10175000000000000000BF65FFFFFFFFFFFFFFFF6D
:10176000FFFF20B30000000000003603FFFFFFFF73
:10177000FFFFFFFFFFFFFFFF87DC0000000000000E
:10178000000000000000D201FFDFFFFFFFFFFFFFAE
:10179000FFFFD2FE00380000000000000000000043
:1017A0000000000000000000000000000000000039
:1017B0009B3CFFFFFFFFFFFFFFFFFFFFFFFFFFFF60
:1017C000FFFFFFFFFFFFFFFFFFFFFFFFFBFFC091DA
:1017D000000000000000D201FFDFFFFFFFFFFFFF5E
:1017E000FFFFFFFFFFFFFFFFFFFFFFFFFFFFFFFF09
:1017F000FFFFFFFFFFFF20B300000000000000001C
:10180000D201FFDFFFFFFFFFFFFFFFFFD2FE003827
:10181000000000000000D201FFDFFFFFFFFFFFFF1D
:10182000FFFFFFFFACFD0000000000000000000013
:1018300000009B3CFFFFFFFFFFFFFFFFFFFF87DC78
:101840000000000000000000000000000000000098
:101850000000000000000000000000000000BF6564
:10186000FFFFFFFFFFFFFFFFFFFFFFFFFFFFFFFF88
:10187000FFFFFFFFFFFFACFD0000000000000000C5
:1018800000009B3CFFFFFFFFFFFFFFFFFFFFFFFF8D
:10189000FFFFFFFFFFFFFFFFFFFFFFFFFFFFF6FF61
:1018A0000060000000000000000000009B3CFFFF03
:1018B000FFFFFFFFFFFFFFFF87DC000000000000CD
:1018C00000000C00FFB7FFFFFFFFFFFFFFFFFFFF60
:1018D000D2FE003800000000000000000700DF9684
:1018E000FFFFFFFFFFFFFFFFFBFFC09100000000B5
:1018F00000000000000000000000000000000000E8
:101900000000000000000000000000000C00FFB715
:10191000FFFFFFFFFFFFFFFFFFFFFFFFFFFF20B302
:101920000000000000000000000000000700DF963B
:10193000FFFFFFFFFFFFFFFFFFFFFFFFFFFFFFFFB7
:10194000FFFFFFFFFFFF87DC00000000000000003A
:101950000000000000000700DF96FFFFFFFFFFFF11
:10196000FFFFFBFFC0910000000000000000070027
:10197000DF96FFFFFFFFFFFFFFFFFFFFF6FF0060A7
:10198000000000000000000000000000EF7BFFFFEF
:10199000FFFFFFFFFFFFFFFFFFFFFFFFFFFFFFFF57
:1019A000FFFFFFFFFFFFFFFFFFFFFFFFFFFFFFFF47
:1019B000FFFFFFFFFFFFFFFFFFFFFFFFFFFFFFFF37
:1019C000FFFFFFFFFFFFFFFFFFFFFFFFFFFFFFFF27
:1019D000FFFFEF7B000000000000FFFFFFFFFFFFA5
:1019E000FFFFFFFFFFFFFFFFFFFFFFFFFFFFFFFF07
:1019F000FFFFFFFFFFFFFFFFFFFFFFFFFFFFFFFFF7
:101A0000FFFFFFFFFFFFFFFFFFFFFFFFFFFFFFFFE6
:101A1000FFFFFFFFFFFFFFFFFFFFFFFFFFFFFFFFD6
:101A2000FFFFFFFFFFFF0000EF7BFFFFACFD0000AB
:101A300000000C00FFB7F6FF006000000000BF656B
:101A4000FFFFFFFF20B3000000000000D201FFDF16
:101A5000FFFFF6FF00600000000000000000D20160
:101A6000FFDFFFFFD2FE0038000000000000000092
:101A70000000BF65FFFFEF7BFFFFFFFFACFD000035
:101A800000000700DF96D2FE003800000000BF65AE
:101A9000FBFFC09100000000000000000000D20128
:101AA000FFDFF6FF00600000000000000000000003
:101AB000D201FFDFD2FE003800000000000000006D
:101AC0000000BF65FFFFFFFFFFFFFFFFACFD000051
:101AD000000000009B3CACFD0700C0390000BF6562
:101AE000ACFD00000000BF65FFFFACFD0000000082
:101AF000BF65F6FF006000009B3CFFFFACFD0000EF
:101B00000700DF96D2FE00380000BF65FFFFFFFF31
:101B1000FFFFFFFFFFFFFFFFFFFFFFFFACFD000028
:101B2000CC01C061360320B30C0020630000BF6508
:101B300087DC00000C00FFB7FFFFFBFFC091000037
:101B40009B3CF6FF006000009B3CFFFFF6FF00603F
:101B50000000BF65D2FE0038000000000000000059
:101B60000700DF96FFFFFFFFFFFFFFFFACFD000058
:101B7000D20120930700C039360320B30000BF65AF
:101B800087DC00000C00FFB7FFFFFBFFC0910000E7
:101B90009B3CF6FF006000009B3CFFFFF6FF0060EF
:101BA0000000BF65D2FE0038000000000000000009
:101BB0000700DF96FFFFFFFFFFFFFFFFACFD000008
:101BC000D20187B4000000009B3C20B30000BF6539
:101BD000ACFD00000000BF65FFFFACFD0000000091
:101BE000BF65F6FF006000009B3CFFFFACFD0000FE
:101BF0000000BF65D2FE00380000BF65FFFFFFFF99
